:020000022000DC
:10600000F0FF032039630200616302006363020052
:10601000656302006763020069630200000000001C
:106020000000000000000000000000006B630200A0
:106030006D630200000000006F630200F579040048
:10604000352803007363020031CD020085D40200BD
:106050001DCE02007363020069D50200F929030016
:1060600073630200ADAD040073630200736302004A
:1060700073630200992803007363020073630200D4
:10608000357A0400B1A60200736302007363020054
:1060900091A70200F5550400818D02007363020090
:1060A0007363020073630200736302007363020090
:1060B0007363020073630200000000000000000030
:1060C0007363020073630200736302007363020070
:1060D00073630200652B03007363020073630200A5
:1060E00021CD020073630200736302000000000010
:1060F00000000000736302000000000073630200F0
:10610000000000000000000000000000000000008F
:10611000000000000000000000000000000000007F
:10612000000000000000000000000000000000006F
:10613000000000000000000000000000000000005F
:10614000000000000000000000000000000000004F
:10615000000000000000000000000000000000003F
:10616000000000000000000000000000000000002F
:10617000000000000000000000000000000000001F
:10618000000000000000000000000000000000000F
:1061900000000000000000000000000000000000FF
:1061A00000000000000000000000000000000000EF
:1061B00000000000000000000000000000000000DF
:1061C00000000000000000000000000000000000CF
:1061D00000000000000000000000000000000000BF
:1061E00000000000000000000000000000000000AF
:1061F000000000000000000000000000000000009F
:1062000010B5054C237833B9044B13B10448AFF3F0
:1062100000800123237010BD7034002000000000B6
:106220008877070008B5034B1BB103490348AFF358
:10623000008008BD0000000074340020887707004B
:10624000154B002B08BF134B9D46A3F5803A002148
:106250008B460F461348144A121A00F063F80F4B8E
:10626000002B00D098470E4B002B00D09847002001
:10627000002104000D000D48002802D00C48AFF3A7
:10628000008000F02BF82000290025F073FD00F0BD
:1062900011F800BF00000800F0FF0320000000001C
:1062A0000000000070340020BC4403200000000007
:1062B0000000000008B5074B044613B10021AFF3FE
:1062C0000080054B1868836A03B19847204600F0A8
:1062D00031F800BF00000000C019060070B50D4D78
:1062E0000D4C641BA4100026A64209D10B4D0C4C8A
:1062F0003BF05AFB641BA4100026A64205D170BDDA
:1063000055F8043B98470136EEE755F8043B9847AB
:106310000136F2E754340020543400205434002075
:106320005834002002440346934200D1704703F8DA
:10633000011BF9E7FEE700BF0649074A074B9B1A16
:1063400003DD043BC858D050FBDC0CF053FEFFF7D4
:1063500077FF000030780700C02E00207034002046
:10636000FEE7FEE7FEE7FEE7FEE7FEE7FEE7FEE705
:10637000FEE7FEE7F7B5134604460A46E9B11348BF
:106380000668E6B1EBB141684D68B3FBF5F105FB7A
:106390001131B1B942EA040515F0030513D1C16802
:1063A0008C4210D3611E07691944B9420BD800957D
:1063B000F5682146A84703B0F0BD0E20FBE7082092
:1063C000F9E70920F7E71020F5E700BF5C3400206B
:1063D00030B401460C4804688CB143681A68013A2D
:1063E00012EA01030ED1C568A9420BD305690A441C
:1063F000AA4207D824690122A44630BC604708207D
:1064000030BC70471020FBE75C340020024B4FF497
:106410003C6043F001031847A01A06004B8802882D
:106420009A4213D842889A4210D380888A8840F2D0
:10643000F313984294BF031AC31A934206D800F28A
:10644000F310904234BF00200120704700207047B5
:1064500013B550E8023F1FFAA3F4B0F806C0644534
:1064600002BFBFF32F8F002211E0B0F80EC06444CA
:10647000B0F80CC0644528BFA4EB0C04C3EA044484
:1064800040E8024CBCF1000FE3D14FF001028DF85F
:1064900003200193019B9DF803000B6002B010BD27
:1064A00013B550E8013F9CB2B0F80EC06444B0F898
:1064B0000CC0644528BFA4EB0C04B0F808C06445C8
:1064C00002BFBFF32F8F002208E0C4EA030440E8B4
:1064D000014CBCF1000FE4D14FF001028DF8032014
:1064E0000193019B9DF803000B6002B010BD50E8C2
:1064F000022FC2EA224240E80223002BF7D1704764
:1065000050E8012FC2EA024240E80123002BF7D1F4
:1065100070470000034B187A0122B0FA80F05A74D9
:106520004009704728FC0220024B187A003018BF3F
:106530000120704728FC0220002070470846704761
:106540000D4B10B5012143600C4B53E8002F42EA7C
:10655000010043E8000494F0000FF6D14AB908495D
:1065600009781974074B08499A60C3E90012074A71
:10657000DA60002010BD00BF581B060028FC022076
:1065800089FC02200CFC022080FB02208C001C00F5
:1065900070B50568AB6886B004460E4673B1142228
:1065A00000216846FFF7BEFEA36805932379019694
:1065B00033B1012B0ED0AB686846984706B070BD6A
:1065C00001238DF8003023690293E3680393636924
:1065D0000493F0E702238DF80030E3681B03029375
:1065E000F5E7436843B1026891680B444360526821
:1065F000934204BF0023436070474BDF704761DF65
:106600007047000013B50A4B00930A4A0A4B9342A5
:1066100008BF002304460193019B0BB902B010BDD3
:106620002046D3E9002190476846FFF7DAFFF3E7F9
:10663000D01B0600FC770700E477070013B50C4B6E
:1066400000930C4A0C4B934208BF0023044601936D
:10665000019808B902B010BDD0E900312046984732
:1066600018B16846FFF7BDFFF2E71120F2E700BF5F
:10667000AC1B0600147807000C78070011DF704788
:1066800010DF704710B50288012A12D80A494388E2
:10669000142404FB02129C1C51898C4209DAC3F5B4
:1066A0007F43FD330B44538100230380438018460E
:1066B00010BD0420FCE700BFB0FD022030B4084B41
:1066C000084A5968948810684A880325033292B2B0
:1066D0001D7000EB8400920030BCFFF74BBE00BF82
:1066E0003CFC0220EC010320094A0A49538814208B
:1066F00000FB0313D96821B9042158681170FFF712
:1067000067BE05231370044B02229A801868F6E7CF
:106710003CFC0220B0FD0220EC01032010B5042255
:106720000C460649FFF726FE30B9054B142202FB42
:1067300004340123237410BD0E20FCE7C81A0600A0
:10674000B0FD022030B5144A142303FB00200A6870
:10675000436803F5805092B15388033302EB8303FF
:106760004FF6FF74834208D21A68013205D05A8866
:10677000033203EB8202904203D2002008E0083388
:10678000EEE79D88A54204D01D8815B10B6001205D
:1067900030BD1346E6E700BFB0FD022008B5074B49
:1067A000191D5888FFF7CEFF18B1BDE80840FFF764
:1067B00085BFBDE80840FFF797BF00BF3CFC022043
:1067C00073B5436804460D4613B31E4AD1688B4225
:1067D0001ED3126993421BD813F0030018D11A4A32
:1067E00021891289914213D121689A6891420FD16F
:1067F000164A5268934201D80A2004E002F58052FA
:106800009342F9D22880B0FA80F0400902B070BDFE
:1068100000232B801E46019601A92888FFF792FFCE
:1068200030B92B8801339BB22B80002BF3D0EDE7DE
:10683000019B226899689142EED16360024B1B89EB
:106840002381E3E75C3400203CFC0220B0FD022001
:10685000033083B240F2FD32934230B50ED90920A5
:106860000BE0228965892A441A4492B2B2F5806FFE
:1068700008D2088062891344638130BD024C2078BD
:106880000028EED00720F8E7B0FD022008220149D9
:10689000FFF770BD901B0600024B034918680822E1
:1068A000FFF768BDEC010320981B0600094A5378E6
:1068B00091780133DBB2994208BF002311789942E5
:1068C0001FBF03705078182303FB002014BF04304F
:1068D0000020704798FC0220B2DF7047B1DF70479C
:1068E000AFDF704786DF704785DF70477FDF704717
:1068F0007EDF7047084A30B500230C2404FB03F107
:106900008D5A854202D10A44508830BD0133142B80
:10691000F4D14FF6FF70F8E74EFA022046DF7047D9
:106920006EDF7047012804D0043804288CBF002093
:10693000012070478378013B072B07D8DFE803F07D
:10694000070606060607040914230380704701237F
:10695000FBE743689B8809339B08F6E710B50446BC
:1069600004F040FA204600F015F9204604F0DEF964
:106970002046BDE8104004F051BC000030B50A6864
:10698000064B072A01D9002005E01401E55A85428B
:1069900002D10A60181930BD0132F2E7600303200A
:1069A00037B500230D460446019301A9FFF7E6FF22
:1069B00038B18378AB4206D1837B9B0703D18368D0
:1069C0000BB903B030BD019B0133019301A92046EF
:1069D000ECE70000F8B5074D074E07460024337872
:1069E000A34200DCF8BD55F8043B38469847013413
:1069F000F5E700BF6CFB02207DFC0220FFF7EABF39
:106A0000FFF7E8BFADDF7047024B9B6903B1184742
:106A1000704700BF1CFA02207DDF704779DF7047A6
:106A20006DDF704758B1CB0801F00701C25C01234C
:106A300003FA01F10A4214BF1846002070470120F2
:106A40007047000070B50A4E3468054654B170684E
:106A500060B1FF2D08D02946FFF7E4FF30B1F3689D
:106A600003FB0544204670BD0024FBE70446F9E71C
:106A70005003032030B5072185B0FFF791FF04468E
:106A8000002837D04568002D36D1407BFFF7DAFF6C
:106A90000721CDE902558DF80A1028B3237B039016
:106AA00003EB83039B0002A8ADF80830FFF742FF19
:106AB0009DF80A00FFF736FFD0B1104B1B78ABB141
:106AC000BDF808500DF106012846FFF7C1FE48B990
:106AD000BDF80630A380E580094B185C092803D077
:106AE00005B030BD0928F7D90320F9E70220F3E704
:106AF0000846F5E70520F3E70020F1E720FC022037
:106B0000E019060038B54FF6FF73984218BF013000
:106B10000D4614BF84B20024FF2C03D94FF6FF7436
:106B2000204638BD21462846FFF77CFF0028F7D1D4
:106B30000134A4B2F0E74B0901F01F0150F8230023
:106B4000C84000F001007047114A73B504460E4674
:106B500001461046FFF7EFFFB8B1043402EB8402A0
:106B600093680193019B83B100242546294601A81F
:106B7000FFF7E1FF18B10021A8B2B0470134013599
:106B8000142DF3D1204602B070BD0024FAE700BFF7
:106B90008CF8022008B50378082B19D30B2B0BD9DE
:106BA000132B15D10B4B0C491878FFF7CDFF0B4B6E
:106BB0000B491878FFF7C8FF0A4B07491878FFF709
:106BC000C3FF094B06491878BDE80840FFF7BCBF72
:106BD00008BD00BFF631002031BB0200F4310020B7
:106BE000A9BC0200F5310020F33100201328014632
:106BF00002D80248FFF79FBF0020704790F802209C
:106C000038B50A4C054620460A46FFF794FF58B1AE
:106C10002846FFF7EBFF38B1901D294604EB8000B2
:106C2000BDE83840FFF787BF002038BD8CF8022050
:106C300010B50A4B19780446FFF7E2FF58B1084B2C
:106C400000205A88A24201D1C0B210BD01301428E0
:106C500003F10C03F5D1FF20F7E700BF4CFA022047
:106C60004EFA022010B50C46FFF7E2FFFF281FBFC7
:106C70000C234343014AD45210BD00BF4EFA0220F8
:106C800008B50246FFF7B2FF38B111460348FFF7D7
:106C900052FF002814BF0220012008BD98F80220EE
:106CA0004B0900EB830001F01F030121994010B54F
:106CB000C94350E8003F03EA010240E8002494F091
:106CC000000FF6D110BD4B0900EB830001F01F034C
:106CD000012110B5994050E8003F43EA010240E825
:106CE000002494F0000FF6D110BD00007FB50378AA
:106CF0008DF804304368029383688DF80C30C368C4
:106D0000049303698DF81430054A064B01A853F823
:106D1000213052F82110984707B05DF804FB00BFFE
:106D200050FB022058FC02201FB503788DF800307C
:106D300043680193037A8DF80830C3680393054ACA
:106D4000054B684653F8213052F82110984705B09A
:106D50005DF804FB48FB022050FC02201FB5012314
:106D60008DF800308DF808100192D0E900136846C4
:106D7000984705B05DF804FB0023435082B04358A8
:106D80000193019B02B070472DE9F0470D789DF803
:106D900020609DF824A004460F469946002D60D13E
:106DA000D0F8243192F800809BB14FF49271FFF734
:106DB000E3FF012363613B70B04550D1D4F8043147
:106DC000002B4CD04FF482712046FFF7D5FF0025F1
:106DD0001DE0D0F81C31FBB14FF48E71FFF7CCFFF2
:106DE000D0F824311BB14FF492712046DFE71378BD
:106DF0009E4207D919F80330C0F81C3513780133C7
:106E00001370D9E70123BAF1000F03D0C3612846FC
:106E1000BDE8F0874361CFE7D0F80831002BCBD035
:106E20004FF48471FFF7A8FFD0F82431002BDAD19A
:106E300013789E42C0D9D0F8181509F803101378BA
:106E40000133DBB21370721E934205D10223C0F8E6
:106E5000003201232362AFE79E42FAD1ACE701255D
:106E6000D5E74FF49271FFF787FF4FF48E71FFF76C
:106E700083FF4FF48471FFF77FFF9FE72DE9FF4702
:106E80000C4605461F46204642F210734FF48271AD
:106E900092460393FFF770FF4FF49271FFF76CFF78
:106EA0004FF48E71FFF768FF4FF48471FFF764FFB2
:106EB0000023012F85F82E3085F82B3008BF0222E1
:106EC0004FF001030CBFC4F80022C4F80032236263
:106ED00023602E68AEB905F12E0905F12B08039B3E
:106EE000002B18DC95F82B301BBB0020039B002BDC
:106EF0000EDC0023C4F800350523C4F80035032058
:106F000006E040F28623AB60AB68C4F8043300208F
:106F100004B0BDE8F087CDE9007653464A464146C5
:106F20002046FFF731FF0028DCD0039B013B039391
:106F3000D5E7D4F8C434C4F8C434002BD5D013F04A
:106F4000010F14BF4FF40240032048F2012213F056
:106F5000020F18BF104613F0040F48F2022318BFA7
:106F60001846C3E72DE9FF470C4605461F46204655
:106F700042F210734FF48271164603939DF83080ED
:106F8000FFF7FAFE4FF49271FFF7F6FE4FF48E71A1
:106F9000FFF7F2FE4FF48471FFF7EEFE0023C4F812
:106FA000003285F82E3085F82B3001232362A36050
:106FB00095F82E2097421FD9B35CC4F81C3595F87C
:106FC0002E30013385F82E302B68E3B905F12E0AF7
:106FD00005F12B09039B002B1FDC95F82B3053BBCD
:106FE0000020039B002B15DC0023C4F8003505238B
:106FF000C4F8003503200DE0B8F1000F01D0E361C3
:10700000E2E76361E0E740F28623AB60AB68C4F877
:107010000433002004B0BDE8F087CDE900783346A2
:10702000524649462046FFF7AFFE0028D5D0039BC5
:10703000013B0393CEE7D4F8C434C4F8C434002B26
:10704000CED013F0010F14BF4FF40240032048F2DA
:10705000012213F0020F18BF104613F0040F48F27C
:10706000022318BF1846BCE72DE9F04793F90050FA
:1070700090B00024013D6E46AD002746A446A046D0
:107080005FF0000E03E05FEA080EBEEB050EB8EB02
:107090000E0952F809A051F80E90A9FB0A9A14EBB8
:1070A000090457EB0A075CF1000C1EF1040EAE4513
:1070B00001DCC645EBDD46F808403C4667465FF01C
:1070C000000C18F10408A845DADDB8EB450FDADD4D
:1070D00046F80840D3F8B0303146984710B0BDE8C4
:1070E000F08713460A46FFF7BFBFF0B5154689B0D3
:1070F0001C4607460E461A4629466846FFF7F1FF2A
:1071000023466A4639463846FFF7AEFF23462A46ED
:1071100069466846FFF7A8FF23466A46314630466F
:10712000FFF7A2FF09B0F0BD07B5142200211148F6
:10713000FFF7F8F8104B53E8021FD888B1EB314F36
:107140004FF0000217BF89B240EA004041EA004018
:1071500004E05968B1EB314F08BF012243E8020156
:107160000029E8D18DF807209DF80730002003B0F2
:107170005DF804FB28FC02200CFC0220024B0022DC
:10718000C3E90022704700BF78FB02202DE9F041DF
:1071900004782C4F9EB00246002C4ED181884FF2CD
:1071A0003143994249D181793B7B994245D103468C
:1071B0004CF2E96C4DF6F30E41F20D28117A8C4237
:1071C0000BD300238DF804305388ADF806303B68AC
:1071D00001A898471EB0BDE8F081D98961451DD04E
:1071E000714510D0414516D1194651F80E0FCDF812
:1071F000560048680989ADF85E10198BCDF85A0021
:10720000ADF8601007E01E4613AD56F80E0F71681A
:1072100003C53189298001341233CFE7194651F86B
:107220000E0FCDF8660048680989ADF86E10198B0D
:10723000CDF86A00ADF87010EDE701238DF8043049
:10724000C5E700BF28F4022008B510461A463AF0F8
:1072500069FB002008BD38B504884CB9821C00F1D8
:107260000A0512F8013B1BB99542FAD100200AE049
:107270000B88A342FAD10822023102303AF044FBD3
:10728000B0FA80F0400938BD08B570B171B103782B
:107290000A78534013F0FE0F08D106220131013065
:1072A0003AF032FBB0FA80F0400908BD0020FCE75C
:1072B0002DE9F04391B00F461C220021804609A819
:1072C000FFF730F801251C22002101A80895FFF7DF
:1072D00029F8394608AA11F9046B0095334610467F
:1072E0000BF04EFA314608A80BF0DFF9013804B272
:1072F000012C07DC3246694640460BF0CAF911B052
:10730000BDE8F0833A4668466946FFF7EAFE10ABEF
:10731000601103EB80001FFA84F909F01F0350F895
:10732000202C05FA03F3134205D03B46424669463A
:107330006846FFF799FE09F1FF3424B2D8E72DE93A
:10734000F0438BB01446129D15F9046B00961F464E
:10735000804689462B460246214602A80BF03EFA9B
:1073600002A9129A0846FFF7BCFE129B02AA4146E8
:107370004046FFF779FE129B02AA21462046FFF7FE
:1073800073FE2B464A463946384600960BF026FADD
:10739000129A394602A8FFF7A4FE02A92B464246DC
:1073A000084600960BF01AFA02A92B462246084618
:1073B00000960BF013FA2B464246214620460096D3
:1073C0000BF00CFA129B224649464846FFF74CFE4A
:1073D0002B4602AA4146204600960BF0FFF9129B6D
:1073E000224639463846FFF73FFE2B464A46394685
:1073F000384600960BF0F2F9324602A920460BF00F
:1074000048F90BB0BDE8F08370B5036813F00105CF
:107410000646144605D013460A4601460BF0B0F95D
:107420000546214630460BF012F945B104F1804281
:10743000013A56F8223043F0004346F8223070BD3E
:10744000F0B50C4689B0082206460BF022F9E36A33
:107450000393236B0493636B0593A36B0693E36B16
:107460000793002708236A4669466846CDE90177F5
:1074700000970BF085F9082305466A4631463046E9
:107480000BF07EF9236B0393636B0493A36B05935B
:10749000E36B0544CDE906376A460823694668462A
:1074A0000BF06EF9082305446A46314630460BF06E
:1074B00067F9236A0093636A0193A36A0293A36B3B
:1074C0000693E36B0793054408236A46314630462A
:1074D000CDE9047703970BF053F9636A0093A36A2D
:1074E000A26B0193E36A02930492636BE26B0393D2
:1074F000CDE90523236A0793054408236A463146EC
:1075000030460BF03DF9E36A0093236B0193636B04
:107510000293236A0693A36A0793054408236A46E5
:1075200031463046CDE9047703970BF0F9F8236B29
:107530000093636B0193A36B0293E36B0393636A02
:107540000693E36A07932D1A08236A4631463046AC
:10755000CDE904770BF0E4F8636B0093A36B019320
:10756000E36B0293236A0393636A0493A36ACDE9EE
:107570000537236B07932D1A08236A463146304698
:107580000BF0CEF8A36B0093E36BCDE90137636A90
:107590000393A36A0493E36ACDE90537636B07930A
:1075A0002D1A08236A46314630460BF0B9F82D1AD9
:1075B0000D4C0FD435B90822314620460BF054F853
:1075C00001280FD008232246314630460BF0A8F898
:1075D0002D1AEFE708232246314630460BF0D0F84B
:1075E0002D18F7D409B0F0BDF01906002DE9F043CD
:1075F0009BB01646229C14F9045B009598460746FA
:10760000894623460246314612A80BF0E7F812A934
:10761000229A0846FFF765FD229B12AA3946384692
:10762000FFF722FD229B12AA31463046FFF71CFDD0
:1076300023464A46414612A800950BF0E1F823463E
:107640004A464146404600950BF0C8F823463A4664
:1076500031460AA800950BF0C1F8229B0AAA4946B8
:107660004846FFF701FD2346324639460AA80095F1
:107670000BF0C6F8229A41463046FFF732FD23460A
:107680000AAA3146304600950BF0A8F82346324648
:10769000394602A800950BF0A1F8229B02AA4146A8
:1076A0004046FFF7E1FC23464A46414640460095E6
:1076B0000BF094F8229A12A902A8FFF712FD02A972
:1076C00023460AAA084600950BF088F823463A4656
:1076D00002A90AA800950BF081F80AA9229B12AA18
:1076E0000846FFF7C1FC23464A460AA948460095CA
:1076F0000BF074F82A4602A938460AF0CAFF1BB0FC
:10770000BDE8F0832DE9F04115468AB0044688466D
:107710001C22002103A8FEF705FE2E1D95F900701E
:1077200003232A46414620460293FFF7DAFC3346FC
:1077300002AA2146204600970BF050F82B464246FD
:1077400021462046FFF790FC0097334605F184025E
:10775000214620460BF054F80AB0BDE8F0812DE92F
:10776000F04793F9006092B00446894610463146CE
:10777000154698460AF0B9FF002840F0938042462B
:1077800049460AA8FFF7ADFC43460AAA214602A8CB
:10779000FFF76AFC0AA908464246FFF7A2FC4346E7
:1077A0002A4649464846FFF75FFC08F1040742466F
:1077B00029462846FFF795FC3B462A4621462046A7
:1077C00000960BF01DF83B462A46294628460096AF
:1077D0000BF016F83B462A462146284600960AF04A
:1077E000FDFF43462A4621462046FFF73DFC3B4627
:1077F00022462146284600960BF002F83B460096AA
:107800002A46214620460AF0FBFF2368DB074CD5B9
:1078100033463A46214620460AF0B2FF31468246B8
:1078200020460AF014FF06F18043013B54F8230080
:1078300040EACA7044F82300424621462846FFF732
:1078400050FC3B4602AA2946284600960AF0C6FF8D
:107850003B4602AA2946284600960AF0BFFF02A925
:1078600008463B462A4600960AF0B8FF434602AA5D
:1078700021462046FFF7F8FB0AAA3B461046214660
:1078800000960AF0ABFF3246294620460AF001FF77
:107890003246494628460AF0FCFE32460AA94846C6
:1078A0000AF0F7FE12B0BDE8F087314620460AF034
:1078B000CEFEC1E703681A78302A27D15A1C02602D
:1078C0005A7802F0DF024F2A03D102330360082006
:1078D0007047582A03D10233036010207047422AB0
:1078E00004D0082013F8012F22B970470233036037
:1078F000022070472E2A07D0A2F13801012903D9AE
:10790000303A092AEED970470A20EBE70A2070477F
:1079100070B58AB014460E460022014601A82DF02B
:107920004BFC2546DDE901239A4204D3049832F04A
:1079300029FF601B04E02DB9049832F023FF204694
:107940000AB070BD01A82DF0E6FB013D06F8010B61
:10795000E8E7000030B50B4B1B68012293F850108C
:107960000D338A4204DB405CB0FA80F0400930BD40
:1079700013F8014B855CA54201D10132F1E70020EB
:10798000F5E700BF24F4022070B592B00C46014622
:1079900068461E462DF010FC0022214609A82DF055
:1079A0000BFC68462DF061F8044609A82DF05DF83F
:1079B000844205460DD0039832F0E4FE0C9832F074
:1079C000E1FE002C01DB002D00DA56B9601B12B07D
:1079D00070BD002C07DA039832F0D4FE0C9832F018
:1079E000D1FE0020F3E768462DF0EEF809A82DF04F
:1079F000EBF8D6E7044A138A9BB223F0410343F025
:107A000040031382704700BF9834002010B58AB03D
:107A10000A46014601A82DF0CFFB0023DDE9011243
:107A2000914203F1010401D201330AD1049832F0EA
:107A3000A9FE202029F004FA14F1FF340AD20AB07A
:107A400010BD01A82DF067FB0A28EFD029F0F8F946
:107A50002346E3E70820EDE770B58EB032F063F916
:107A60000546002876D03D4C94ED000B32F09EF890
:107A70003B490246284634F034F894ED020B32F0CC
:107A800095F838490246284634F02BF894ED040B5B
:107A900032F08CF834490246284634F022F894ED4E
:107AA000060B32F083F831490246284634F019F8C3
:107AB00094ED080B32F07AF82D490246284634F04E
:107AC00010F894F8382032B394F839300492013B1E
:107AD000059394F83A3003A803F5FA63069317F078
:107AE000ADFAA36A0C93E36A0B93236B089000260C
:107AF0000A9308A8636B09930D9617F09DFBCDE9D7
:107B000000011C4930462BF077FB9DED000B06462B
:107B100012F048F932461849284633F0E2FF94F84B
:107B20003C0032F055F815490246284633F0D9FF9B
:107B300094F83B0032F04CF811490246284633F0E5
:107B4000D0FF94ED100B32F031F80E490246284672
:107B500033F0C7FF28460EB070BD00BFB034002020
:107B600089C40600641B0600681B06006C1B060027
:107B7000721B0600791B0600263C06007E1B0600D1
:107B80005C2B0600891B060030B58BB04FF0C0435C
:107B90000193054608B1002303602022002102A8BA
:107BA000FEF7C0FB002202A94FF0C04034F046FFB0
:107BB000D0B10024029B039A23F07F43033323F0C8
:107BC0000303203352B11C44032202A901A834F05C
:107BD000BDFF0028EED120460BB030BD002DF3D004
:107BE0002A6813442B60EFE70446F4E72DE9F04FD1
:107BF000002493B04FF0C046202280460D460AA8CC
:107C00002146CDE906640894FEF78CFB01220AA9FF
:107C10003046099634F012FFA8B907AB019308ABC0
:107C200042464FF0C141009306A82B4635F0DEF9DD
:107C30000698013834F07AFF069035F01BFA0120DF
:107C400013B0BDE8F08FDFF83C910B9B002B69D09F
:107C5000069A089BDDF824B0D3185B4503931CD02B
:107C60000A9B23F07F43203304934FF0010A0AF16B
:107C7000FF373B01DE1B4E443046059332F0E0FAFD
:107C800070B13B01DF1B59F807108B4519D90AF178
:107C9000010A42F6E0629245E9D921230AAA25E0C9
:107CA000304632F085FA0028EBD1304632F0D2FA75
:107CB0000028ECD032680F230E32B2FBF3F292446C
:107CC000E5E7049B0BEB03029142E0D2039BA3EB9D
:107CD0000B020A4449F80720D9E712F8011B08F8FB
:107CE00004100134B4FBF5F105FB1144013BF4D160
:107CF000089B203308930A9B23F07F4A099B0AF1D3
:107D0000030A07AE2AF0030A03F1200B019608AF1D
:107D100000972B464246594606A835F067F9BAF156
:107D2000000F07D101220AA909A834F00FFF00288B
:107D30008BD172E7089B079AE81A2B1B834228BF56
:107D40000346A24203D9121B934228BF1346BBB17C
:107D5000534528BF53461A46594608EB040003937F
:107D600022F0D0FF039B089A01961A441C44AAEB08
:107D7000030A9B440892B4FBF5F305FB1344C7E7E1
:107D800018465DE70435002030B58BB04FF0C04495
:107D90002022002102A80194FEF7C4FA002202A9C1
:107DA000204634F065FE70B1032202A901A8DDE986
:107DB000015434F0CBFE0028F6D124F07F44233563
:107DC0002C4424F00304C4F1C1400BB030BD0000CA
:107DD00070B400230D4D1A4642F6E064C3EB031164
:107DE0002944981C01334E7B4A73A3428E7B8880C2
:107DF0008A73F3D1064B83F8152383F81623054BBA
:107E000001221A8070BC32F06BBA00BF043500202A
:107E100004F1022002350020F8B50646B0F80B0048
:107E20000C46C8B132F04EF8074633F019FC451C39
:107E3000384632F0A7FC284631F0CAFE214633F01E
:107E40006BF9044638B10146304633F0D1FC204688
:107E500032F098FC681CF8BD0125ECE738B5074CFA
:107E600025780023EDB202461946237031F022F93D
:107E700025700348BDE8384028F062BC003500207A
:107E8000E2C10600F8B504460E46174639F084FDF7
:107E90000146204631F030FF054660B10C4B1C888E
:107EA000A4B224B10022114629F052FD044628460E
:107EB00032F068FC25463B4632460021284629F030
:107EC00011FD0446284632F05DFC2046F8BD00BF97
:107ED0000235002038B50022054633F02FFE044657
:107EE00050B100231A460146284629F079FD204664
:107EF000BDE8384032F046BC38BD000070B5EFF345
:107F0000108672B60D4A94680123A4B993600C4B95
:107F10000C4DD3F8801029401160C3F88050D3F87D
:107F2000841051604FF0FF32C3F88420047006B90A
:107F300062B6002070BD0370F9E700BFE8030320BC
:107F400000E100E0FC06FFBD38B50B4C0B4D2B7873
:107F50005BB12CF0CDF840B914F1FF34F7D20849E9
:107F60000420BDE838402DF05DBD002CF7D02CF08A
:107F7000BFF80028F3D138BD80841E000804032018
:107F8000EC1A060020292DE9F0470BD9244A254E8A
:107F90002139C9B200231446DFB2B94205D814F81A
:107FA00001C0B6BB4008BDE8F08712F8017B013381
:107FB0003E44F1E7745CC82C1ED81EF80450DFF86C
:107FC0006C90194B4FF000085FFA88FA54450DD8B1
:107FD00003EB0509994511D101316145EADB023214
:107FE000504320F0704007300009DCE719F801AB7E
:107FF00008F101085344E7E70023E9E713F8018B90
:10800000B8FBF7F407FB1484E4B2A242B8BF2246DF
:10801000E0E700210A46DFF814E00D27DDE700BFA6
:10802000E41B0600C31C0600E71E06001E1E060019
:1080300073B5054610460E4633F08FF9002304460B
:108040000093014633460822286809F0D1FB2146F7
:1080500002B0BDE8704033F06BBA10B504460121A0
:10806000007922F08BFE2079032123F087FA6079D2
:10807000012122F083FE60790321BDE8104023F046
:108080007DBA0000F7B5002201912749064633F07A
:10809000C1FC0546C8B1014601AB0122304629F0BA
:1080A0009FFC58B921482DF08BFB214A1E491378BB
:1080B000304643F00403137034F043F8284632F09E
:1080C00061FB0124204603B0F0BD02461949304649
:1080D00033F034FD074632F076F9044628B9019AA8
:1080E0001449304633F0E6FCEBE7384632F0BAFE8E
:1080F0000646019832F0B6FE3044B0F5007F05D94F
:108100000B4A137843F0020313702C46B6F5007F38
:1081100006D2C6F5007300220199384632F09AFD66
:10812000384632F02FFBCDE7151B06001D1B06005D
:1081300001350020511B0600437882781B01120292
:1081400002F4E06203F030031343027802F003020A
:108150001343C278120302F48052134302791204CB
:1081600002F4E02213434279120502F48012134311
:108170008279120602F080721343054AC2F818355C
:10818000C379017AC2F81415C2F81035704700BFE0
:108190000070004010B588B012788DF80C200021D6
:1081A000FF2202918DF80D2001214FF6FF72104C35
:1081B00001908DF81C10ADF80E208DF8103027F0CE
:1081C00043FA70B12BF094FF58B914F1FF34F6D292
:1081D000084904202DF026FC01A827F045FA08B034
:1081E00010BD002CF4D02BF083FF0028F0D1F3E772
:1081F00080841E00FC1A060010B5002388B0CDE96B
:10820000030301920E4C029302228DF81C2027F0EA
:108210001BFA70B12BF06CFF58B914F1FF34F6D291
:10822000084904202DF0FEFB01A827F01DFA08B034
:1082300010BD002CF4D02BF05BFF0028F0D1F3E749
:1082400080841E00FC1A060037B50B015BB249B2F0
:10825000044643EA01008DF804001A4D50B203436E
:10826000120152B28DF805302B78114302438DF87C
:1082700006108DF8072013B302AB03EB941302AA88
:1082800013F8040CC4F30113134413F8043C43EA39
:1082900000201FF02DF82B788BB102AAC4F38103C4
:1082A00004F003041344144413F8040C14F8043CBD
:1082B00043EA002003B0BDE830401FF019B803B016
:1082C00030BD00BF00040320002A70B403460D46F1
:1082D00003D1442270BC39F025BBA0F102011EDAA3
:1082E000A2EB820202F01F04521105EB8202C4F5D8
:1082F00004756D110233023203EB8505C4F12006CB
:10830000106852F8043F00BA1BBAF340A040034380
:108310001BBA41F8043F8D42F2D170BC704702EBAA
:10832000420202F01F046FF00300521100FB0252E0
:10833000023A03F14200C4F1200652F8045F52F8F9
:10834000043C2DBA1BBAB340E5402B431BBA41F89D
:10835000043F8842F1D1E0E7024B4FF4807043F0D4
:1083600001031847C01A060010B586B00446002263
:10837000684616F0CDFD2046009916F089FE20468D
:1083800006B010BD38B501230B7004460D4631F020
:10839000D0FE88B100220B49204633F0CFFB10B14C
:1083A00033F049FF287020460022074933F0C6FB0E
:1083B000BDE8384033F04ABE2046BDE8384033F0CF
:1083C0004FB900BFCC1A0600D11A0600F0B5184DFF
:1083D000184B2C68242161435A1800265E505660C1
:1083E00006885E5286789670468B5683C68BD683F7
:1083F000067E16760431467E56760B441362818BD8
:1084000091838278022A2E460CD1051D00F11402B8
:10841000286869681F4603C7083595423B46F7D16F
:1084200028683860013404F007043460F0BD00BFF0
:10843000280303200402032030B50B4B19680B4BB3
:108440000022914201D1002009E09D788478A54264
:1084500006D11D880488A54202D1054B186830BD9D
:1084600001320433EDE700BF8CFC0220C001032081
:1084700068FB02202DE9F74F8B4690F8C612019257
:108480007623804601FB03000091FFF7D5FF81466C
:1084900070B3194E3568052D2AD8184C0099019AE9
:1084A0004FEAC51A04EB0A07762303FB01817A80A1
:1084B000381D1A4639F036FABBF1000F14BF0023FD
:1084C000022304F80A300E4BC7F87C901A68013575
:1084D000954235601D460BD10027E36F2046984733
:1084E0002B6801379F4204F18004F6D300233360E8
:1084F00003B0BDE8F08F00BF1001032010FE022082
:108500008CFC022070B590F8C63216467622A0B0D8
:1085100002FB03000D46FFF78FFF044660B17C228B
:10852000002101A8FDF7FEFE01238DF80430ADF80F
:108530000660029501A8A04720B070BD9EDF70477D
:108540002DE9F34790F8C64290F8C552762314FB04
:1085500003F4071905EBC50397F804C004EB4303C4
:108560006E1C0A336645034413D000F11C0A07F160
:10857000220E0CF1FF384FF01209A244ECB2A445D0
:108580000BD9A8451C891AD13B899C4226D10023CE
:108590001DE01B893889834205D101230B7000201F
:1085A00002B0BDE8F0870133ADF80430ADF8060045
:1085B00000230B70104601A9FFF7C0FFF0E709FB8D
:1085C00005F301343EF80360B4420DD1534490F8F2
:1085D000C542013480F8C5420135CFE70134ADF81A
:1085E0000440ADF80630E3E7013EADF80440ADF8D5
:1085F0000660DDE79DDF704737B590F8C53290F82B
:10860000C6220C46C3B1013B7621DBB25143122591
:1086100005FB031303445B8A01339BB2ADF80430BE
:10862000762303FB020201A91389ADF80630204628
:10863000FFF7E0FF03B030BD762303FB0203DB88C6
:10864000ECE79BDF7047000038B54FF433720D46FE
:1086500000210446FDF766FE114AA4F8CA52002321
:108660001360104A84F8C9321268226084F8C63256
:1086700084F8C532224601212846FFF7E2FF11287F
:1086800006D020B9012384F8C73284F8C80238BD67
:10869000012284F8C72284F8C8221846F7E700BFF1
:1086A00010010320C001032070B50C4690F8C922C8
:1086B000174901320968D2B28A42034680F8C922BA
:1086C0004FF0000521D290F8C61280F8C552013152
:1086D000C9B280F8C612762011FB00F00D4E1A18B0
:1086E00056F821101950012115712046FFF7A9FFF6
:1086F000014648B183F8C75222461846FFF702FFE9
:10870000054B03221A705C8070BD80F8C752F7E7F2
:108710008CFC0220C001032010FE02202DE9F34151
:108720000C460546C8B1C1B18E4B1B78ABB103886E
:10873000302B4AD014D8112B00F0048194F8C832A1
:108740005BB12B88303B1F2B07D8B4F8CA32A988FD
:10875000994202D12046FFF777FF02B0BDE8F081D1
:10876000322B57D0332BE9D18288B1F8CA329A42E2
:10877000E4D1C08891F8C6C291F8C56258B9762391
:1087800003FB0CF7122303FB0673294623446A8973
:108790009042C0F0AD80762202FB0C42731C12792D
:1087A000002793428DF8077000F0C68084F8C53228
:1087B0000DF10701AA882046FFF7C2FE01460028F6
:1087C00000F0908084F8C77261E08388B1F8CA2213
:1087D0009A42B3D1C688A6B991F8C632762213FB65
:1087E00002F3CA18C168E1500369C2F806308188F3
:1087F0002046FFF701FF014600289FD084F8C7629A
:1088000045E000212046FFF735FEA9882046FFF706
:108810004BFF93E78288B1F8CA329A428ED1C3885F
:10882000002B53D191F8C612AA7A762311FB03F1DB
:10883000601805F10C0E03791A44062AD4BFD2B28F
:108840000622027103EBC30201EB4202224400261E
:108850000779BB420EF10A0E02F1120221D3122255
:10886000013B02FB03430B445A8A03899A422DD2EF
:10887000062F2BD084F8C572A9882046FFF7BCFECE
:10888000014600283FF45AAF002384F8C732AA8873
:108890002046FFF737FE344B03221A70AA885A800D
:1088A0004CE7F446A2F108075CF80A8D42F8088C00
:1088B000DCF8048042F8048CBCF808C0A7F808C0B3
:1088C000013356809680D6801681C1E7002684F851
:1088D000C5620DF10701AA882046FFF731FE014667
:1088E00000288BD19DF80730002B3FF427AF26E0FE
:1088F000CA89A2F52452082A08D8DFE802F0141722
:108900000507070707071A008A899A829A8A3AB1E7
:10891000DA8A2AB11A8B1AB15A8B002A7FF43BAF3C
:108920000130063133E78A89DA82EFE78A891A83D0
:10893000ECE78A895A83E9E701238DF80730AA8892
:1089400001215FE78288B1F8CA329A427FF4F6AE1D
:10895000002381F8C73281F8C8324FF6FF73A1F8BF
:10896000CA32EBE674FC022010FE022062DF704780
:10897000A3DF7047A1DF704770B50E4A0E4C126836
:108980002368934210D00D4924225A438D18885AE7
:10899000AE78012E09D10022A988FFF7EBFF18B9A4
:1089A000013303F00703236070BD18321144FFF751
:1089B000DFFFF4E72803032024030320040203203D
:1089C00030B58BB004460D461C2200210DF1060087
:1089D000FDF7A8FC02AA022301A809920122ADF822
:1089E00022308DF81C208DF808208DF80630ADF867
:1089F0001E50ADF80440FFF7E9FCFFF7BDFF002073
:108A00000BB030BD2DE9F0470388382B9EB00546EA
:108A10000C460BD0392B20D0112B1BD10B8982880F
:108A20009A4204BF4FF6FF730B8113E00A898388D3
:108A30009A420FD103895BB14A8B9A4208D1C2880E
:108A40000B68ADF8102006218DF8041001A8984796
:108A5000FFF792FF1EB0BDE8F08782880B899A422B
:108A6000F8D143898A8C9A4234D1C389082B05D026
:108A700003220B688DF8042001A898476A7C9DF8B2
:108A80000D30297C8DF80C10500862F3000360F360
:108A90004103900860F38203D00860F3C303120916
:108AA00062F30413EA7C8DF80D308DF80F20AB7C57
:108AB0006A698DF80E300229029209D80C2B34BF56
:108AC000022303238DF8043001A823689847C1E7E7
:108AD0000323F7E78A8E9A42BCD1B0F80E8000F1EA
:108AE000100600254FF0080901F1EC07A845B1D99F
:108AF00094F8DC30082B00F2EF80DFE813F0090077
:108B000027002F004100610069009500DC00F000A3
:108B1000735D84F8DD306A1C33B1012B0DD008235E
:108B200084F8DC301546E1E7042384F8EC3004F1E6
:108B30003C03C4E934390123F2E7052184F8EC1041
:108B400004F1BC01C4E934130223E9E77359C4F802
:108B500008310435032384F8DC30C7E7D4F8E83063
:108B6000725DE018691C80F80C213AB10133C4F839
:108B7000E830022384F8DC300D46B7E70323F9E739
:108B8000735DD4F8D420C4F80031934205F101009C
:108B900004D3082384F8DC300546A7E7D4F8D010C6
:108BA0001B01CA18D268C4F80421D4F8D820002ABE
:108BB000EFD0CB5C13B1013AC4F8D8200423E9E725
:108BC000735DA4F8FC30052384F8DC3001358DE7B3
:108BD000735DB4F8FC20D4F8D01042EA03220023DD
:108BE000A4F8E430D4F80031A4F8FC201B0105F10E
:108BF000010AC81852B10389A3B1C368002B0CBF86
:108C00000723062384F8DC3055466FE7CB5C13B1AD
:108C1000236838469847D4F8D830002B14BF032374
:108C20000823EFE70723EDE7D4F80021D4F8D0308C
:108C3000B4F8E41003EB02131B898B420BD9B4F890
:108C4000FC308B4207D94A1CA4F8E420D4F8043144
:108C5000725D5A540135B4F8E420D4F80031B4F808
:108C6000FCC0D4F8D0001B01944500EB030103D0F5
:108C7000098901398A421CD1C35C1BB1D4F8043183
:108C800000219954B4F8E420B4F8FC309A4221D37E
:108C9000D4F80031D4F8D0201B01D35C13B1236881
:108CA00038469847D4F8D830002B14BF0323082344
:108CB00051E706234FE7B4F8E430B4F8FC209342C0
:108CC0003CBF0133A4F8E430B4F8E43038BF0135D8
:108CD0009342DDD007233EE784F8DC9006E7454663
:108CE00004E7000038B520252A4640240021174813
:108CF000FDF718FB224600211548FDF713FB22461D
:108D000000211448FDF70EFB10244FF400720021DF
:108D10001148FDF707FB224600211048FDF702FB32
:108D2000142200210E48FDF7FDFA224600210D48CD
:108D3000FDF7F8FA224600210B48FDF7F3FA2A4620
:108D400000210A48BDE83840FDF7ECBA88F502205A
:108D50004CF802200CF80220DCF50220DCF702209F
:108D6000A8F50220FCF70220ECF70220BCF5022057
:108D700028DF704729DF704769DF704760DF704781
:108D800007B50A4B00930A4A0A4B934208BF0023D7
:108D90000193019B13B903B05DF804FBD3E90020F4
:108DA00090476846FDF71DFCF3E700BFC41B0600B3
:108DB0000C780700FC7707001FB50021039001AA7B
:108DC00044F20100CDE9011119F07EFB08B5FFF76F
:108DD000F3FF0000F0B50378022B8BB004463FD0C0
:108DE000042B00F0B280002B40F0A2805A4B428846
:108DF0001A81B0F850205A83B0F86C20DA86B0F8A7
:108E00006A209A86554EB0F85C20DA84B0F85A2071
:108E10009A8464251C4646F001064FF47A40B04718
:108E2000013DFAD1E18C2089FFF7CAFD40B19023C2
:108E30000193042381B20DEB030201201EF092F98D
:108E4000E18E2089FFF7BCFD002871D093230193A8
:108E500004230DEB030281B201201EF083F967E0C9
:108E6000021D92E803003E4D85E80300237A012BA2
:108E700067D8FFF737FF2B79022B5BD8AB790B2B29
:108E800058D82022002101A82C68FDF74BFA324B5C
:108E90008DF80940598BADF81E1002A909910121E6
:108EA0008DF81C10210A00228DF80A10210C240EC6
:108EB0008DF80B108DF80C40C3F8CC201646052118
:108EC00010461C4693F83C50B5B10AAD6F18451ECC
:108ED000022D01F1010207F8200C0AD80DF1280C2F
:108EE000B3F84450624402F8205C2D0A07F81E5C77
:108EF000CA1C1146013601220130082803F1100373
:108F0000E0D10AB1C4F8CC602389ADF80430022363
:108F10008DF8063001A8D4F8CC30C4F8D830ADF8BC
:108F20002210FFF753FAFFF727FD002384F8DC3007
:108F30000BB0F0BDD423019304230DEB03020721F2
:108F40008AE7082300211E2087E74369072BEFD11A
:108F50000823034AF6E700BF28F40220B01A0600EF
:108F600080FC02207FB50F4D0F4C104E01A8FDF77D
:108F700044FB034678B9B44218BF234602950393D5
:108F8000039B002BF2D00198D3E90021904702A85F
:108F9000FDF727FBF4E7052801D0FFF70DFF04B02C
:108FA00070BD00BFB81B0600CC770700E477070050
:108FB00030B5124DC7B04FF486740DF1020103A80D
:108FC000ADF80240FDF71BFB034688B90C480D4A7B
:108FD0000195904208BF18460290029B002BECD0EE
:108FE00003A8D3E90021904701A8FDF7FAFAF4E7B6
:108FF000052801D0FFF7E0FE47B030BDA01B0600FA
:109000008C770700CC770700024B1B780BB1FFF77A
:10901000CFBF7047E901032010B5084B9A685AB1D9
:1090200050B9EFF3108172B6054A1C6814605C6891
:109030005460986001B962B6002010BDE8030320B7
:1090400000E100E0F7B51B4F3B7873B31A4E0120E7
:109050003070FDF7F3FA11284FF0000527D00220F9
:10906000FDF7D0FA0DF107008DF80750FEF746FF27
:10907000FDF704FB04469DF807003D70FFF7CCFFA9
:1090800054B90E4B34709A684AB11A6822F48002BF
:109090001A600320FDF7B6FA204603B0F0BD084B76
:1090A0004FF48002C3F88020F3E70824F4E72C464D
:1090B000F2E700BF89FC022088FC0220E8030320BD
:1090C00000E100E073B5234E3478002C3FD1224DEF
:1090D000012320462B70FDF7B1FA112834D0204629
:1090E000FDF790FA1D4B8DF80340186801900DF1C3
:1090F0000300FEF703FF1A4901A8FDF7C1FA044671
:10910000B0FA80F0400930709DF80300FFF784FF4B
:10911000D4B9144A2C7092F816335B09012B08D984
:10912000042B06D0104B996839B94FF480031360B3
:1091300007E042F20200FFF73FFE1A6842F48002A5
:109140001A600120FDF75EFA204602B070BD0824C7
:10915000FAE700BF89FC022088FC0220C41906003F
:10916000C924040000E100E0E803032038B5831EB1
:10917000012B54D82A4C237A002B50D0022B09D132
:10918000032835D0274B00221B68E2601A7942B1D0
:10919000012A27D0637C002B33D1BDE8384000F092
:1091A0004BB8D3E905128D1AB5F5805F94BF5219FB
:1091B00002F580529A619142ECD102284FF00003EF
:1091C00008BF19462372174B18BF0D211868FDF709
:1091D000DFF9154B1A885B889A42DBD11348FDF7FB
:1091E00086F9D7E71A6901321A615B699A42E3E7A7
:1091F000E3680133082B01D8E360CBE70023E36089
:10920000DBE70B4B1B7853B10A4B1B781BB1BDE856
:109210003840FFF717BFBDE83840FFF753BF38BDF0
:1092200028FC0220A4FD02206CFC02200CFC022081
:1092300088FC022089FC0220F8B52A4C2A4D237AAA
:1092400083B92A4F2A4E39463046FDF701F918B93D
:10925000286000236360F8BD7A88336813442B606C
:10926000002BF6D0022323722B681A7992B1012ABF
:1092700028D018460321FDF78BF900232372636081
:109280001A4B1A885B889A42E5D11948BDE8F84024
:10929000FDF72DB9D3E90520121AB2F5805F28BF7A
:1092A0004FF48052D3E903159208012A014438BFD4
:1092B00001222844FFF75EFD50B11128D9D10123C6
:1092C0002372C8E7D3E903021044FFF751FDF3E727
:1092D000237C002BBFD10146BDE8F8400220FFF7F8
:1092E00045BF00BF28FC0220A4FD02206CFC022028
:1092F0000CFC022000F0FD03012B08D1044B0022DE
:109300005A74421E504250411874FFF795BF70477F
:1093100028FC02200A4930B40B1D012253E8000F3B
:1093200040EA020443E8004595F0000FF6D120B969
:109330004B7C13B930BCFFF77FBF30BC704700BF18
:1093400028FC02202DE9F74F184D83460E4628468B
:1093500001A991469A46FDF7A3F820B3BDF8047021
:10936000D5F8008018EB07041DD018220021201D1D
:10937000FCF7D8FF0123237148F807B0BDF804209B
:10938000BDF80630C4F808A0360B9A42E660C4F86F
:10939000149002D12846FDF7B3F8FFF7BBFF002079
:1093A00003B0BDE8F08F0420FAE700BF0CFC0220F8
:1093B0002DE9F74F174D83468A46284601A9914665
:1093C0009846FDF76DF810B3BDF804602F68BC191E
:1093D0001DD018220021201DFCF7A4FF00232371BB
:1093E00047F806B00C9BA360BDF80420BDF806301A
:1093F000C4F814809A42C4E9039A02D12846FDF7C2
:109400007FF8FFF787FF002003B0BDE8F08F04204E
:10941000FAE700BF0CFC022073B50546B8B1C1F3F2
:10942000C70401F0070301269E40035D33420ED0BE
:1094300000230DF107008DF80730FEF75FFD2B5D6F
:109440009DF8070023EA06062E55FFF7E5FD02B05A
:1094500070BD000038B5094B5D686DB1FF280BD0B9
:1094600084B221462846FDF7DDFA28B12146284678
:10947000BDE83840FFF7D0BF38BD00BF5003032020
:1094800070B50F4E04460025237BAB420ED84FF635
:10949000FF732380A3700023C4E901334FF47F439B
:1094A000A381A37B23F00303A37370BD336823B1AF
:1094B000607B2844C0B2FFF7CDFF0135E4E700BF71
:1094C0005003032037B5FDF76BFA054698B14468A1
:1094D00024B10A4B01941B7833B903242846FFF7C3
:1094E000CFFF204603B030BD01A8FDF7CBF80446FE
:1094F0000028F3D0F1E70524F3E700BF20FC0220A9
:10950000FF2810B5044609D801460548FFF784FF37
:1095100021460448BDE81040FFF77EBF10BD00BFE4
:10952000140103203401032073B504780C4006466F
:109530000D4612D10DF107008DF80740FEF7DEFC55
:1095400031789DF807000D4202BF0D4335700124AC
:10955000FFF762FD204602B070BD0024FAE7F8B5BF
:10956000064600240127A5B205F0070107FA01F11C
:10957000C9B206EBD500FFF7D7FF20B90134B4F527
:10958000807FF0D125462846F8BD00002DE9F74F31
:109590001F46531E072B80460E46144600F2998044
:1095A000FF2800F2968001464D48FDF73BFA05463C
:1095B000002800F08E8031464046FDF7F1F98146E3
:1095C00038BBFF214FF6FF70FDF7EAF98146F0B195
:1095D000A0F80080867099F80D80B8F1FF0F76D161
:1095E000404B1A689B46CAB94FF6FF73A9F8003082
:1095F00089F802300023C9E901334FF47F43A9F809
:109600000C3099F80E3023F0030389F80E30112046
:1096100060E0037B9C42DED00F205BE05A68002AAA
:10962000E2D00022DBF808105FFA82FA514502D836
:109630004FF0FF0819E0DBF8040090B301230AF0B3
:10964000070103FA01F1C9B200EBDA000192FFF75A
:109650006BFF019A28B3B8F1FF0F08BFD046AAEB01
:10966000080A0AF1010AA24520D1B8F1FF0F89F8D2
:109670000D80B9D089F80C4099F80D00FDF7E2F99A
:1096800058B304EB84042401A4B2A408BE7078602B
:109690003C8025B1082E02D1A400063C8480002025
:1096A00018E0B8F1FF0F0FD14FF0FF080132B9E712
:1096B000DBF8001021B140460192FFF7CBFE019A82
:1096C00008F101085FFA88F8D045F1D3ECE70025EE
:1096D000D0E7072003B0BDE8F08F0320FAE700BF12
:1096E000140103205003032007B520B1032816D02E
:1096F00003B05DF804FB254B1B78012BF8D1244AFD
:109700002449C1F808331360C1F808331360224BB1
:109710004FF40052C3F88020204B1870E8E7002374
:109720000DF107008DF80730FEF7E8FB174B1A78AC
:10973000012A25D11948017801BB194A194911603C
:109740005A7812F0010F134A1EBFD2F8041541F0E7
:109750000101C2F80415D2F8001221F00101C2F88B
:1097600000129B780C4A5B01DBB282F80D334FF498
:109770000053C2F8803113600123037009F0A2F88E
:109780009DF80700FFF748FCB2E700BFD8010320AF
:1097900004D0004000D0004000E100E0E0010320E0
:1097A000DC010320A997020073B5002306460DF1E2
:1097B00006008DF80630FEF7A1FB214B1D78002D29
:1097C00037D1204C8DF807500DF10700FEF796FBBE
:1097D0002168636862683F2B98BF5D1C63683F2BFC
:1097E00094BF01330023A942636005D123683F2B56
:1097F00094BF013300232360134B9DF807009E5450
:1098000023686268934288BF4132D31AA2689A42A1
:1098100038BFA360FFF700FC226863683F2B94BF4A
:10982000013300239A4201BF084A0123C2F80833DA
:1098300053609DF80600FFF7EFFB02B070BD00BF5C
:1098400089FC0220B40103207001032000D00040F5
:1098500013B50DF106010446FCF7B2FF80B10A4AC8
:10986000BDF80630142101FB0323DA6852B1A27A55
:1098700042B1DA680020013ADA60A07202B010BD8D
:109880000A20FBE70620F9E7B0FD0220F7B50D46F8
:109890000DF106010446FCF793FFC0B1BDF8063098
:1098A0000C4A6168142000FB03230C33012253E8A7
:1098B000000F00EB020643E8006797F0000FF6D1B7
:1098C00029600C3169600020A27203B0F0BD0A204B
:1098D000FBE700BFB0FD022010B50B4B1A68042A4D
:1098E0000FD01968094A42F82100012253E8001FED
:1098F00001EB020043E8000494F0000FF6D10020D1
:1099000010BD0C20FCE700BF2C0303200CFA022042
:10991000028843889A4202D10148FCF7F1BD7047A2
:109920005C01032038B5094C054601462046FCF78A
:10993000B7FD40B12888236803441C220021184643
:10994000FCF7F0FC38BD0346F7E700BF5C010320DD
:109950002DE9F0411C46184B1B7806460F4615466C
:109960002BB1DFF85C80A38823B10A2000E002203D
:10997000BDE8F08198F800302BB92146A088FCF7AB
:10998000E1FE20B92060A3880133A380EBE72368C0
:109990001EB1998832889142EFD11FB119883A8857
:1099A0009142EAD19B682B6023686B60034B1B8953
:1099B0002B810020DCE700BF20FC02203CFC0220C1
:1099C000B0FD022030B587B04CF2070305460C46C7
:1099D000ADF8043003AA0F4B01A90020FFF7B8FF30
:1099E00010B1002007B030BD01A903A8FFF74EFF5A
:1099F0000028F6D10723A370019B5A882280029A7F
:109A000062609B8803F580432B8003A8FFF720FF4B
:109A10000120E7E778FB02201FB50023A0F5804076
:109A2000A1F58041CDE90233ADF80400ADF8061090
:109A300002AB0DF1060101A8FFF78AFF002818BF4D
:109A4000052005B05DF804FBF0B5FF2887B004469B
:109A50000E4615461F4629D80846FCF763FF28B373
:109A600003AA2046FFF7D8FF18B10524204607B007
:109A7000F0BD01A903A8FFF709FF04460028F4D1AF
:109A8000019BAE705A882A802FB9029B6B6003A895
:109A9000FFF7DEFEEAE73B6892009A4204D802999B
:109AA000686837F03FFFF2E70424DFE70724DDE7CB
:109AB0002DE9F04110220546A6B000212D48FCF703
:109AC00031FC35B929462846FCF72AFF26B0BDE807
:109AD000F0816A0028492748DFF89C8004AE37F0FF
:109AE00021FF382200213046FCF71CFC00245023C3
:109AF000CDE9013412AF0397502200213846FCF71C
:109B000011FC01AB02AA072138F8020BFFF79CFFFA
:109B100020F002000528D9D09DF85930032B26D813
:109B2000C4EBC402B318DDF85910B1500134BDF8CC
:109B30005D209A80A5429DF85F209A71DCD10DF1DD
:109B4000170313930DF11E0314930DF125031593C1
:109B50000BAB16930DF1330317930DF13A031893E2
:109B60000DF1410312961993E9B23846ACE743F27E
:109B70000220ABE74003032030030320F0B50223AB
:109B8000194D0B8000F580544FF6FF760830012701
:109B9000A0420ED2036801330BD04388033300EB9D
:109BA00083039C4206D20AB1012313704FF48063F1
:109BB0000B80F0BD8388B34212D0038883B18368E1
:109BC000D5F800C0634500D92B600B88B0F802C0FF
:109BD000033363440B804388033300EB8300D7E7F0
:109BE000002AF2D01770F0E778FC022070B5064D1D
:109BF0000646002455F8043B0BB130469847013423
:109C0000042CF7D170BD00BF0CFA02202DE9F04FF3
:109C1000DFF8A892DFF8888287B006464F46D9F869
:109C2000003053B99D4C9E492046FCF711FC18B1F9
:109C3000B8F802302068184438603D6829784B1E17
:109C4000052B00F2DE80DFE813F006004C004C002C
:109C5000D300D3003D0126B1924B00225A6001246B
:109C6000D0E02B79032B0AD8DFE803F0020E1A2389
:109C700001232B71FCF710FE002800F0B480894B03
:109C800000225A600E24BDE0874B1A78022A4FF05A
:109C9000000240F0E7811A705868FCF7F7FDEBE727
:109CA00000232B71814B022218689A80FCF790FBED
:109CB000E2E77E4C00262E7120687B4DFCF7E6FD26
:109CC0007B4BD4F800C05A8814235343EA18EE544F
:109CD00051682160A188C2F804C011810222A280CB
:109CE000CAE7B5F814A0AA7DDFF8BCB11423AEB161
:109CF000022A06D903FB0AB3EA88198903320A4407
:109D00001A81142303FB0ABAEB88BAF80A20C3F5B8
:109D10007F43FD331344AAF80A30A0E703FB0AB3DC
:109D200018895C6804EB8004062A5FD8DFE802F03B
:109D30002846323E1E50040041F61D54AB7D022BD6
:109D400007D9142202FB0AB2EB88118903330B44B2
:109D50001381142303FB0ABAEB88BAF80A20C3F56F
:109D60007F43FD331344AAF80A304BE0514852496F
:109D700000234360AB690360FCF722FD002865D037
:109D800002230422AB75A9182046FCF7F3FA50B35E
:109D90000E24D3E72B69002B14BF03230123AB75DB
:109DA000042205F10C0104F10800EEE7EA882969B4
:109DB0000123AB75920004F10C00E6E703290CBF08
:109DC000052306230422AB7505F10801A018DCE782
:109DD0000623AB75384B1988364B5868FCF79EFC48
:109DE00004460028AAD107B0BDE8F08F0F24A5E7EC
:109DF000002E7FF434AF2B79012B36D0D3B1022B58
:109E000045D00F241422002101A8FCF78BFA41F65B
:109E10001D539C4208BF00243B6802941A78023A02
:109E2000042A00F2EE80DFE812F0CF00DB000A0126
:109E30001201190102232B71CDE902660DF1020115
:109E4000EB68019301A8FCF7BBFC08B90A24D9E729
:109E50000298BDF802108388EB8003882B81FCF701
:109E60005DFC0446002CCDD1BDE7DFF854A001AA6B
:109E700053463146A81DFFF76BFD044650B9BAF8AA
:109E800004100298FCF74AFC04460A2CEAD141F679
:109E90001D54B7E7CAE90066F7E700BF5C0103207D
:109EA00070FC022020FC0220B0FD0220EC01032007
:109EB0003CFC02208C340020F4030320A8FD022087
:109EC00014040320002E7FF4CAAE694BDA7AAAB1DB
:109ED000DE721A78013A062A93D801A151F822F0CD
:109EE000939F02008D9F0200A19F0200A79F020086
:109EF000039E0200AD9F0200BF9F02001A78072A4E
:109F0000E7D801A151F822F0299F0200D39E020058
:109F1000D39E0200459F0200599F0200799F0200D4
:109F2000799F0200419F02001A8901321A810022A2
:109F30005A80DA724F4A1278B2FA82F252099A7251
:109F4000012207E04C4958688A884088033202445D
:109F50008A8002221A70BCE7464C5A88464914256A
:109F600005FB02420868546850608888108102220C
:109F70008A800C600622EDE70722EBE73D490022CC
:109F80009A72CA6842B9097C31B15A80FCF706FC62
:109F900067E79A7A002AF1D100221A705A8064E0A9
:109FA000FCF78CFB5DE7FCF79FFB5AE7314A5B88C7
:109FB000142101FB03235868FCF768FC51E70022D9
:109FC0005A60FCF769FC4CE701228DF804201A89DD
:109FD000ADF810209A88ADF81220DB68039310E0EA
:109FE00002228DF804201A89ADF810209A88ADF865
:109FF0001220DA6803929B7D9A1F534253418DF8D9
:10A00000143001A8FFF7F2FD00233B60B8F80020F0
:10A01000B8F802309A4202D11848FCF768FA184B97
:10A02000012253E8000FA0EB020143E8001494F072
:10A03000000FF6D100293FF4D6AE0026EFE503224B
:10A040008DF80420DA88ADF810201A89C3E70422BD
:10A050008DF80420DB88ADF81030D2E705238DF8A9
:10A060000430CEE7074B012119705A600FE700BF9B
:10A070003CFC0220B0FD0220EC0103205C01032027
:10A080006C01032020FC02204068FFF7BFBD0000E8
:10A0900010B4094B012253E8000F00EB020143E822
:10A0A000001494F0000FF6D118B95DF8044BFFF7D7
:10A0B000ADBD5DF8044B70476C010320F7B51F463A
:10A0C000324B1B7805460C46002B59D009884FF6B9
:10A0D000FF73994256D06388002B53D063689B0767
:10A0E00052D142B926890DF102013046FCF7B0FB8E
:10A0F00028B103B0F0BD13885688ADF8023001A82E
:10A10000FFF710FC014658B9BDF80230204A14216F
:10A1100001FB032358890338801B58810820E8E796
:10A12000077000238375BDF8023083826368036182
:10A130000122184B53E800CF0CEB020043E8000E5D
:10A140009EF0000FF6D1C86023880B8163888B8056
:10A15000032F04BF04238B75CE8004BF2B688B6153
:10A16000002401A84C81FFF7D3FB6C60CB682B6007
:10A17000094BAC721B892B81FFF78AFF2046B8E799
:10A180000220B6E70420B4E70320B2E720FC022057
:10A19000B0FD022078FC02203CFC022030B589B0E2
:10A1A000FF28044601921D463ED88B781846FCF7DE
:10A1B000B9FB002838D0A4F58042ADF81420A3F5EF
:10A1C0008042ADF816204A6806920A88079219461E
:10A1D00002AA2046FFF720FC0528019A0ED102238F
:10A1E00052B905A902A8FFF769FF07281ED00FD8AA
:10A1F000A8B1032009B030BD01AAF2E72AB10D4B86
:10A200001B7813B101A8FCF73DFA03230022E8E70D
:10A2100008280DD00E280CBF11200320EAE7002DDE
:10A22000E8D0029B2B60E5E70720E3E78620E1E723
:10A230001120DFE720FC022037B5074B054693E8E5
:10A2400003006C46002384E803001A462146284692
:10A25000FFF7A4FF03B030BDC819060037B50446A8
:10A260008378407B0025CDE900558DF80230FCF75E
:10A27000E9FBA0B1237B019003EB83039B006846BD
:10A28000ADF80030FCF756FB2346626833F8080B44
:10A290006946FFF783FF072815D002D878B103205D
:10A2A00011E0112811D08628F9D1A37B23F00303F4
:10A2B00043F00103A3730A4B01221A7003E0A37B4E
:10A2C00023F00303A37303B030BDA37B23F0030388
:10A2D00043F00203A373024B01221A702846F2E7EF
:10A2E0000CFE02202DE9F043364DC268064687B0C9
:10A2F0002B4600202F4699688A421AD107EB00109E
:10A300003378DFF8C480092B1AD0132B3ED0082BEA
:10A310003ED1747A002C3BD100283BD0FFF7B0F837
:10A320003046FCF71BFB98F80030A3B907B0BDE836
:10A33000F0830130082803F11003DCD10020DFE7AF
:10A34000747A2CBB30B3837B846043F00203837345
:10A35000012388F8003000231E464FEA061907EB58
:10A360000902927B910702D4D20705D524B1284671
:10A37000FFF774FF80B901230136082E05F110059F
:10A38000EBD1002BD2D188F80030CFE70124C7E70A
:10A390000024C5E70446C3E74FF6FF738628ADF8EF
:10A3A000063037F80930ADF8083016BF03900623A1
:10A3B000072301A80CBF8DF804308DF80430FCF79A
:10A3C000CDFAB3E7600303200CFE02204FF6FF73C3
:10A3D0004380FFF787BF00002DE9F0412B4F2C4948
:10A3E000DFF8AC8000238AB04FF6FF703B70CDE9F8
:10A3F0000033FCF787FB4FF6FF760446B4422AD0C1
:10A40000A4F58045ADB26B4602AA002105A8ADF8BF
:10A410001450FFF79DFA0A2804D01E4B1B7853B93D
:10A4200002251EE02046FFF76BF820464146FCF768
:10A4300069FB0446E2E7B54212D005A8FFF772FABD
:10A44000012358B1052202700371C58005A8FFF7EA
:10A450005FFAFFF71DFE0AB0BDE8F0813B70FAE736
:10A460000425142200210DEB0200FBF75BFF0723FC
:10A470008DF8143005A84FF6FF73ADF81840079516
:10A48000ADF81630FFF72EFFE5E700BFC4FD022050
:10A490003401032020FC022070B5044686B014224B
:10A4A000002101A8FBF73EFFA08923782B4D00F582
:10A4B000804080B25A1EADF80800042A25D8DFE893
:10A4C00002F00303032F440043F6FE76B042E18915
:10A4D00004D901F5804292B2B24216D8DA1E534234
:10A4E00053418DF80D30A368049363688DF80C1008
:10A4F0008BB908238DF804309DF8143043F0010324
:10A500008DF8143001A8FFF761FF2B780BB1FFF72E
:10A5100063FF06B070BD09228DF804200593F1E7B2
:10A5200043F6FE739842F0D8E389002BEDD16368BF
:10A530003BB90A238DF80430FEF7E2FF01232B70AC
:10A54000E0E70B238DF80430F8E713238DF804308F
:10A550004FF6FF73ADF80830D4E700BFC4FD02200A
:10A5600073B5154EB378054623B318B343690BB3DF
:10A57000002404740DF107008DF80740FDF7BEFCC0
:10A580000DF10600FCF792F990B1022303709DF8DB
:10A590000630456073709DF80700FEF73DFD24B955
:10A5A000064B4FF48012C3F80021204602B070BD64
:10A5B0000424F0E70824F8E798FC022000E100E01A
:10A5C0002DE9F7431E4FBB7805460E469046A3B3D0
:10A5D00098B304292FD943697BB3437C0024012B12
:10A5E0000DF107000CBF8946A1468DF80740FDF725
:10A5F00085FC0DF10600FCF759F9D0B10123037079
:10A60000104B4560D3F80435C0E90498C0E9023620
:10A610009DF806307B709DF80700FEF7FDFC24B91D
:10A62000094B4FF48012C3F80021204603B0BDE867
:10A63000F0830424EFE70724F7E70824F5E700BFD9
:10A6400098FC02200010014000E100E013B50B4629
:10A65000497A0F4C024669B9D4E901101C7A002CE2
:10A6600018BF01465868FFF7ABFF08B1FCF7CCF9FB
:10A6700002B010BD002119726369002BF8D00121CE
:10A68000ADF806008DF8041001A89847F0E700BF68
:10A690001CFA0220054B9B782BB10368187C10B97B
:10A6A00059745A6170470820704700BF98FC022017
:10A6B000F8B51F491F4B0025C1F84051C1F844515E
:10A6C000C1F84851C1F84C51C1F80051C1F80451CA
:10A6D0001B684BB3D1F8044517490968641A24F084
:10A6E0007F442F461A68A24209D8A41A15441A7C3E
:10A6F000DE691AB11F74D3E905209047AEB90F4A3D
:10A700000F4B11781B788B4205D10133DBB2022B42
:10A7100008BF0023137012780A4B43F822500A4BEB
:10A720004FF48012C3F80021F8BD3346DAE700BFCA
:10A7300000100140E403032000020320FD01032078
:10A74000FC010320F401032000E100E038B50C4BCC
:10A750000C4C4FF40032C3F8802001254FF48033B5
:10A76000C4F84833C4F808336560FBF74FFE064B66
:10A77000A56000241C60FBF749FE044B1C7038BD2B
:10A7800000E100E00010014000020320E20103208C
:10A790002DE9F04F9D4A9E49137809789D4D9942C5
:10A7A00085B035D00133DBB2022B08BF0023137014
:10A7B00099489A4B1278046853F8221063180026BF
:10A7C00023F07F430360B44630462B6823B11A68F8
:10A7D0008A420CD9521A1A604FF001082B68DFF830
:10A7E00044A201930027B6B9DFF840B265E0DF6804
:10A7F000C3F800C0891A1044DA692A60002FE4D037
:10A80000221822F07F42DE61C3E901271E46DCE701
:10A810000026B046E2E73446F6697F4A636812686C
:10A82000DFF80CC2A068991A21F07F41614500F25F
:10A83000A58001442160012222742A680023C4E912
:10A840000133E361002A40F0A2802C60CBE75A1C60
:10A850009BF80210D2B291428BF8002004BF002274
:10A860008BF80020182202FB03B31A799C68022A95
:10A870001CD0032A12D0012A1FD1207CE8B9D96844
:10A8800061601A69A2605A69E2609B69A361644BC6
:10A890001B78002B18BF01466160BEE700222B68C1
:10A8A0001146002B66D142B12B6006E029680A46AA
:10A8B0008946002A59D1002323749BF800309BF865
:10A8C00001209A42C3D12B682FB9019A9A4202D132
:10A8D000B8F1000F43D0002B73D0D3F800A0514D36
:10A8E0004D4BD5F804751C68DFF848813E1B98F87D
:10A8F000003026F07F4603369BB94FF48033C5F80D
:10A900004433C5F80433484B4FF400324FF001098B
:10A91000C3F880211A60C5F80090FBF777FD88F82E
:10A920000090B2452CBF5444A41924F07F44C5F8CC
:10A930004045D5F80435DB1B23F07F43E41B03338C
:10A9400024F07F44A3420AD9D5F80435C5F8403530
:10A95000FBF75CFD344B4FF40032C3F80021304B61
:10A9600000221A7005B0BDE8F08F94422CD09146B9
:10A97000D2699EE719740122DB6992E7D31A23F0AA
:10A980007F43834234BFC31A0023236053E7216807
:10A990001368994213D8591A1160E26155E7091AF0
:10A9A000D8691A4638B1034618688842F7D3401A66
:10A9B0001860184613462160E061DC6113E7134616
:10A9C000F2E7FFF7C3FECAE74C4511D1CB692B6014
:10A9D00073B9DFF844E00120CDE90212CAF808009B
:10A9E000CEF800300E4B1870FBF710FDDDE90212B7
:10A9F0001368D269C9F81C2012B1106803441360AF
:10AA00002B68994218BF012755E700BFFC010320BE
:10AA1000FD010320E403032000020320F4010320CE
:10AA2000E10103200010014000E100E098FC022059
:10AA3000FEFF7F00E2010320B3DF7047024B0349B2
:10AA40001878FCF781B800BF1EFC0220D9B40200C0
:10AA500010B54FF6FF7304469C42084609D1FEF735
:10AA60007EFDB0F5807F044601D14FF6FF7420468D
:10AA700010BDFF2CF9D804F0070301219940C4F35D
:10AA8000CF03C9B21844FEF74FFD0028EFD1ECE721
:10AA900073B50546FBF72EFF00240646019401A975
:10AAA0002846FBF76BFF90B974B9FF2D1BD80F49EF
:10AAB0002846FFF7CDFFFFF78FFC4FF6FF718E4260
:10AAC00002D03046FCF7CEF8204602B070BD817847
:10AAD0002846FEF7F7FC10B1052818BF0324019B98
:10AAE00001330193DBE70724EEE700BF34010320C5
:10AAF00008B5FCF79DF8FF281DBF0C234343034A0C
:10AB00004FF6FF7018BFD05A08BD00BF4EFA0220A2
:10AB100010B504464088FFF7EBFFA0802046BDE853
:10AB20001040FBF76BBF30B587B005460C461422CA
:10AB3000002101A8FBF7F6FB072301A88DF80430DC
:10AB4000ADF806500394FFF7E3FF07B030BD70B5D2
:10AB500086B006460C4615460021142201A8FBF7D4
:10AB6000E1FB3046ADF80660FFF7C2FF0D2CADF8F3
:10AB7000080019D103238DF804309DB12B7813F010
:10AB8000010F0CBF022301238DF80C3000238DF838
:10AB9000103041F20113ADF80E3001A8FBF71AFF97
:10ABA00006B070BD0223EFE7862C0BBF06230723F8
:10ABB0008DF804308DF8043018BF0394EDE730B5FC
:10ABC00087B005230D4614468DF80430ADF8060015
:10ABD000FFF78EFFADF8080001A8CDE90354FBF79D
:10ABE000F9FE07B030BD6FDF704700002DE9F0417E
:10ABF000CEB020AE502380460CADB82200213046A6
:10AC000001930395FBF78EFB0DF1970305930DF16F
:10AC1000AE0306930DF1C503079337AB08930DF10F
:10AC2000F30309930DF585730A931C4F04960DF2F7
:10AC300021130B930024444507D1E2B2002104A85C
:10AC4000FFF7D1FF4EB0BDE8F08150220021284629
:10AC5000FBF768FB01AB02AA072137F8020BFEF7EE
:10AC6000F3FE20F002000528ECD06B7C032B12D8F9
:10AC700017230DF1310203FB04630DF1450152F876
:10AC8000040B43F8040B8A42F9D111881980927899
:10AC90009A700134CFE743F20220D3E73003032058
:10ACA000F8B50D490D4DFBF72DFF4FF6FF76044625
:10ACB000A5F12007B44201D12046F8BDFF2CFBD8F6
:10ACC00021462846FBF7AEFE0028F5D0204639463F
:10ACD000FBF718FF0446EDE71401032034010320BD
:10ACE00073B5104B104C93E803006D46002385E8C4
:10ACF00003001A4629462088FFF750FA4FF6FF76E0
:10AD00002388B34201D0112801D102B070BD18468A
:10AD1000FFF7C6FF00231A4629462080FFF73EFAB8
:10AD2000EEE700BFD019060064FB0220044B1A882E
:10AD30004FF6FF739A4201D0FFF7D2BF704700BFB2
:10AD400064FB0220F0B5234B1B7885B0002533B39C
:10AD50004FF6FF70FFF7A4FF0423019301246B4417
:10AD600002AA062106460095ADF80A50ADF8084043
:10AD7000CDF80CD0FEF768FE072828D04FF6FF77F5
:10AD80002C4688B105280ED04FF6FF739E4203BFB4
:10AD9000114B1F80114B002304BF1C600123104A7C
:10ADA000137005B0F0BD0095009B3046A34224BF50
:10ADB00037461C46FFF774FFBDF808309B0001932F
:10ADC00002AA01AB06210646FEF73EFED9E723465E
:10ADD000E5E700BF7CFC022068FC022060FB02204B
:10ADE00005FE02202DE9F0418588044686B02846FC
:10ADF000FBF780FD23786080083B032B1ED8DFE83B
:10AE000003F0021F2F66637A53B93F4A116849B1B4
:10AE1000E068814206D113603C4A1580E3600DE092
:10AE2000012B0BD13A4B1B7843B1384B1B88AB42FB
:10AE300004D1237A062B01D1FFF784FF20465FE07F
:10AE4000637A002BFAD1304A11680029F6D0E06805
:10AE50008142F3D12F4913600A68013A0A60DDE7A5
:10AE60002D4F3D788DB34FF6FF70FFF719FF4FF66A
:10AE7000FF739842804619D12849FBF743FE4045AD
:10AE8000064613D100251422294601A83D70FBF780
:10AE900049FA0C2320468DF80430ADF80860ADF86F
:10AEA0000660FBF797FD01A8FBF794FD184B1B7894
:10AEB00033B1164BA2881B889A4201D1FFF742FF9B
:10AEC000002DBBD106B0BDE8F0810125EEE7124BA5
:10AED0001A78002AB2D00021142201A81970FBF7B9
:10AEE00021FA0D238DF804304FF6FF73ADF80830CA
:10AEF000ADF806302046A3680393FBF76BFD01A86D
:10AF0000FBF768FDDEE700BF08FE022068FC0220B8
:10AF100005FE022060FB022067FB022034010320B3
:10AF200038B505460C46FBF761FE80B32946194843
:10AF3000FBF701FE2378003018BF012060F3000307
:10AF400023702846FFF7D4FD4FF6FF73C01A23780D
:10AF500018BF012060F3C30323702846FBF746FEA9
:10AF600018B129460C48FBF7E6FD237860F341034E
:10AF700023702846FBF73AFE18B129460748FBF72D
:10AF8000DAFD237860F382032370002038BD43F29A
:10AF90000200FBE794F802209CF80220A0F80220AF
:10AFA0002DE9F0412B4B1B7888B00746002B4CD085
:10AFB000294B2A4C93E8030023780DF1040888E814
:10AFC000030033B1264E34684CB1112008B0BDE8FF
:10AFD000F081FFF7B7FE2378002BF6D0F2E7214A85
:10AFE000214D12882B68BA4217D1C3B114222146D1
:10AFF00003A8FBF797F9082338468DF80C30FBF7C8
:10B0000079FC0623ADF80E0003A8ADF810708DF89A
:10B010001430FBF7DFFC2046D8E75A1C17D0013369
:10B020002B6000220E4B41463846FFF7B7F8002848
:10B03000CCD0002333602B68112803F1FF332B6041
:10B04000C3D0862818BF0320C0E70820BEE713201E
:10B05000BCE700BF7CFC0220D819060005FE0220D8
:10B0600008FE022068FC022060FB0220AEDF704771
:10B07000AADF70472DE9F0470E4690B016F0100594
:10B08000804691461F46189C0CD011238DF8043041
:10B0900023788DF8053001224FF0000362F342035C
:10B0A0008DF806301C22002109A8FBF73BF98DF82A
:10B0B000246005B101AD62788DF8082042F64D2379
:10B0C000A278ADF80C308DF8092000230B22CDE9D1
:10B0D00006330E954FF0010A02AD8DF80A20089351
:10B0E00003AE199BB8F800008DF80EA004AA09A9B8
:10B0F000CDE90465ADF81C90FFF7BAFF48BB42F6F6
:10B100000813ADF80C3063788DF80830A3788DF80B
:10B11000093003466AF342038DF80A30199A3B78E6
:10B120008DF800307B78CDF81A00ADF81E008DF850
:10B13000013032F8080B8DF80EA0022304A9CDE9E6
:10B140000465ADF81830ADF81C30CDF820D007F00C
:10B150003BFF10B0BDE8F0872DE9F04391B0994670
:10B1600011238DF8043013788DF805300024012662
:10B170004FF00003154666F34203074688461C223B
:10B18000214609A88DF80630FBF7CCF801AB0E93E9
:10B190006B78A9788DF808300A238DF80A3003AB54
:10B1A0000493C1F3030202ABA24214BF1A2212227B
:10B1B000059308238DF824208DF80910CDE9064465
:10B1C00004AAADF81C3009A94B4638888DF80E60EA
:10B1D000ADF80C800894FFF74BFF11B0BDE8F08389
:10B1E000A8DF704770B50C4C054620460E46FBF7AD
:10B1F000A2FC80B12846FBF7F9FC60B1B01D04EB5E
:10B20000800029461AB1BDE87040FBF75CBDBDE87F
:10B210007040FBF745BD70BD8CF8022073B5037814
:10B220001D4E082B04462BD1437A4BBB057A072DC4
:10B230001BD0082D2AD0012D22D16A4629468088AC
:10B24000FEF702FCE0B9019B1B78CBB1A088FBF7AD
:10B2500051FB4FF6FF73984212D0104B2A461978D3
:10B26000FFF7C0FFFFF7EAFB0AE08088FBF742FB2D
:10B270004FF6FF73984203D001223178FFF7B2FFF7
:10B2800007493078FBF760FC02B070BD19460548ED
:10B29000FEF7C2F8F4E700BF1DFC02201EFC0220EE
:10B2A000A9B2020066FB02202DE9F047012186B019
:10B2B00007464048FEF738F9054600285BD0384677
:10B2C000FFF716FC4FF6FF739842804646D00122E6
:10B2D0004FF0030A01AB0821404602F10109FEF7D5
:10B2E00055F91FFA89F9064678BB02990A460323E5
:10B2F00042F804AB06313846FBF7EEFA044690B943
:10B3000008214046FBF74CFB18B30822A0F8008048
:10B310008270FEF7A3FF0446112C48D030D8CCB978
:10B320002E4625461CE00C280DD0052800D13446B9
:10B3300008214046FEF7C6F8002818BF03244A46F5
:10B34000002EC7D1E8E72E46F2E7072816D00446BC
:10B35000E2E7052421463846FFF7E5FB002635469F
:10B36000154B2A4619783846FFF73CFF1EB931467F
:10B370001048FEF751F806B0BDE8F0870C24E9E765
:10B38000862C06D043F202039C42E3D100252E46D0
:10B39000E6E71422002101A8FAF7C4FF062301A85A
:10B3A0008DF80430ADF80670FFF7B2FBEEE700262B
:10B3B000D6E700BF66FB02201DFC02202DE9F0410C
:10B3C00088B006461422002103A84FF6FF74FAF74E
:10B3D000A9FFA642ADF80E6057D03046FFF788FBB4
:10B3E000A0421ED10024032527464FF0010839460C
:10B3F0002B4622463046FBF771FA042801463BD023
:10B40000082835D00B2823D115F0020315D1C7B970
:10B41000DCB90F2303A88DF80C30FFF779FB00226D
:10B420002EE0002301AA0821FEF70EFB0028D9D147
:10B43000029B9F1D9C881D68D7E701254FF00008DF
:10B44000D5E703251C461F46F8E703253C46F5E7EC
:10B45000B8F1000FDDD0112811D043F20203984259
:10B46000DDD008B90E23D5E73046FFF75CFBD6E701
:10B47000B8F1000FF6D1CCE7B8F1000FC9D0012226
:10B48000034B30461978FFF7ADFE08B0BDE8F081F8
:10B490001CFC022030B5057885B00446BDB9408853
:10B4A000FFF78CFF0DF1070360880393FFF720FB84
:10B4B0002B4602AA0121FEF7C7FA40B9039B1B786D
:10B4C0002BB1044B608819780122FFF78BFE05B081
:10B4D00030BD00BF1EFC0220F0B52C4E87B0317885
:10B4E0000446FBF78DFB0546002842D12848FFF7AC
:10B4F000A3FA10BB264B43F2030719884FF6FF72DD
:10B500002046FBF7EDF9B84201461BD11A880132FB
:10B510001A80F2E7142201A8FAF704FF102301A809
:10B520008DF80430ADF80640FFF7F2FA012501224C
:10B5300015E02046FFF742FFF9E703212046FFF719
:10B54000F2FAF4E7082804D015D80028E2D006283B
:10B55000F4D12046FFF7CCFAFEF76EFE00220D4B29
:10B5600020461978FFF73EFE2A4631782046FFF73D
:10B5700039FE07B0F0BD43F202039842D7D043F240
:10B5800001439842D5D01128D8D1D0E71FFC022022
:10B59000100403201EFC0220FFF710BF2DE9F04F1E
:10B5A00089B00546924601938846D9B99C4BCDE9AE
:10B5B00006111B68059308AA12E9070002AB83E88D
:10B5C00007001A4641462846FFF7F9FA954B029FB5
:10B5D0001B7843B99DF811302BB90526304609B0C8
:10B5E000BDE8F08F00272846FBF74AFB012800F052
:10B5F000C580022840F0C7802FB939462846FBF79E
:10B6000077F9044633E0884B524619782846FFF70D
:10B61000E9FD2846FFF76CFA4FF6FF73984204469F
:10B62000834629D0BAF1000F26D1534605AA072137
:10B63000FEF70AFA0446002840F0DA80069B93F8E9
:10B640004420D20740F1D98003F1340202F1120103
:10B650002846FBF749F9044602E0112C18BF0324E1
:10B66000B4FA84F100224909284600F065FA862CD4
:10B6700048D1002601224AE03E7816F0010669D042
:10B680004FF6FF739C4263D16848FDF768FFB0F541
:10B69000807F63D0A04260D08346012605AB0122A3
:10B6A00007215846FDF772FF044600285AD1584634
:10B6B000FBF7E0F94FF00109044628B9394628465E
:10B6C000FBF716F9044648B107215846FDF7FAFE84
:10B6D00008B1052849D1042C08BF1124B4FA84F11B
:10B6E0004A464909284600F027FA002C3FD14EB1BE
:10B6F0004F4B284619780122FFF774FD594628461A
:10B70000FBF7B0FAA4F111035E425E410022494BFF
:10B7100028461978FFF766FD474B324619782846C8
:10B72000FFF760FD0D2C5FD031D8082C5CD00B2CBE
:10B730005AD0002C0CBF00260326019B002B3FF49F
:10B740004DAF34F008033FF449AF112C46D145E723
:10B750000026A3E74FF00209B0E7A3460126B14651
:10B760000324B1E74FF00109AEE70324B6E7002E4A
:10B770003FF47DAF5846FFF78BF978E7002F7FF451
:10B780003CAF3C4601E043F202040026BEE7862CB3
:10B7900013D043F202039C4226D0112C26D1274B12
:10B7A000424619782846FFF71DFD254B5246197869
:10B7B0002846FFF717FD002610E7204B4246197870
:10B7C0002846FFF70FFD1E4B524619782846FFF713
:10B7D00009FD019B2646002B3FF400AF3A46214667
:10B7E0002846FFF7B4F9F9E62646A6E70326A4E7BC
:10B7F00005287FF432AF112432E7598D03F1180286
:10B8000000297FF423AF03F12C01343311F8010B2D
:10B8100000287FF41BAF8B42F8D10B2420E700BF38
:10B82000E0030320E8010320F0310020140103208D
:10B83000F9310020F4310020F3310020F2310020F2
:10B84000F131002010B504464088FFF751F9237804
:10B85000A080052B06D0122B0AD02046BDE8104050
:10B86000FBF7B8B8A1686088BDE8104000F032B8B6
:10B870000C4B1B689BB10C4B217A1B7803F0010227
:10B8800091420CD8617AC3F34003994294BF0021DE
:10B890000121012300226088FFF780FEDDE70121FE
:10B8A000F7E700BFE0030320E301032010B586B0F3
:10B8B00004461422002101A8FAF734FD04230DEBFD
:10B8C00003008DF80430ADF80640FFF7BBFF06B06B
:10B8D00010BD00002DE9F04F8A4BDFF850B21B6815
:10B8E00091B00026CDE90966089308AF04460D46DD
:10B8F00097E8070005AB83E807001A46294620466B
:10B90000FFF75DF9804BDDF81490D3F800A02046D6
:10B91000FBF7B6F99BF8001005462046FBF770F9D7
:10B920002022804631463846FAF7FCFC012DCDF83E
:10B9300004B00BD1754B324619782046FFF752FC04
:10B94000B9F1000F2DD14FF6FF767DE0002D40F0CC
:10B95000CA8043F2020B00226D4B20461978FFF794
:10B9600041FC6C4B2A4619782046FFF73BFC6A4B9A
:10B97000002219782046FFF735FC684B0022197821
:10B980002046FFF72FFC3BF0080307D0BBF1110F57
:10B9900004D0059A59462046FFF7D9F811B0BDE802
:10B9A000F08F99F8003013F0010F4FF6FF7B27D18D
:10B9B0005B4BCDF82CA00F935E46012D4FF0000598
:10B9C00040F098803B464A4629462046FAF78EFFCB
:10B9D000834600287BD1002D40F08F80B8F1000F06
:10B9E00009D0019B204619780122FFF7FBFB314665
:10B9F0002046FBF737F9ABF111035D425D41AAE741
:10BA00002046FFF775F8584506460AD14548FDF728
:10BA1000A6FDB0F5807F01D0B04217D14FF0030BE7
:10BA200055E0012D15D1DFF8E4B020469BF8001059
:10BA3000FBF7E6F868B92046FFF738FF9BF80010DF
:10BA40002046FBF7DDF820B98525BBE706464FF019
:10BA5000010803AB012207213046FDF797FD1128AD
:10BA6000834634D0BBF1000FD8D1594650220498F8
:10BA7000FAF758FC049B1D70DDF810B0CDF82CA02F
:10BA80000BF1340308930BF118030C930BF1010332
:10BA90000D932046224B0F93FBF7CAF8FF28BDD029
:10BAA000214A0C2101FB002050F8042FCBF8112073
:10BAB0008288ABF8152082798BF817203046FAF788
:10BAC000D9FF05288346A9D000283FF476AFB8F106
:10BAD000000F02D03046FEF7DBFFBBF1860F8AD1A4
:10BAE0000025012238E7B9F1000F7FF45AAF4FF675
:10BAF000FF7685253B46002266E7B8F1000F3FF44C
:10BB00007AAFE7E7E0030320ACFD0220F03100202C
:10BB1000F6310020F5310020F4310020F33100200F
:10BB2000C5FD0220140103204EFA0220F931002045
:10BB30000021FFF7CFBE000070B5184B0E4686B04F
:10BB400015460A4619780446FFF74CFB26B3144BFA
:10BB50002A1C197818BF01222046FFF743FB6B1EF1
:10BB60005A425A410F4B20461978FFF73BFB0E4BC8
:10BB7000002219782046FFF735FB1422002101A886
:10BB8000FAF7D0FB012301A88DF80430ADF8064088
:10BB90008DF80C50FFF756FE06B070BDF73100204F
:10BBA000FA310020F8310020F9310020F0B587B0DB
:10BBB00004460F4616460021142201A81D46FAF736
:10BBC000B1FB03238DF80430094BADF80640002289
:10BBD00019788DF80C702046ADF80E608DF8105075
:10BBE000FFF700FB01A8FFF72DFE07B0F0BD00BF77
:10BBF000F731002030B587B005460C4614220021ED
:10BC000001A8FAF78FFB072301A88DF80430ADF8DF
:10BC100006500394FFF716FE07B030BD2DE9F04142
:10BC20001E4B0E46197804461746FAF7E9FF0146FF
:10BC300080B32046FEF75CFF194B05461978204675
:10BC4000FAF7DEFF174B00281978204614BF4FF093
:10BC500001084FF00208FAF7D3FF50B12846FEF76B
:10BC600017FF3B46324641462046BDE8F041FFF70C
:10BC70009DBF4FF6FF739D42F3D007212846FDF785
:10BC800021FC01460028ECD00528EAD02046FFF729
:10BC9000B1FFE6E73B463246E6E700BFFA31002057
:10BCA000F8310020F931002070B5094B19780446AD
:10BCB000FAF7A6FF074B054619782046FAF7A0FFCA
:10BCC0002A46014601232046BDE87040FFF766BCC6
:10BCD000F1310020F231002008B5074B1B780A46ED
:10BCE0003BB100231946FFF759FC082808BF112073
:10BCF00008BD0820FCE700BF7CFC022013B5194CEE
:10BD000023884FF6FF729A4227D0174B20881B7862
:10BD100080B223B36946FFF703F948B140F28D13AF
:10BD20000193042381B20DEB030201201BF01AFAE8
:10BD30009DF8001011F002010FD12088FFF7CCFF11
:10BD400030F0080309D04FF4CB730193042381B280
:10BD50000DEB030201201BF005FA02B010BD082014
:10BD6000DCE700BF203200207CFC02202DE9F04FF0
:10BD7000BA4B1E78A1B00446002E00F08F820388D3
:10BD8000102B40F0BB80071D0FCF09AD0FC50FCFA3
:10BD90000FC597E8070085E807009DF8285005F0D3
:10BDA000FE05062D08D0FBF7E9F99DF828305B0861
:10BDB000012B04D9022B7FD04FF6FF770FE007A9A4
:10BDC0000DF10E00FDF7FEFD0028F5D008990AA838
:10BDD0001131FBF759FA0028F1D0BDF80E70BDF80B
:10BDE00024804FF6FF73984573D09D4BDFF88892FF
:10BDF00093F800A0012251464046FFF7F3F9404670
:10BE0000FAF716FFFF2809D1CB4600255146BBF8AB
:10BE10000200FAF7F5FE002856D1E8B20C25684377
:10BE200009EB00034FF6FF7229F800201A1D0A984B
:10BE30005860A3F80280BDF82C109DF82E30918038
:10BE4000937146E0042D37D10B9FBDF82920089946
:10BE5000ADF810203A0C9DF82B308DF81A205FFABF
:10BE600082F814AA8DF81230ADF8187001F11003A1
:10BE70007FBA914613F8010902F8010B8B42F9D100
:10BE80000D22002118A8FAF74DFA4846ADF86E7059
:10BE90008DF86D80FAF742FDBDF87E305BBAADF8E3
:10BEA000143003229DF87D308DF8163005A904A8C2
:10BEB00035F02AFD002890D007A90DF10E00FDF7FE
:10BEC00081FD0028BED177E70135142D0BF10C0B55
:10BED0009CD14FF6FF739F4210D039464046FAF787
:10BEE000C1FE002314A8ADF85280ADF854708DF84F
:10BEF0005030FAF785FD14A8FFF7CCFA2388113BE0
:10BF00000D2B7ED8DFE813F00E007D0023004500E6
:10BF10007D007D007D007D00EF009B017D007D00A8
:10BF20007D00DA00237AA6883D2B4E4B30461978E7
:10BF300041F23D0518BF4FF48855FAF761FE00281D
:10BF40005FD0002229463046FFF768FE59E0A088FE
:10BF5000FAF796FE0128014608D1237AA08813F04B
:10BF6000010F14BF01220222FFF7E6FD254614222D
:10BF700035F8046F002114A8FAF7D4F90435052325
:10BF80008DF85030ADF85260169514A8FFF75AFCA2
:10BF900037E004F11006FBF7F1F814A909A8FDF742
:10BFA00011FDA0B1159D304605F14601FBF753F98F
:10BFB00030B905F12A013046FBF74DF90028ECD0E5
:10BFC000BDF82450A0884FF6FF739D4242D1A0884F
:10BFD000FEF78EFD054600220121A088FFF7ACFD8B
:10BFE0004FF6FF739D4249D10025002329461A468A
:10BFF000A088FAF777FC0146002855D0A088FFF703
:10C00000F9FD194B19491878FAF79EFD2388A58880
:10C01000522B00F03981542B00F04381502B40F01B
:10C020003681237B012B40F03281A27A012A40F035
:10C030002E81218942F60213994240F028810C4B4F
:10C040001C7828462146FFF7CDF80A492046FAF722
:10C050007BFD1CE12946FAF705FEBCE77CFC0220CB
:10C060004CFA0220F7310020F3310020A9BC020075
:10C070001DFC0220A9B202004EFA0220002314AADD
:10C0800007212846FDF7E0FC0028ADD1159D95F865
:10C090004430DB0706D4314605F14600FBF7DBF8F8
:10C0A0000028A1D03435A0E7002DAAD12B4641F2BB
:10C0B00006020021A088FFF779FDA2E714220021E3
:10C0C00014A8FAF72FF912238DF85030A388ADF891
:10C0D0005230237AC3F30002C3F340038DF8582093
:10C0E0008DF8593051E7277AA588DFF86882002F4C
:10C0F00040F096802846FEF7FBFC98F80010814639
:10C100003A462846FFF76EF8637A13F004087AD0AF
:10C11000072109AB01224846FDF738FA014698B1DC
:10C120002846FFF767FD3E4602238DF85030637ABC
:10C13000ADF8525013F0040F14BF012302238DF801
:10C1400058308DF8596020E7DDF828B0FBF716F875
:10C150000BF11103009314A907A8FDF733FC18B9DC
:10C160004F464FF6FF78BEE0BDF81C704FF6FF73E8
:10C170009F42F0D0DDF854A00BF101080AF1110341
:10C1800010220AF101014046019335F0BDFB019BED
:10C19000024618BB18F8011BC1B900998845F9D1AE
:10C1A000194600980192FBF76FF89BF81130019A3D
:10C1B00003F0FC03042B06D09AF8113003F0FC03C3
:10C1C000042B40F09A80002AC5D099E00AF10101C1
:10C1D00011F8010B20B99942FAD1E1E70022DFE71B
:10C1E0000122DDE707221F809A70FEF737F801462B
:10C1F00018B12846FFF7FEFC00264FF6FF7398455E
:10C2000040F0968090E7504B28461978FAF7F8FCF2
:10C210000646002888D04846FEF73AFC464683E7A3
:10C22000667A98F80010284606F00306FAF7E8FC4C
:10C2300000283FF4E6AE32463946284684E6434BB2
:10C24000A0881978FAF7DCFC054600287FF4D9AEFF
:10C25000A2881046FAF7CAFC08B9012327E711465D
:10C260003B48FAF768FC0028F7D03A4BA0881978C9
:10C270002A46FEF7B7FF02238DF85030A388ADF8A9
:10C280005230ADF8585080E62846FFF797F8324B09
:10C2900032491878FAF758FCFEF7D0FB21B0BDE818
:10C2A000F08F1422002114A8FAF73CF81123284635
:10C2B0008DF85030ADF85250FEF71AFCADF854002E
:10C2C000FDF7BAFF264B284619780022FEF78AFFB1
:10C2D000244B284600221978FEF784FF14A8FEF7A5
:10C2E00017FCD4E7B84607214846FAF759FB03463E
:10C2F00000287FF477AF05217BE700283FF42BAFC0
:10C30000DFF8648039462846FAF7ACFC98F800104C
:10C310002846FAF775FC0028E4D12846FFF7C6FA4C
:10C3200098F800102846FAF76BFC0028DAD1064688
:10C33000054B28461978FAF763FC00283FF4F4AE61
:10C340004846FEF7A5FBEFE6F9310020FA31002060
:10C350009CF80220F73100201CFC022099B5020055
:10C360001FFC02201EFC0220F031002070B5114B92
:10C370001868C04390FAA0F00124B0FA80F01728A2
:10C3800001D9182070BD04FA00F153E8002F42EAE9
:10C39000010543E8005696F0000FF6D1C240D207DF
:10C3A00006D51868C04390FAA0F0B0FA80F0E6E72E
:10C3B000C0B2E7E78CF8022010B50378182B0446CA
:10C3C00002D1FFF7D3FF207010BD37B50191019A5C
:10C3D00005466AB100242246214601A8FAF7ABFBC4
:10C3E00018B105EB420301329C800134142CF3D1C7
:10C3F00028462A6003B030BD2DE9F04703888488C1
:10C40000112B8CB0064642D01A2B45D0102B3BD1B5
:10C410002A4DAB68DB4300936A686B4653E8001F04
:10C4200001EA020043E8000797F0000FF6D10099F7
:10C4300001A8FFF7CAFF0DF108094FF00008019BA2
:10C44000984504D3132C10D90420FCF7B5FC39F817
:10C4500002AB00270137514605EB8700FAF720FCB5
:10C460001D2FF7D108F10108E9E721461448FAF732
:10C470002AFC21461348FAF726FCF37B012B03D054
:10C4800011482146FAF71FFC0CB0BDE8F0870C48B4
:10C490002146FAF705FCF7E7057A0C482D09012D2E
:10C4A000214606D9FAF70FFC022D21460848F0D0A4
:10C4B000E8E7FAF7F5FB21460548EAE78CF80220A1
:10C4C00094F8022090F8022098F802209CF80220AC
:10C4D000A0F80220034B1A8882420CBF18460020A5
:10C4E000704700BF38FA022070B50388112B04464C
:10C4F00043D002D8102B1BD070BD122B53D0502B21
:10C50000FAD1304BC288DB899A42F5D1038A022BDB
:10C51000F2D185882846FFF7DDFF01460028EBD0E1
:10C52000A37CDB0739D52846BDE87040FEF78EB8FE
:10C53000C37B012BE0D14FF6FF70FFF7CBFF054621
:10C5400020B90420BDE87040FAF75EBAA6881E4AFA
:10C550000680002303721368C5F80A300A30536856
:10C56000436004F11001F9F759FF164B6872DB893B
:10C57000002BC1D129463046D6E78088FFF7AAFFB5
:10C5800004460028B8D04068FDF7EAFF08B1FAF782
:10C590003BFA4FF6FF732380AEE74068FDF7E0FFFC
:10C5A0000028A9D0CEE786883046FFF793FF0546DE
:10C5B0000028A1D004F108010A30F9F72FFF6872B2
:10C5C000D8E700BF1CFA0220540103207BDF70472C
:10C5D0007ADF704776DF704775DF704737B585B211
:10C5E0002846FFF777FF034670B1164C017A227B8D
:10C5F00091420BD200F10A012846FFF7EDFFE8B1A6
:10C60000112801D0FAF700FA03B030BD00220272FF
:10C61000237C43B13B212846FFF7DCFF30F00803C1
:10C6200001D0FAF7F1F96369002BEDD000228DF803
:10C630000420ADF8065001A89847E5E71A7A0132C0
:10C640001A72E1E71CFA022064DF70472DE9F74F08
:10C650000C9CBDF834B02788002580468A46914658
:10C660002E46B8F80020B2420BDC35B12288013AE0
:10C67000D21B92B2FF2A39D8DA55002003B0BDE8A8
:10C68000F08FD8F8042052F82600019000220DF116
:10C69000030101A8FFF7D8FF0028EFD19DF8032080
:10C6A0004A4521D12288002D14BF0020022002EB30
:10C6B00009010144594519DC3DB9013292B2228089
:10C6C00003F802A022880132228022880DF10301A2
:10C6D0001A4401A8FFF7B8FF0028CFD121889DF8A0
:10C6E00003200A44228001250136BAE70C20C5E761
:10C6F0002DE9F341089CBDF824501746CDE90045CB
:10C7000002220646FFF7A2FF48B9102239463046FA
:10C71000CDE9084502B0BDE8F041FFF797BF02B090
:10C72000BDE8F0812DE9FF470023138090F82D30FC
:10C7300006460D4614463BB302A8FAF771F90028E5
:10C7400040F0FB8013880822CA54238801339BB22F
:10C750001B222380CA54238801339BB2CA18DDF8F8
:10C7600009102380E950BDF80D30938023889DF88F
:10C77000082006339BB212F0FE0218BF012223806C
:10C78000EA54238801332380B378FBB12388043330
:10C790001F2B21D802A8FAF741F9002840F0CD80DC
:10C7A00023880322EA54238801339BB21922238071
:10C7B000EA542388BDF8082001339BB2E91823808E
:10C7C000EA54120A4A70238802332380F278AAB10D
:10C7D0002388D91C1F2901D90C20AEE00221E9547D
:10C7E000238801339BB201212380E95423880B4421
:10C7F0009BB22380EA5423880B4423807268AAB139
:10C800002388D91C1F29E7D8022192F90020E95476
:10C81000238801339BB20A212380E9542388013302
:10C820009BB22380EA542388013323803389002B71
:10C8300076D1338A5BB11F23CDE9004307222B4613
:10C84000032106F11000FFF753FF002875D1338B49
:10C850005BB11F23CDE9004315222B46142106F1BD
:10C860001800FFF745FF002867D1326A002A67D118
:10C87000776A4FB3BB882188981C8A1C02441F2A00
:10C88000AAD8FE28A8D803336B54238801339BB25F
:10C89000FF222380EA54238801339BB223803A8805
:10C8A000EA54E918120A4A702088023080B22080C7
:10C8B000BA884AB1B96800294AD0284435F032F81C
:10C8C0002388BA881344238096F82C30002B79D122
:10C8D000307890B33388012B3AD023889F1C1F2FC8
:10C8E0003FF67AAF012805D1727802321A441F2A26
:10C8F0003FF672AFC3F11D039BB202A9E819ADF870
:10C900000830FAF789F8C0B93278022A40F09880E6
:10C91000BDF808209A4240F2AF80ADF8083098E0A8
:10C920001F23CDE9004306222B46022106F1080011
:10C93000FFF7DEFE00283FF47CAF04B0BDE8F087CF
:10C940002788BB1D1F2B3FF647AF1188052901D84B
:10C950000720F2E76FF4486C01EB0C039BB24FF237
:10C960007D3C6345F4D95388052BF1D96FF44860B9
:10C97000181880B26045EBD94FF6FF70814203D0A2
:10C98000834201D09942E3D80523EB552388013334
:10C990009BB212212380E954238801339BB2238068
:10C9A0001188E954E818090A4170238802339BB2C0
:10C9B00023805288EA54E918120A4A702388023305
:10C9C000238055E7B36A002BC2D04FF000084FF028
:10C9D0000C094FF0160A96F82C305FFA88F2934251
:10C9E0007FF676AFB16A09FB02F28F18BB88981CFC
:10C9F000FE283FF6F1AE208803332B542388013301
:10CA00009BB2238005F803A0238801339BB22380C7
:10CA10008A5AEA54E918120A4A702088023080B211
:10CA20002080BA884AB1B968002991D0284434F0EE
:10CA300079FF2388BA881344238008F10108CAE7E4
:10CA4000012A7FF46AAF72789342FFF466AFADF8C3
:10CA500008200821BDF80830FE2B3FF6BDAE228825
:10CA60000133AB542288013292B22280A954228829
:10CA700013442380002060E70921EBE7002370B511
:10CA800013600D460646C0B10368B3B1C08810F00C
:10CA9000030414D10846FAF7A9F8002808BF1425A2
:10CAA000EDB2142D0DD03379AB420CD9F188336837
:10CAB00005FB01351560204670BD0E20FCE7072000
:10CAC000FAE70520F8E70420F6E770B505468AB0D6
:10CAD0000C46002962D0002860D00388502B33D048
:10CAE000572B6AD0102B59D181886069002601AA82
:10CAF0000196FFF7C3FF022302AA218AA888ADF896
:10CB00000A60CDF80CD0ADF80830F9F77BFF0028AB
:10CB100044D1A369002B41D0039B1B78DB073DD593
:10CB2000019B0BB101221A701822002104A8F9F709
:10CB3000F9FB02238DF81030AB88ADF81830019B5B
:10CB400005940793A36927E08188606902AAFFF72B
:10CB500095FF1822002104A8F9F7E4FBEA8821894F
:10CB6000AB88ADF818309142029B0594079317D11A
:10CB7000298A022914D18BB1AA7C12F0010215BFB7
:10CB800001221A701A70032308BF8DF81030A369B0
:10CB900018BF8DF810100BB104A898470AB070BDEB
:10CBA000A3899342FAD1A369002BF7D005F11202B1
:10CBB00008922A8AADF82420EEE78188606902AAEB
:10CBC000FFF75CFF01460028E8D1029E3378002B76
:10CBD000E4D0182204A8F9F7A5FB01238DF8103042
:10CBE000AB880594ADF818300796ABE70028A8BFCE
:10CBF00000F160404FEA4111BABF00F00F00044B52
:10CC000000F56140C9B2B4BF195480F800137047F1
:10CC100014ED00E000F01F024009800000F16040C8
:10CC200000F5614001239340C0F8803103607047F4
:10CC300031DF70470023435082B043580193019B7A
:10CC400002B070477FB5D0F8246105460C46002E2F
:10CC500044D04FF49271FFF7EDFF02238DF80030BE
:10CC6000D0F88034C0F880340393D0F83C358DF888
:10CC70000830E36801930023C4E906336846D4E929
:10CC800000139847D5F8443173B14FF4A271284688
:10CC9000FFF7D0FFA3693BB10023A361D5F83C1592
:10CCA000E2682046FAF75AF8D5F82031A3B14FF4DC
:10CCB00090712846FFF7BEFF63696BB1D5F84C252C
:10CCC0008DF808200023A2688DF80030636101927E
:10CCD000D4E900136846984704B070BDD0F810310D
:10CCE000002BCFD04FF48871FFF7A4FFA169D0F8D3
:10CCF0003C359942C6D1E369E26873B1D0F800329D
:10CD000023F02003C0F80032E369A3612369E360E4
:10CD1000E6612046FAF722F8B4E7A361F9E70000DC
:10CD200001490248FFF78EBFE8F902200080024067
:10CD300001490248FFF786BFC4F9022000200040E5
:10CD4000F8B501F06043B3F1005F04460F4661D1CE
:10CD50000379314D242101FB0351486820B121683A
:10CD60004FF40476C1F80863242101FB03539E6944
:10CD700056B1D96900293CD020B123684FF4047220
:10CD8000C3F80423112033E09A61DF60DE614FF4C1
:10CD900088712068FFF74EFF4FF4A2712068FFF7FB
:10CDA00049FF2368C3F83475C3F83825236826BBC8
:10CDB00001221A6021792368242202FB0152526861
:10CDC00012BBD3F81001D3F84421D3F82441104307
:10CDD00002D1002CF5D00246242303FB0155002389
:10CDE0009C4214BF032018469A42AB6118BF0F2023
:10CDF000F8BD1F61DA610126C9E7D3F8002242F0CD
:10CE00002002C3F80022D5E74FF40472C3F80423CC
:10CE10000020EDE71020EBE7C4F90220F0B52F4C1D
:10CE200089B094F82930019394F828300093636A0C
:10CE300004F12E0204F12B014FF04020F9F7A4FF7A
:10CE40002746F0B994F82BC0266ABCF1000F20D118
:10CE5000217B8B1E012B1CD8626AA3699A4218D1D0
:10CE6000E269237D6262C6F34016032984F8283004
:10CE700084F8296007D100964FF040212046FAF748
:10CE800071F809B0F0BD4FF040212046F9F7F6FFE8
:10CE9000F7E7134D0FCD03AC0FC42B682360BCF133
:10CEA000000F18D04FF04022D2F8C434C2F8C43476
:10CEB00099070CD501238DF80830002387F82C3012
:10CEC0007307DED4D7E9003102A89847D9E75A079B
:10CED000F3D50223EFE78DF808C0EEE794F90220BE
:10CEE000A0F902202DE9F7439846244BC1F80833F6
:10CEF00090F82C3004468E46154603F0FF0933B1F6
:10CF00008368C1F80433112003B0BDE8F083012623
:10CF100080F82C60C0F82080944600F10C07BCE833
:10CF20000F000FC7DCF800303B606B6884F82830D6
:10CF3000EB6863626B78CEF888352B78B34213D0F8
:10CF40001BB918F1000618BF012684F82960009665
:10CF50002B79EA6871462046FAF704F82368002B1B
:10CF6000D2D184F82C30CFE784F829902B79EA6865
:10CF700071462046F9F782FFF0E700BF86420400C1
:10CF800003681F2B83BF03F01F03036001484FF0AA
:10CF9000A04070470003005007B5019001A8FFF7BB
:10CFA000EFFF019B03F5E073022240F8232003B05A
:10CFB0005DF804FB2DE9F04102680179254C034638
:10CFC0000020C2F80005242202FB0142526882B10F
:10CFD0001A682148C2F808031A68120B50B20125DA
:10CFE000400902F01F0205FA02F220301B4D45F8FD
:10CFF00020201A684FF0FF35D2F80C05D2F81485BE
:10D00000D2F80865D2F81075C2F80C55C2F814555C
:10D010001B68A842C3F80855C3F8105501D0FFF7A4
:10D02000BBFFB8F1FF3F02D04046FFF7B5FF7A1CC7
:10D0300002D03846FFF7B0FF731C02D03046FFF72E
:10D04000ABFF242303FB0141002381F820304B6018
:10D05000BDE8F081C4F902201003020000E100E005
:10D0600007B5019001A8FFF78BFF019B03F5E07363
:10D07000032240F8232003B05DF804FB07B50190BC
:10D0800001A8FFF77DFF019BD0F81005D84000F004
:10D09000010003B05DF804FB07B5019001A8FFF79C
:10D0A0006FFF019A01239340C0F80C3503B05DF87F
:10D0B00004FB07B5019001A8FFF762FF019A012365
:10D0C0009340C0F8083503B05DF804FB2DE9F04F3C
:10D0D000834608469BF8007053499BF8088041F846
:10D0E0002720524A0169524C42F82710242202FBA1
:10D0F000084287B092F82020002A40F09380D0E9BF
:10D10000006A437D0293836990F814900393D0E9F9
:10D110000215037F0193701C05D03046FFF7C9FF4D
:10D120003046FFF79DFFBAF1FF3F0AD005A8CDF8C2
:10D1300014A0FFF725FF059B03F5E07C002340F8D2
:10D140002C30DBF80400039BC0F82435029BDBF88D
:10D15000040049EA0303C0F86C35DBF80400B9F1B8
:10D16000010FC0F80C65C0F814A519D14A1C09D0EC
:10D1700005A80591FFF704FF059A02F5E072002665
:10D1800040F822606B1C05D02846FFF792FF284626
:10D19000FFF766FFDBF80420C2F80855C2F8101547
:10D1A000242202FB08F804EB0805224A44F8087020
:10D1B0006A604FF48871DBF80400FFF73BFD4FF421
:10D1C0009071DBF80400FFF735FD4FF49271DBF846
:10D1D0000400FFF72FFD4FF4A271DBF80400FFF706
:10D1E00029FDDBF804201449C2F80413DBF804001D
:10D1F000019940F30730FFF7F9FCDBF8040040F336
:10D200000730FFF707FDDBF8043000200822C5E9EE
:10D210000600C3F800250123686185F8203007B0B7
:10D22000BDE8F08F0820FAE750FC022048FB0220FE
:10D23000C4F90220296D0200100302002DE9F34118
:10D240000579374E24236B43F2180C46517F8046F4
:10D25000002962D1F3580BB10123537794E80F00F2
:10D26000242707FB056707F10C0C8CE80F00F87FFB
:10D27000FF2803D0BB7FC3B1FFF71BFF226822B199
:10D2800002F06043B3F1005F06D1A36883B103F0FD
:10D290006043B3F1005F0BD0242303FB056500233B
:10D2A0006B77102002B0BDE8F081FFF7F5FEE5E7EF
:10D2B000D8F800306168C3F84425C3F84815D4E9AC
:10D2C00002120020C3F83415C3F83825C3F818013A
:10D2D000D3F818210192019AC3F850050122C3F82E
:10D2E00040051A6124226A43B25892B9D3F8182132
:10D2F000002AFBD0242303FB0565E87FFF2803D029
:10D30000A97F19B1FFF7C8FE0020CBE7FFF7D1FED8
:10D31000FAE74022C3F80423C4E71120C2E700BFA4
:10D3200070F90220F0B51C4E85B0154607460C4634
:10D33000FAF70AFE012333704FF6FF73AB4228BFA2
:10D340002B4607B3FA1815490A60F4B1E2181449DC
:10D3500014480A60002C144A0294A5EB0305CDE999
:10D360000073694608BF002315600393FFF766FF4B
:10D37000024660B1002404200C49347028F052FBAE
:10D38000204605B0F0BD3A46DDE72246DFE7FAF772
:10D39000DBFD0120F5E700BF080403200C04032097
:10D3A0000404032028320020FC030320D91A0600BD
:10D3B00030B5154B1B7887B0044613B3FAF7C4FD9C
:10D3C00001238DF806400DF10602104C1048237021
:10D3D000CDE9022300250DF1070202A9CDE90423BE
:10D3E0008DF80750FFF72AFF024620B10949257042
:10D3F000042028F017FBFAF7A7FD9DF8070007B0F7
:10D4000030BD4FF0FF30FAE700040320080403208A
:10D4100028320020D91A0600C30914BF13020B02D8
:10D4200010F0400F70B5064614BF1046084618436A
:10D4300014460D46FFF7BCFFB1064CBF23022B027A
:10D4400016F0100F14BF204628461843FFF7B0FF10
:10D4500032074CBF23022B0216F0040F14BF2046E4
:10D4600028461843FFF7A4FFB3074CBF2002280249
:10D4700016F0010F08BF2C462043BDE87040FFF7AF
:10D4800097BF000007B5114BD3F81831D3B1104B3B
:10D49000104900221A60C87F1B680193FF28019B76
:10D4A00003D08B7F5BB1FFF7F7FD00234B770B7247
:10D4B000D1E90031084803B05DF804EB1847FFF7E5
:10D4C000F8FDF2E703B05DF804FB00BF0030004058
:10D4D0001831004070F9022078F9022007B5019058
:10D4E00001A8FFF74DFD019B00EB8300D0F800275A
:10D4F00022F44032C0F80027D0F8003743EA014355
:10D50000C0F8003703B05DF804FB00000E4B034485
:10D5100093F93020072A02DD0021FFF7DFBFD3B2E5
:10D52000072B10D8930003F1804303F5C043D3F8D1
:10D53000101521F00101C3F81015012303FA02F2BE
:10D54000024BC3F80823704704F902200060004032
:10D5500000F1804000F5C040002382B00360036802
:10D560000193019B02B070472DE9F04F002489B070
:10D57000CDE90244624D4FF48072012102F18043F3
:10D5800003F5C04390B21B68012B06D1D5F80433D4
:10D590000B4202D0FFF7DCFF0C430432B2F5907F60
:10D5A0004FEA4101EAD1574B1B68012B0ED14FF4D2
:10D5B000BE70FFF7CDFF4FF0A04344F00044D3F816
:10D5C00010350293504BD3F81035039314F0FF0F2E
:10D5D0001AD04E4F01260025264210D0AB0003F191
:10D5E000804303F5C043D3F81005D3F8101557F85E
:10D5F000253023B1C1F30141C0F30520984701351F
:10D60000082D4FEA4606E7D1002C75DA0DF118080F
:10D6100000230693C8F804304FF0FF33CDE90433FC
:10D62000DFF8E8A0DFF8E89000252F4619F9014B54
:10D63000631C48D0E4B2012324F0C00604F00702C2
:10D6400003FA02F2F00808AB191811F8103C134263
:10D6500039D00AEB0603A40993F930305AF823B005
:10D66000BBF1000F08D1032C2DD118F800C04CEAF3
:10D67000020C08F800C001E0032CF6D001A80196C6
:10D68000FFF77EFC019B11F8181C03F5E07C1142AA
:10D6900050F82C00C0F3014005D0022813D1032C10
:10D6A0000BD1214604E003280DD1032C05D1022122
:10D6B0003046FFF713FF0135EDB2BBF1000F02D08A
:10D6C00021463046D8470137042FAFD1A5B14FF0DE
:10D6D000A0430299D3F8102503F540739142D3F883
:10D6E000103502D10399994206D00292069ACDE9EB
:10D6F0000332079B059395E709B0BDE8F08F00BFA3
:10D70000006000407C6100400003005004F90220EA
:10D7100064F902202DE9F04F8A46234F8BB006466C
:10D7200011465046144604F0C0FF3B68FBB1042587
:10D73000C0EB441014FB05FB00B205FB04654FF081
:10D74000FF38043D28FA00F84FF040093B6859467D
:10D750003046984758B12B6803EA08032B602146EE
:10D76000304604F0C2FF20B1B9F10109EED100202A
:10D7700017E023463246514602A804F0D1FF214665
:10D78000019002A804F0B1FF019B003318BF0123F0
:10D790005B00002814BF5842C3F10100C0B2012849
:10D7A000E2D10BB0BDE8F08FAC340020F8B50E46E6
:10D7B000D11C48BF911D144641F387010546671EE1
:10D7C00004F0A2FF00214AB2A24201F1010100DBF4
:10D7D000F8BDBB1A23F00300B25C03F00303DB00C7
:10D7E00002FA03F32A581A432A50ECE7F0B5002551
:10D7F0004F1E6CB28C4205F1010500DBF0BD3B1BF6
:10D8000023F0030603F003039659DB0026FA03F323
:10D810000355EEE72DE9F041B3F9024014F11F057D
:10D8200048BF04F13E050F4603F1240645F34715B2
:10D83000904601462B463246384604F0A1FFB8B95F
:10D84000B4EB451F16DA6211012304F01F0403FA3A
:10D8500004F457F822301C4214BF012400242B4644
:10D8600032463946404604F08BFF2046BDE8F08141
:10D870000124F4E70446F2E72DE9F04FD1B0CDE9F9
:10D8800005015B9D95F9004048A8914622461F4638
:10D8900004F0FFFEA3000793069BA2001344194661
:10D8A000224638A8029304F0F4FE95F90060002F98
:10D8B00000F08F803246394628A804F0EAFE0DF5C4
:10D8C000807A324630AF48A9504604F0E2FE324634
:10D8D00038A9384604F0DDFE2B4628AA38A948A806
:10D8E000F9F703FC2B4628AA38A948A8D5F8A46064
:10D8F000B0472B4628AA39465046F9F7F6FBBDF942
:10D9000068310497023B1BB2002B69DCD9F8003068
:10D91000009503F001084FEA481840AADB4302EBE8
:10D92000080A03F0010330AA90445B0140AA1A449C
:10D93000039230AAD3184146039A0493504605F146
:10D940000409F9F753FE4B4640AA48A908A80094D9
:10D9500004F044FF08A908462B464246F9F784FB29
:10D9600008A908462B46069AF9F77EFB214608A827
:10D9700004F0BBFE00285FD0214608A804F0C4FED6
:10D9800008A92B46029A0846F9F76EFB08A92B4610
:10D9900052460846F9F768FBDDE903014346524663
:10D9A0000095F9F7CCFC2B4608AA30A940A8F9F756
:10D9B0009CFB224640A9059804F06BFE2246059B7D
:10D9C000079C234430A9184604F063FE51B0BDE81B
:10D9D000F08F314628A804F097FE012328936EE7C4
:10D9E0001FFA83F85B1108F01F0259F823300095E5
:10D9F000012101FA02F21A42049B13BF20270027DB
:10DA0000202600260AEB070B1F440AEB06030393AC
:10DA1000049B039A1E44334639465846F9F7E6FDFF
:10DA200008F1FF383B4600955A4631460398F9F70E
:10DA300086FC0FFA88F367E710AF224608A938463C
:10DA40000DF1600B04F025FE20AE224649465846F3
:10DA500004F01FFE2146304604F056FE0123214605
:10DA600028A8209304F050FE22465946384604F078
:10DA7000FBFD28B9224620A908A804F00AFE7FE78A
:10DA80003B68DA0709D42146384604F0E0FD224617
:10DA900049463046F9F7B8FCE6E7189BDB0707D4A0
:10DAA0002146584604F0D3FD2246494628A8F1E70E
:10DAB000002823461CDD5A463946384604F030FE1D
:10DAC0002146384604F0C3FD224628A9304604F01A
:10DAD000CBFD002805DA23464A463146304604F09D
:10DAE0004FFE234628AA3146304604F019FECEE701
:10DAF0003A465946584604F013FE2146584604F06B
:10DB0000A6FD2246314628A804F0AEFD002805DA1D
:10DB100028A923464A46084604F032FE28A923468F
:10DB20003246084604F0FCFDBEE70000084B1A68C8
:10DB3000D20706D4E02283F800230122C3F8802113
:10DB40001A604FF080430122C3F81825704700BFC8
:10DB500000E100E038B5074C051E04F1080318BFCA
:10DB60001C4623682BB11A6822605B6828469847D8
:10DB7000F7E738BD8C04032020B9034B01225A700B
:10DB8000FFF7E8BF704700BF8404032020B9054BAE
:10DB900001225A70FFF7DEBF012802D1014A9070BE
:10DBA000F8E7704784040320F0B513241C80D0F8F4
:10DBB0007C41059E4CBBD0F88041002C49D1D0F867
:10DBC0008441002C67D10020F0BDD0F87C7137F87B
:10DBD00034401F883C441C80877CECB2A742EAD9C1
:10DBE0000CFB04070135B7F814E08E454FEAC40773
:10DBF000EBD142F64D23138001239370D470D0F8FB
:10DC00007C21D25B32800120DEE700254FF00A0C38
:10DC1000E2E7D0F8807137F834401F883C441C801C
:10DC200090F87870ECB2A742C9D90CFB0407013513
:10DC3000B7F87AE071454FEAC407EAD142F64D23BE
:10DC4000138002239370D470D0F88031DB5B338073
:10DC5000D9E700254FF00A0CE2E7D0F8847137F8D5
:10DC600034401F883C441C8090F8DE70ECB2A74220
:10DC7000A9D90CFB04070135B7F8E0E071454FEA7C
:10DC8000C407EAD142F64D23138003239370D47066
:10DC9000D0F88431DAE700254FF00A0CE4E710B53C
:10DCA000138A022B86B004460FD103686BB1907CB7
:10DCB000059210F0010F14BF022003208DF804001C
:10DCC0000868029001A92046984706B010BDACDF55
:10DCD00070470000054B1B68082B01BF044B1868F8
:10DCE000B0FA80F0400918BF0020704730010010E2
:10DCF000340100108DDF704777DF7047D0E92432A0
:10DD0000D0F88C101A44D0F89830C0F894200B4406
:10DD100090F82110C0F89830D9B1D0F88410002ABA
:10DD2000BCBF5218C0F89420D0F894208A42A4BFF7
:10DD3000521AC0F89420D0F88820002BBCBF9B1842
:10DD4000C0F89830D0F898309342A4BF9B1AC0F81E
:10DD500098307047D0F89430C0F89C30D0F89830A4
:10DD6000C0F8A03070470368C91A436870B5D21A6A
:10DD7000D0E9236302FB03F4724301FB064501FB78
:10DD80001322D0F89440D0F898302C441A44C0F8AC
:10DD90009440C0F8982070BD012813B5044609D0FE
:10DDA00018B103282BD002B010BD234B0122C3F8B9
:10DDB0008020F8E700230DF107008DF80730FAF70F
:10DDC0009DF81E490B7883B94B608B600B61CB606B
:10DDD0001B4B1A7912B91B4A1A609C801A4B1B788C
:10DDE0000BB9FFF7A3FE01230B70CB680133CB60A7
:10DDF00001238B709DF80700FBF70EF9D3E7FFF7BF
:10DE000095FE00230DF107008DF80730FAF776F83C
:10DE10000A4BDA68013ADA60DA68002AEAD10B4A7A
:10DE2000012111604FF08041D1F8182412F48032A2
:10DE3000FAD19A70DEE700BF00E100E0840403201D
:10DE4000980403208DDB020089FC02200C000040B6
:10DE50002DE9F04186B005460C4617468988D0F872
:10DE600078016A469846FEF709FE10B16B6803B167
:10DE700098470098F0B1228AE389BDF83010134426
:10DE80008B4217DC04F112063146404433F04AFD60
:10DE90002B687BB104228DF80420E2893868ADF844
:10DEA0000C20228A0290ADF80E20CDE9046401A96D
:10DEB0002846984706B0BDE8F081000070B5002202
:10DEC000104905462DF03AFE2EF0C0F80E4B0F49D2
:10DED0000646032258682DF031FE044630B1002278
:10DEE000B1B22DF079FD20462CF04CFC084B18689F
:10DEF0002BF0C0FD00210446284614F035FE2046D4
:10DF000070BD00BFB22A060098340020BF2A060068
:10DF10002004032010B5838AC3F30C0413F4604378
:10DF200001D1204610BDB3F5005F02D10620604349
:10DF3000F8E7B3F5804F01D1E000F3E71B0407D504
:10DF40000022044900682DF0F9FD2EF07FF8EEE77D
:10DF50000020E7E7B531060008B542B200210220F3
:10DF6000FFF7CAFE40F2EA71BDE8084014F064BF52
:10DF700038B5054608460C462CF0F6F8002808BFD0
:10DF8000002422460F4928462DF094FD0E4B4FF6F3
:10DF9000FF72198884B18A4206D1002040F63551BB
:10DFA000BDE8384014F048BF00221888114619F027
:10DFB0008DF90828F2D1F0E78A42EED0188819F0DE
:10DFC00083F9F6E79B2A06003A320020014B1888B5
:10DFD00015F016BB3A320020014B188815F010BB23
:10DFE0002032002008B5084B1A884FF6FF71914285
:10DFF00009D018881321FEF7EDFA4FF4F171BDE84E
:10E00000084014F019BF08BD2032002007B50023D6
:10E010000846072269460093CDF80330F9F778FCEB
:10E020000A4B1A884FF6FF7191420BD018886A4646
:10E03000012119F04FF940F6DF3114F0FDFE03B075
:10E040005DF804FB43F20200F5E700BF3A3200201E
:10E0500038B500220E4905462DF070FD0446A8B9DA
:10E060000C4925F0C9F80A490446024628462DF015
:10E0700021FD2A46084920462DF01CFD00202BF0EA
:10E080009FFD0649024620462DF02BFD204638BD57
:10E09000592A06005E2A060095630600912A0600AA
:10E0A000F8B5044628B9244A136823F48043136062
:10E0B000F8BD22492CF00EFD0028F4D120462CF0AA
:10E0C00065F80546A0B11C4A1368204643F4804316
:10E0D00013602EF02DFA53EC102B10EE100A194697
:10E0E00017F08AF940F6E121BDE8F84014F0A4BE2B
:10E0F00020462CF01EF80028DAD00F4A1049136889
:10E1000043F48043136020462A462DF017FD2EF07D
:10E1100081FA2A4606460F4620460A492DF00EFD92
:10E120002EF078FA02460B463046394617F064F96D
:10E1300040F6E721D8E700BF240403202B2E060079
:10E14000302E06003C2E0600084B1A6818B142F427
:10E1500000521A60704722F400521A60044B186093
:10E16000044B01221A7014F0C3BC00BF2404032026
:10E17000DC040320D904032030B51B4B1B68DB03F0
:10E180008BB004460D462DD51C2200210DF1060052
:10E19000F8F7C8F8220A8DF80A20220C8DF80B2017
:10E1A000124A8DF80940518BADF81E1002A9099151
:10E1B0000121022312898DF81C10240E062185F0FE
:10E1C000010501A88DF80830ADF82210ADF8042043
:10E1D0008DF806308DF80C408DF80D50FAF7F6F8F2
:10E1E000FAF7CAFB0BB030BD2404032028F4022048
:10E1F00010B504462BF0B8FF094B0A49002808BFA8
:10E200000024224618682DF055FC201C18BF012060
:10E2100014F0A4FD40F2CC71BDE8104014F00CBE27
:10E22000983400209B2A06002DE9F74F464B4749BA
:10E230000746032258682DF081FC064600283CD092
:10E2400000224349DFF8088138462DF077FC31463B
:10E250008146684626F0A1FB009CF4B120462DF0D3
:10E26000E9F90022414605462DF068FC0123002211
:10E2700049468246F9F788FB10BBB5F80D3003F527
:10E280000073A5F80D302C46504629462DF050F964
:10E29000684626F076FB002CDED000982CF072FA4F
:10E2A0003946002C4CD001A826F077FB019D4DB9D2
:10E2B0003246494620462DF02EF903B0BDE8F08FD6
:10E2C0000024E1E7B5F80D3003F50073A5F80D3033
:10E2D00028462DF0AFF901222946074620462DF0A9
:10E2E0004FFD1C49804628462CF0F4FB1A49824613
:10E2F00028462CF0EFFBBAF1000F00D170B1404678
:10E300002DF098F98346B0B1BAF1000F0FD0012279
:10E3100039462DF00FFB58462CF034FA40463A4669
:10E3200029462DF0F8F801A826F02BFBBEE7394668
:10E330002DF063FDEFE7394640462DF04FF8EDE74D
:10E3400030462DF0CDFAB3E798340020E82B0600D4
:10E35000422D0600EF2B0600F82B0600F8B5054607
:10E3600008460C462BF0E5FE0646D8B100222B49A4
:10E3700020462DF0E3FB2DF05EFF002206462849E3
:10E3800020462DF0DBFB044698B12BF0C9FE80B986
:10E3900020462CF0F7F9224622490320BDE8F84038
:10E3A00027F040BB2CB122461F49032027F03AFB3F
:10E3B000344628462BF0D8FE40B33DB348F248011E
:10E3C0001A482BF0A3FC074688B1224600212DF005
:10E3D000AEFD2A46164938462DF06CFB154B164902
:10E3E00018683A462DF066FB38462CF0CBF9281C0D
:10E3F000314618BF012014F0DBFC40F2DC6114F060
:10E400001BFD2046BDE8F8402CF0BCB9094B0A4979
:10E4100018682DF096FE0025E9E700BF522E060091
:10E42000042D0600592E06008D2E060085E90200F7
:10E43000A62E060098340020AB2E06002DE9F843E6
:10E4400080460C462BF090FE30B92F494246012001
:10E45000BDE8F84327F0E6BA20462BF097FE0546C4
:10E460002046C5B12EF064F857EC106B00243246FC
:10E470003B463046394632F0DBFF30B90022234BB1
:10E480003046394632F0ACFFC8B121490120BDE821
:10E49000F84327F0C7BA2BF04CFE50B12A461D496D
:10E4A00020462DF04BFB40B12EF0B4F806460F4647
:10E4B000DDE714B122461849C9E7184F0026184D68
:10E4C000D5F804902BF02CFC1649024648462DF056
:10E4D00008FB4246144968682DF0ECFA08211348FD
:10E4E0002BF014FC054628B12146FFF737FF2846DC
:10E4F0002CF048F932463B460D4822F091F8BDE831
:10E50000F8432CF03FB900BF7E2B060000002440EA
:10E51000CF2B0600D72B0600AC2B060000409F40F7
:10E5200098340020E82B0600DF2B060029E20200C9
:10E5300035E5020037B5144C00210846FFF70EFF01
:10E540000322124960682DF0F9FA00220190104967
:10E5500060682DF0F3FA0D49054660682DF0F1FD75
:10E560000B4960682DF0EDFD019B33B12DB1012306
:10E5700001AA2946002022F075F8294601982CF0BE
:10E58000D7FF03B030BD00BF98340020E82B060051
:10E59000DF2B06001FB54FF08052D2F8A430D2F81E
:10E5A000A820D8B20290C3F307200190C2F307213C
:10E5B000C3F3074000901B0ED2B241F0C0010348E4
:10E5C0002CF086FB05B05DF804FB00BF042C0600B0
:10E5D00038B52BF0A8FB1E4D044628782BF0F8FA2E
:10E5E0001C49024620462DF07CFA68782BF0F0FAA0
:10E5F0001949024620462DF074FAA8782BF0E8FA63
:10E600001649024620462DF06CFAE8782BF0E0FA25
:10E610001349024620462DF064FA28792BF0D8FAE7
:10E620001049024620462DF05CFA68792BF0D0FAAA
:10E630000D49024620462DF054FAA8792BF0C0FA75
:10E640000A49024620462DF04CFA204638BD00BF4C
:10E650003004032097320600663506009A32060021
:10E660009E320600A2320600A6320600AA3206003A
:10E670002DE9F04786B00D46014601A826F08DF938
:10E68000019838B9044601982CF07CF8204606B071
:10E69000BDE8F0872CF0CEFF0022994906462DF008
:10E6A0004DFA0746002800F0E180002294492846F0
:10E6B0002DF044FA3946804602A826F06EF901246E
:10E6C0000298002840F0A180414638462CF030FFE7
:10E6D00000228C4930462DF031FA0746E0B1002285
:10E6E000884928462DF02AFA804638462BF0B4FE99
:10E6F000002800F0BD8040462BF0AEFE002800F060
:10E70000B780414638462CF095FC002841463846F3
:10E7100008BF00242CF00CFF00227B4930462DF06E
:10E720000DFA074610B30022764928462DF006FA66
:10E73000804638462BF047FE98B140462BF043FE0A
:10E7400078B138462CF08EFB814640462CF08AFB8F
:10E75000814506D80123002241463846F9F714F9CD
:10E7600000B10024414638462CF0E2FE0022674901
:10E7700030462DF0E3F9074680B100226349284670
:10E780002DF0DCF90146804638462CF053FC41461A
:10E790000028384608BF00242CF0CAFE00225C493D
:10E7A00030462DF0CBF9804670B12BF0C2FC40B161
:10E7B000414605A826F0F1F8DFF85491059F002F97
:10E7C00062D140462BF0DEFF0022524930462DF048
:10E7D000B5F9804670B12BF0ACFC40B1414605A8BC
:10E7E00026F0DBF8DFF830A1059F002F6CD1404602
:10E7F0002BF0C8FF30462BF0C5FF01A826F0C1F86A
:10E80000002C3FF43DAF01243DE7B8F1000F10D0DC
:10E810002CF010FF014603A819F0BAF9414604A8EC
:10E8200026F0BBF84FF00009049838B9B9F1000F91
:10E8300000D1002402A826F0A4F841E72CF0FAFE4B
:10E84000014605A819F0A4F99DF816209DF80E3090
:10E850009A4207D1BDF81420BDF80C309A4208BF87
:10E860004FF0010904A826F08CF8DDE701242FE71A
:10E8700038462BF039FB814640462BF035FBA9EB9F
:10E8800000035842584140E7B7F80D3003F50073D4
:10E89000A7F80D300022494628462DF04FF9824650
:10E8A00080B1002239462DF06BFA002808BF002401
:10E8B0002BF068FF384651462CF03AFE05A826F0AA
:10E8C00060F87BE70446F5E7B7F80D3003F5007311
:10E8D000A7F80D300022514628462DF02FF9814629
:10E8E000014638462CF0A6FB49460028384608BFAA
:10E8F00000242CF01DFE05A826F043F874E700BFA5
:10E90000EF2B0600502B0600552B0600422D06006B
:10E91000F82B0600602B0600712B060073B5054628
:10E920000E462BF0FDFB38B91549032027F07AF885
:10E930000024204602B070BD30462BF0F1FB0028C9
:10E94000F2D02BF0EDF904460028F2D0294601A8B8
:10E9500026F023F801980028EBD02CF06BFE05463A
:10E9600001463046FFF784FE18B1294620462CF0B8
:10E97000B7FF28462BF006FF01A826F002F8E9E7CA
:10E980002A2B06002DE9F04F87B000AFC7E902013E
:10E990001446002A6CD09149002024F02DFC00225E
:10E9A000054638618E4920462DF0C8F88C4902464C
:10E9B00028462DF096F800228A493D6920462DF020
:10E9C000BDF88849024628462DF08BF82BF0A8F9AF
:10E9D00080462BF0A8F900228246834920462DF07C
:10E9E000ADF88146E8B102467F4938692DF062F8FA
:10E9F000002307F1140148467B612CF07BFA0446A2
:10EA0000002844D148462AF01DFA0546786125F0D1
:10EA100077FB05F5807383422ED97449012027F0D6
:10EA200001F8B8F1000F07D0D8F8003023B1424602
:10EA30006F4938692DF03EF850462CF032FA20B17B
:10EA400052466C4938692DF035F8524641464846E1
:10EA50002CF061FDFB68002B40F0B78007F110033C
:10EA600001220021B86822F03DFF38692BF08AFEB0
:10EA70001C37BD46BDE8F08FEB1D23F00703ADEB5F
:10EA8000030D6C462A46214648462AF003FB7B6963
:10EA9000002BC6D0B8F1000FCED0BAF1000FC0D015
:10EAA000002514E0092A09D1A91C2144701ED7F8B9
:10EAB00010B02CF003FC5049024619E0911E0129C8
:10EAC00027D89B4602239E4216DA013635447B69DD
:10EAD000AB42A6D96319665D5A78082AE2D1A91C0F
:10EAE0002144701ED7F810B02CF0E8FB43490246D1
:10EAF00058462CF0F6FFE8E73BF8021F40487B60E1
:10EB00002CF0E6F8014640462CF036FF7B680233D5
:10EB1000D9E7911F012908D8A81C204419F0CEF884
:10EB2000014640462CF028FFCFE7162A2BD0212A99
:10EB300032D1A81C204419F0C1F8122383463B604F
:10EB4000BBF1000F1BD00122594650462DF018F999
:10EB50003B6878605919701CC01A214427F052FC98
:10EB60007A6803463AB130B10146386010462CF05D
:10EB700035FCD7E90032194610462CF0D9FC58462E
:10EB80002BF000FEA1E759881D482CF0A1F82DF0CC
:10EB90002DFF04238346D2E7FF2A96D1D8789B78AD
:10EBA000D7F810B043EA00202BF012F815490246BE
:10EBB00058462CF096FF291D2144F01ED7F810B0BE
:10EBC00027F020FC1049024692E7D7E90301FFF73E
:10EBD0004FFD00287FF442AF47E700BF422F0600F9
:10EBE000422D0600A12A0600742F0600522F0600AF
:10EBF000EF2B0600F82B0600502B0600792F06009D
:10EC00004D6B0600712B0600602B06002DE9F047C6
:10EC100088B000AF0023884607F108010546BB60B5
:10EC20002CF068F90446002D38D0E0B928462AF0C7
:10EC300009F90646B86025F063FA06F58073834249
:10EC400006D96249012026F0EDFE2A4660493CE0E3
:10EC5000F31D23F00703ADEB030D6C46324621464E
:10EC600028462AF017FABB68002BEED040462BF05E
:10EC70007BFA28B1574B5849186842462CF01AFFC6
:10EC800056490B6813F0400F88460AD154490120B9
:10EC900026F0C8FE2037BD46BDE8F0870028E2D147
:10ECA000D3E7504A10884FF6FF73834201D14E4993
:10ECB000EDE70968090601D54C49E8E7D7F808905F
:10ECC000B9F1100F05DD4A491022012026F0AAFEF5
:10ECD000E0E7484909781FFA89F5002944D1464EF2
:10ECE000B2F800A0B27C1FFA8AFA002A69D09A45CD
:10ECF00069D007F10C025146D6F87801FD80FDF786
:10ED0000BDFE20BBF868002859D01330D6F87C31FE
:10ED1000F8601B88AB4219D321462A4632F002FE26
:10ED20000023C7F81230FB82B38A3B820123BB74F5
:10ED3000BB1DC7E9063407F110015046FCF796F9F0
:10ED400028B9FB88AB4218BF0C2000E00C2040F62D
:10ED5000BB3114F071F800289CD1D8F8003043F092
:10ED60008003C8F8003095E71688B6B29E422AD0D4
:10ED7000DFF884A0FD8007F10C023146DAF8780153
:10ED8000FDF77CFE0028E2D1F868C0B10230082D02
:10ED9000F86004D81FFA89F2214632F0C3FD00233F
:10EDA000C7F81230FB82BAF84E313B820123BB74A4
:10EDB000BB1DC7E9063407F110013046BEE7052048
:10EDC000C5E70720C3E70820C1E700BF522F0600B0
:10EDD000AB2D0600983400203B2D060024040320B0
:10EDE000452D060020320020592D0600682D060012
:10EDF000802D0600D80403203C3200202DE9F04F7E
:10EE00009C4B91B01B681B0700AF044607D59A497D
:10EE1000012026F007FE4437BD46BDE8F08F16F00E
:10EE200049FB20462BF085F90546002800F01881A3
:10EE3000214607F1140025F0B0FDDFF860A27969E2
:10EE400089B10023BB61B1F80D3003F50073A1F85F
:10EE50000D3007F1180018F09BFE024638B18749C3
:10EE6000012026F0DFFD78692BF08CFCD3E7D7F882
:10EE70001480B8F1000F03D040462CF0DBFB804635
:10EE8000414607F11C0025F088FDF96985B179B18B
:10EE9000B1F80D3003F50073A1F80D3007F1200033
:10EEA00018F076FE024670B17549012026F0BAFDD1
:10EEB000F8692BF067FC40462BF064FC07F1140066
:10EEC00025F05FFDBBE707F128003C8C97F8226036
:10EED000FBF7B2FD08B1F9F76FFF4FF00009002210
:10EEE00007F13001388DC7F8309019F0FDFC052886
:10EEF00010D043F2030290420CD0A8B93B8EA3423B
:10EF000014D197F83230B34210D1B7F82890B9F144
:10EF1000000F0FD1386A18F0E7FE5A49044602463E
:10EF2000012026F07FFD3EE0F9F746FF3B8D0133DF
:10EF30003B85D4E7FC691CB120462CF07BFB0446E2
:10EF40000022514920462CF0F9FD00224F49064687
:10EF500020462CF0F3FD2DF06EF90022B8604C49EC
:10EF600020462CF0EBFD2DF066F9F860C6B10023C9
:10EF700007F1240130467B622BF0BCFF834620BBA7
:10EF8000304629F05FFF7862786025F0B9F87A683A
:10EF900002F5807383420ED93E49012026F042FDDE
:10EFA00030462BF0EFFB20462BF0ECFB07F11C006A
:10EFB00025F0E7FC69E7D31D23F00703ADEB030D54
:10EFC000EB46594630462AF065F87A6A002AE7D0BF
:10EFD000002179853A85494607F12802BAF80000F0
:10EFE000C7F82CB0FEF773FE40F2915113F024FFE6
:10EFF000BB6880F00100C5B213B9FB68002BCFD00D
:10F00000BAF800204FF6FF719142C9D0FB68BAF8F8
:10F010000000A7F830900022002BC7F83220FA86B3
:10F020007A6A7A8214BF0222012287F8322007F11D
:10F03000300107F11202C7E90E2BFCF717F830F088
:10F040000802ADD01328ABD043F201429042A7D0C2
:10F0500040F2A65113F0F0FE002818BF00259FE7EC
:10F06000002C3FF4D8AE22460B49032026F0DAFCF0
:10F07000D1E600BF24040320273006004F300600ED
:10F080006830060098300600C63E0600883006004C
:10F090008F300600522F0600BC30060020320020C0
:10F0A000B0B5264B264982B0044600AF02465868E8
:10F0B0002DF058F820462BF033F840B10023391DCD
:10F0C00020467B602BF016FF6CB968BB1BE0204626
:10F0D0002BF009F80028F1D1CCB1224619490320C0
:10F0E00026F0A0FC13E0F8B9204629F0ABFE054657
:10F0F000786025F005F805F5807383420AD9124936
:10F10000012026F08FFC1149032026F08BFC0837E4
:10F11000BD46B0BDEB1D23F00703ADEB030D2A4642
:10F120006946204629F0B6FF094826F029FB40F23F
:10F130002541002013F080FEE9E700BF983400204D
:10F14000B62E0600112F0600522F0600BF2E060015
:10F15000EB2E06002DE9F04F9BB000AF0D460446A4
:10F160003C22002107F12C00F7F7DCF8022387F896
:10F170002C302846062387F82F302AF0DAFF0028A3
:10F1800079D000228C4928462CF0D8FC38B12DF0DB
:10F1900052F8002814BF0223002387F82C300022E5
:10F1A000864928462CF0CAFC38B12DF044F80028D6
:10F1B00014BF0623052387F82F30002280492846F4
:10F1C0002CF0BCFC8146D0B1002307F10C01FB60A0
:10F1D0002BF090FE064600283CD1484629F032FE2E
:10F1E0008046F86024F08CFF08F58073834225D9AF
:10F1F0007449012026F016FC48462BF0C3FA284635
:10F20000002271492CF09AFC054640B13B6D6BB36E
:10F210002CF026FA3B6D188028462BF0B3FA2046D6
:10F220002AF07EFF80B3B4F80D3003F50073A4F824
:10F230000D3020466C37BD46BDE8F08F08F107035E
:10F2400023F00703ADEB030D6E46424631464846B8
:10F2500029F020FFFA68002ACED084B06B464FF622
:10F26000FF713B6519809A809E60C5E7574903206E
:10F2700026F0D8FBD0E7002DD1D055492A460320EF
:10F2800026F0D0FB0024D4E720462AF02CFF0546C8
:10F290000028C8D120462AF04CFF002800F08680C4
:10F2A00020462BF079FB0C235843073020F0070051
:10F2B000ADEB000D214607F1080025F06EFBE84696
:10F2C000DFF800A14446A946B86870BB87F85850DB
:10F2D000C7F854803F4B1B68DB030AD53E4BBB6429
:10F2E0004FF231421A803D4A127B9A700122A7F8F0
:10F2F00044201F2307F1080207F10C0107F12C003D
:10F300003B81FDF70FFA18B1354B5B68002BB9D084
:10F3100040F2F63113F090FD0028B3D107F10C0153
:10F32000388927F06FF8044683E72CF083F907F15A
:10F330000C018346C7F80C902BF0DCFD0646BBF1B0
:10F34000000F10D078B9584629F07CFDF86078603D
:10F3500024F0D6FE7A6802F5807383421BD95146A9
:10F36000012026F05FFB58462BF00CFAB86828B154
:10F37000B0F80D3003F50073A0F80D302CF066FEE8
:10F38000FB682080A380A66007F1080025F0F9FA49
:10F3900001350C3498E7D31D23F00703ADEB030DC3
:10F3A0006E463146584629F075FEDCE7002C91D0B8
:10F3B00022460C4963E700BF222C06002B2C0600D6
:10F3C000602B0600522F0600712B0600382C060019
:10F3D0006C2C0600240403203804032028F40220A7
:10F3E00098340020A22C060008B5064A136823F4BE
:10F3F0000073136014F060F940F20B21BDE808407F
:10F4000013F01ABD2404032008B5054A136843F419
:10F410000073136013F0FEFCBDE80840FEF7E2BD88
:10F420002404032008B518F037F841EC100B08BD90
:10F4300010B50F4B1B884FF6FF729BB293420446E8
:10F4400003D10C4A1288934208D00B4821F078F976
:10F450000A4A136843F00803136010BD2AF084FEC3
:10F46000002814BF20460020BDE8104015F096BDCE
:10F470003A320020203200200C2D06002404032004
:10F4800010B504462AF055FE224630B92CB10B497E
:10F490000320BDE8104026F0C5BA094B0949586859
:10F4A0002CF060FE14F020FB074B1B681B0704D5F3
:10F4B0000020BDE81040FFF7BBBF10BD832F060042
:10F4C00098340020AC2F06002404032038B5104CDB
:10F4D00010490022054660682CF030FB2CF0B6FD88
:10F4E000C3B285B143F0010098420FD064682AF09E
:10F4F0006FFB0849024620462CF0F3FA0020BDE8D5
:10F500003840FFF795BF03F0FE00EDE738BD00BFC0
:10F5100098340020482E06002DE9F04190B00646B0
:10F520000F462AF006FE40B93EB132465F4903203D
:10F5300026F078FA10B0BDE8F081002303938DF82F
:10F54000063002935A4B049303AB0693594B07932F
:10F5500001220B238DF80720ADF820300DF10702B2
:10F56000ADF82C300DF1060309920C93524A534B1F
:10F570000A924FF003080D93042202AB04A9384607
:10F58000ADF81480ADF838800F9326F0C3FF002843
:10F59000D0D003984A4D4B4C2AF042FF48B1039A11
:10F5A000494968682CF086FA236843F00803236011
:10F5B00009E0039B002B4FD1434968682CF0C1FD43
:10F5C00023685B06F0D403982BF0DCF89DF8073035
:10F5D000002B46D023683D49980658BF23686868C9
:10F5E0005CBF43F0080323602CF0ABFD9DF80630B0
:10F5F000002B4AD02368D5F80480DA0358BF23686B
:10F600004FF001005CBF43F0080323602AF0D8FAF2
:10F610002F49024640462CF064FA32462D4968686C
:10F620002CF0A0FD3A462C4968682CF09BFD029A0C
:10F630001AB1236843F008032360284968682CF056
:10F6400091FD02982BF09EF8236813F0180F28D034
:10F650000020FFF7EDFE6DE72149404626F0E2F974
:10F66000B1E72368D5F80480990648BF23684FF0B6
:10F67000000044BF43F0080323602AF0A1FA1349B5
:10F68000024640462CF02DFAB0E72368104968681E
:10F69000DB0342BF236843F0080323602CF051FDD5
:10F6A000BBE7304615F0FCFC44E700BFBC30060069
:10F6B000412D0600B42F0600B92F0600BE2F06000C
:10F6C0009834002024040320C82F0600F72F0600DA
:10F6D0000030060009300600133006001D30060019
:10F6E000D22F060013B56946044618F05BFA28B914
:10F6F0000749012026F096F902B010BD054B0649D6
:10F70000586822462CF0D6F90020FFF791FEF3E767
:10F71000C32D060098340020F92D060038B50A4C98
:10F7200005462DB9094B002C08BF1C46204638BDA4
:10F730003CB1204632F030F9013D01300444EDB2D5
:10F74000EFE7024CF2E700BF5326060044720700C1
:10F7500070B50D4C064620780D4640B1FFF7DEFF30
:10F760000A490246012026F05DF9002070BD09F02B
:10F77000F7FD074B2670186028462AF07BF9054BE9
:10F7800018600120F2E700BF28040320362A060093
:10F79000200403202C04032037B505460021052052
:10F7A0008DF80610FFF7D4FF58B1074B18682AF000
:10F7B00061F901990446284613F044FA204603B043
:10F7C00030BD0446FAE700BF2004032037B50546E4
:10F7D0000C4605200021FFF7BBFFB8B1214601A868
:10F7E00018F040F9024638B10949012026F01AF90B
:10F7F0000024204603B030BD064B18682AF03AF9C1
:10F8000001990446284613F01DFAF2E70446F0E792
:10F81000853006002004032013B5002104208DF854
:10F820000610FFF795FF50B1064B18682AF022F931
:10F830000446019813F04CFA204602B010BD04466D
:10F84000FAE700BF2004032013B50C460420002172
:10F85000FFF77EFFB0B1214601A818F003F9024678
:10F8600038B10949012026F0DDF80024204602B015
:10F8700010BD064B18682AF0FDF80446019813F0F5
:10F8800027FAF3E70446F1E7853006002004032059
:10F890002DE9FF4100228846264906462CF04EF904
:10F8A0000022254907462CF049F96946054618F01B
:10F8B00079F9044658B9294638462BF039FE1F49D4
:10F8C000032026F0AFF8204604B0BDE8F0813846AA
:10F8D0002AF058FF00221A4930462CF02FF92CF05C
:10F8E000AAFC074620B1304609F09AFD0446EAE733
:10F8F00031460220FFF72CFF20B9002428462AF0C9
:10F9000041FFE0E748210F482AF000FA04460028AA
:10F91000F3D00146022302AA3846CDE9025820F06E
:10F92000A1FE20462AF02EFF074B18682AF0A2F805
:10F930000446E3E795630600422D0600E62A06002A
:10F94000912A0600E13503002004032070B5044627
:10F950000E4600200E4923F04FFC054610B9002545
:10F96000284670BD22460B492CF0A4F82846FEF725
:10F970006FFB044628462AF005FF002CEFD03146E5
:10F980002046FFF785FF054620462AF0FBFEE7E705
:10F99000422F0600422D060070B5064650B12AF0EF
:10F9A000C8FB044630B928493246032026F03AF80D
:10F9B000204670BD0022254930462CF0BFF8054690
:10F9C0002AF0AEFB0446284624B92AF0DBFE2A467C
:10F9D0001F49EAE72AF0D6FE00221E4930462CF0E5
:10F9E000ADF82CF017FE02460B4604460D4631F0EA
:10F9F0001FFD30B9002200232046294631F0FAFCD1
:10FA000008B1154D00242B462246144820F008FE6C
:10FA1000054601460120FFF79BFE78B108211048FA
:10FA20002AF074F9044628B13146FEF797FC2046C7
:10FA30002AF0A8FE0B4B18682AF01CF8044628464A
:10FA40002AF0A0FEB4E700BFCF2C0600042D06006C
:10FA5000592E0600D72B060000409F409D32030020
:10FA60003D370300200403202DE9F041B2B00546E4
:10FA7000884601460CA819F06DFB002800F0D480E0
:10FA80000BAA1F92694A20920AAA2292684A694BDD
:10FA9000239209AA1D9325920923674AADF878306D
:10FAA000ADF88430ADF890302692ADF89C3008AABD
:10FAB000ADF8A830ADF8B43006AB28922E935F4A6B
:10FAC0005F4B29922F9307AA0B2300242B92ADF8AA
:10FAD000C0305C4ABDF83770BDF839608DF817400A
:10FAE0000DF117034046CDE90A44CDE90844CDE9BC
:10FAF00006442C9231932AF01CFB40B95249012054
:10FB000025F090FF0025284632B0BDE8F08107229D
:10FB10001DA9404626F0FEFC0028EFD00B99099A5B
:10FB200000290A4404DA079B09925B1A07930B9495
:10FB30000A98089B0028034405DA06990893091AD5
:10FB4000069100210A91D21B002AC8BF09990B987F
:10FB5000C8BF8A1AA3EB0603C8BF0992002BC8BF0F
:10FB6000089A0A99C4BFD31A0893079B099A002BD5
:10FB70001A4404DAC31A0B930023099207930698D8
:10FB8000089B0028034404DA091A0A91002108930B
:10FB90000691D71B002FC8BF099A07990698C8BFBE
:10FBA000D71BA3EB0603C8BF0997002BC2BF089A57
:10FBB000D31A0893DDE90823002B01DC002A2CDD91
:10FBC000CDE901100092DDF86B40DDE90A210CA8B7
:10FBD000A0479DF8173003B3DDE90610BDF9534087
:10FBE000099A089BA0420244B8BFADF85300BDF982
:10FBF00057008242C8BFADF85720BDF95520914249
:10FC0000BDF95920B8BFADF855100B4493420CA86C
:10FC1000C8BFADF8593019F079FAB5F80D3003F5D1
:10FC20000073A5F80D306EE705466CE72531060038
:10FC3000A69B060022310600494306002831060033
:10FC40002E3106002B3106003A31060070B592B015
:10FC500004460D46014601A8164619F07BFA80B10C
:10FC60003246294601A819F0E4F801A819F04EFA25
:10FC7000B4F80D3003F50073A4F80D30204612B02F
:10FC800070BD0446FAE7000030B593B00D4601465A
:10FC900001A819F05FFA00284CD0BDF92720BDF962
:10FCA0002B309A4244DC2AF03EF8044618B3BDF9E2
:10FCB000270029F08DFF2049024620462BF011FF36
:10FCC000BDF9290029F084FF1C49024620462BF08B
:10FCD00008FFBDF92B0029F07BFF19490246204699
:10FCE0002BF0FFFEBDF92D0029F072FF15490246E9
:10FCF00020462BF0F6FEC5B100226FF07F038DF891
:10FD00002B208DF82C308DF82D208DF82E304FF0D3
:10FD1000FF327F2301A88DF827208DF828308DF839
:10FD200029208DF82A3019F0F1F9204613B030BDA2
:10FD30000024E0E70446F8E72231060025310600FA
:10FD4000283106002B31060070B592B004460D46EE
:10FD5000014601A8164619F0FDF958B3BDF809305F
:10FD6000022D23F070039BB21ED0032D1FD0012D56
:10FD700008BF43F03003ADF809304EB1BDF809308B
:10FD8000DA064CBF83F0400383F02003ADF809305E
:10FD900001A819F0BBF9B4F80D3003F50073A4F80D
:10FDA0000D30204612B070BD43F06003E3E743F02E
:10FDB0005003E0E70446F4E770B592B004460E46FF
:10FDC000014601A8154619F0C5F978B101A8ADF8AA
:10FDD0001A60ADF81C5019F099F9B4F80D3003F51C
:10FDE0000073A4F80D30204612B070BD0446FAE747
:10FDF00000B593B0014601A819F0ACF910B101A803
:10FE0000FEF788F813B05DF804FB000000B593B06E
:10FE1000014601A819F09EF900B3BDF8180010F4CE
:10FE200060430DD0B3F5005F0CD0B3F5804F0F49A0
:10FE300018BF00211B0407D439B929F0C9FE0DE011
:10FE40000B49F7E70B49F5E70B4941F6FE731842FA
:10FE500007D0C0F30C0209482AF03AFF13B05DF84E
:10FE600004FB08462BF079FAF8E700BFAB31060037
:10FE7000A4310600A0310600E4310600AF310600CF
:10FE8000F0B593B004460E46014601A815461F463C
:10FE900019F060F908B3012E9DF81E10A8BF0126C5
:10FEA000012DA8BF012546EAE67666F3010145EA81
:10FEB000E57565F3830187F3020767F3051101A870
:10FEC0008DF81E1019F022F9B4F80D3003F5007307
:10FED000A4F80D30204613B0F0BD0446FAE7F0B5A3
:10FEE00093B004460F46014601A816461D4619F078
:10FEF00031F9A0B1189BADF8253001A8ADF81F70FD
:10FF0000ADF82160ADF8235019F000F9B4F80D30C8
:10FF100003F50073A4F80D30204613B0F0BD04467D
:10FF2000FAE700002DE9F04F2DED028BA7B08B46CC
:10FF3000154629F0F5FE8246002800F0C08058469C
:10FF40002AF06EFA002800F0BA8028462AF0F1F86C
:10FF5000002800F0908008AA1992804A1A9206AAF6
:10FF60001C927F4A7F4B1D9204AADFF804921793DC
:10FF70001F920A237C4AADF86030002600274FF01C
:10FF80000008ADF86C30ADF878302092ADF88430D0
:10FF9000042202AB17A92846CDE90867CDE9066718
:10FFA000CDE90489CDE90267229326F0B3FA00284F
:10FFB00000F085809DED028B32463B4651EC180BDC
:10FFC00031F004FA002851D1B0EE480AF0EE680A88
:10FFD0002EF0DEFC53EC102BB0EE480AF0EE680A6F
:10FFE000CDE900232EF0C4FDDDE9002355EC104BD4
:10FFF000DDE904673046394630F080FF32468046FE
:020000023000CC
:1000000089463B46204605F10041CDE90A8930F09A
:1000100075FFDDE90823CDE90E01CDE91223304655
:1000200022462B46394630F069FFDDE90623CDE94B
:100030000C01CDE91089CDE914230122594617A8F6
:1000400028F0B4FD17A824F06AFC58B117A824F0D2
:1000500037FF064617A80F4624F0ECFD17A824F03A
:100060005EFC90BB17A824F02EFC28E034463D46E9
:1000700042464B46BCE728462AF0D2F9C8B128468A
:100080002AF00FFF0628044613D12946012217A89B
:1000900028F08CFD0AAD17A824F012FFE5E8020154
:1000A00017A824F0C7FD013CF5D117A824F00BFCDC
:1000B000C3E72E49032025F0B5FC4FF0000A504657
:1000C00027B0BDEC028BBDE8F08F17A824F0F8FE36
:1000D000044617A80D4624F0ADFDDDE90A2330469D
:1000E000394630F00BFFDDE90E2380468946204675
:1000F000294630F003FF02460B464046494630F0A1
:1001000047FDDDE9122330F043FD41EC100B29F0EF
:100110004DFD014650462BF02FFCDDE90C23304607
:10012000394630F0EBFEDDE9102306460F46204647
:10013000294630F0E3FE02460B463046394630F0A1
:1001400027FDDDE9142330F023FD41EC100B29F0ED
:100150002DFD014650462BF00FFC73E77C62060034
:10016000F03206002C710600F6320600FD32060061
:100170000000F03F2DE9F04F2DED028B8DB0436A6A
:10018000059390ED048B1F02836AC0F884701E02F1
:10019000C0F88860B0EE480AF0EE680A044606939C
:1001A0002EF0F6FB59EC108BB0EE480AF0EE680A20
:1001B0002EF0DEFC94ED067B404653EC172B4946AF
:1001C0005BEC10AB8DED007B30F0C2FF0022624B88
:1001D00030F094FE0022614B30F0DAFC31F03EF951
:1001E000DDE900230790C4F88C005946504630F0F2
:1001F000AFFF0022584B30F081FE0022574B30F009
:10020000C7FC31F02BF9C4F890000546059830F092
:100210000BFE29F00043CDE908010698CDF80880CF
:10022000039330F001FEDDE90223CDE90A01DDE9A7
:10023000080130F063FED0462BF0004942468B4661
:100240004B468246DDE90A0130F058FE02460B4675
:100250005046594630F09CFCDDE9002330F04EFE5C
:1002600000223E4B30F094FC31F0F8F842464B4609
:100270008346DDE9080130F041FEDDE90A238046CE
:100280008946DDE9020130F039FE02460B46404660
:10029000494630F07DFCDDE9002330F02FFE2F4B86
:1002A000002230F075FC31F0D9F894F820305BB1C1
:1002B000226863680BEBDB71A2EB6102226000EB4A
:1002C000D072A3EB620363602368059A5B44A3606A
:1002D00063680344E360079B0BFB03F3013300FBFC
:1002E000053303EBD373D201A2EB6303C4F894305C
:1002F000079B58430130069B0BFB150505EBD57595
:10030000D80194F82130A0EB6505C4F898503BB9AA
:100310000DB0BDEC028BBDE8F08F3B44C4F89430C7
:10032000D4F89430002BF8DBD4F894309F420BDDE6
:10033000D4F89830002B0BDBD4F898309E42E7DCE1
:100340009B1BC4F89830F7E7DB1BC4F89430EBE74D
:100350003344C4F89830EBE7000070400000E03F01
:100360002DE9F04F97B00C46164629F0D9FC05460A
:10037000002800F08480002C00F081802368062B88
:100380007DD12146012207A828F010FC01AF0024EE
:1003900007A824F0EAFD013447F8040B07A824F06D
:1003A00049FC062CF4D107A824F08DFA304629F038
:1003B000C0FE30B10022354930462BF0BFFB2BF098
:1003C00045FEDDF80480059EDDF80890069FB8EB39
:1003D000060448BFA6EB0804B9EB070348BFA7EB28
:1003E00009039C42A8BF1C46002C08BF01244FF4FF
:1003F000A04393FBF4F4B4F5805F44DA40F2991320
:100400009C42B8BF1C460028C8BF4FF480544A46DF
:10041000C8BF94FBF0F4414628462BF0B7FAC4F568
:10042000805BA2460BFB0BFC0AFB0BF04FEA2C3C5B
:10043000049A40F3D3200CFB09F302FB0032039B28
:100440000AFB0AF10CFB08FC03FB00C3091301FBC8
:10045000072201FB063102F5006201F5006112136B
:1004600009132846A2442BF091FABAF5805FABEB52
:10047000040BD7DD3A46314628462BF087FA28464A
:1004800017B0BDE8F08F40F25554BCE7EB310600E1
:1004900030B593B00C46014601A8154618F05AFE37
:1004A00020B12A46214601A818F004FE13B030BD41
:1004B0002DE9F04F9BB0014609A818F04BFE28B972
:1004C0000023039303981BB0BDE8F08FBDF82930DB
:1004D0009DF82F40DB06A4F1020347BFBDF82D7045
:1004E000BDF82B60BDF82B70BDF82D60012B70D9C5
:1004F000082CB8BF082407FB04F31F33082C4FEA6D
:100500006313D8BF4FF001094FEA83030093D4BFB0
:1005100009FA04F94FF00009009B09EB490505F1C0
:100520001A0803FB068A504629F022FC0390002893
:10053000C6D029F099FE422303704D2343700C234B
:1005400083733B1280F802A0C3744FEA2A2A331245
:100550004FF0010E082C80F803A080F80A80877401
:100560000675437580F816E0047634DD0123A34058
:10057000013B0693009A0823B3FBF4F30193E310C5
:100580000593731E02FB0355431902934FF00008B5
:10059000B04597DA08F101030493029B072C03F19D
:1005A0001A0577DD4FF00009B94579DA4246494628
:1005B00009A818F07FFD2A46002308339C4202F860
:1005C000010B4FEA1020F8DC059B09F101091D44DD
:1005D000EAE704248FE79DF82F30032B14D100F1B4
:1005E0001A0200234B4502F10302BFD043F300017E
:1005F00002F8031C43F3400102F8021C43F380019C
:1006000002F8011C0133EDE7042B14D1DFF8D4C04C
:10061000034600F1300E3CF8022B111221F00701C5
:100620009976D11021F00301D200D9761A770333DD
:100630007345F0D19AE7082B17D000F11A01002278
:100640009DF82F300EFA03FC944501F103018DDD76
:10065000C2EB022393FBFCF3DBB201F8033C01F88D
:10066000023C01F8013C0132EAE7DFF87CC00346B6
:1006700000F2FD2E3CF8022B111221F007019976B1
:10068000D11021F00301D200D9761A7703337345D4
:10069000F0D16BE7DDF804B04FF0000ABA451CDB7F
:1006A000029B009ADDF810809B1A029370E74B1CA6
:1006B000424609A8079318F0FDFC069B1840079BCB
:1006C00009FA04F940EA090919465945EFD1019B95
:1006D00005F8019B9A449B44E0E751464FF000091E
:1006E000F3E700BFC22606000227060038B5FFF771
:1006F000DFFE054610B90025284638BD0BF064FA28
:10070000044628462AF03EF8002CF4D0214604483E
:100710002AF0DEFA054620462AF034F8ECE700BF5E
:100720000931060010B5FFF7E1FF044608B121F0DA
:1007300051F820462AF026F80248BDE8104020F083
:1007400087BB00BFE2C106002DE9F04F9DB0064611
:100750000D4601460BA818F0FDFC044620B9002404
:1007600020461DB0BDE8F08F8DB15C4928462AF0C7
:10077000B1F9804658B95A4928462AF0ABF90446DF
:1007800030B92A465749012025F04CF9E8E7A04640
:100790000021304607F0C0FE01218346304607F0B5
:1007A000BBFE9DF8377000FB0BF47C430734064614
:1007B000E410B8F1000F35D029F0B5FA054600284D
:1007C000CDD0584629F004FA4749024628462BF076
:1007D00088F9304629F0FCF94449024628462BF0B6
:1007E00080F9012F07D0384629F0F2F94049024636
:1007F00028462BF076F99DF83030ABB9082F05D09C
:10080000BDF8313003F00F03042B0DD1002239491C
:100810000B982BF093F90246364928462BF061F9E4
:100820002C469DE703344546204600212AF046FD2C
:10083000044618B9284629F0A5FF91E70146002291
:1008400002A824F0B9FCB8F1000F0CD15FFA8BF1CB
:1008500002A824F03EFCF1B202A824F03AFC39468A
:1008600002A824F036FC0026B1463346B24627E003
:100870001A4651460BA8009318F01CFC0AF1010A15
:1008800009FA07F9D34549EA000907EB0602009B7C
:1008900002DC01334FF0000A16460AE0083E29FA4E
:1008A00006F1C9B202A8CDE9003224F012FCDDE95C
:1008B0000032072EF2D8D6086FF0070101FB06269A
:1008C000DDE902129142D3D3059829F05BFFB8F11C
:1008D000000F3FF445AF22469EE700BFEB44060001
:1008E00013390600E2300600F8300600FE3006003C
:1008F00005310600D04206002DE9F843D0F89C707F
:100900007F3706460D4602D50020BDE8F883D0F8B3
:10091000A0207F32F8D4D0F88430BB42F4DDD0F888
:1009200088309342F0DDF46A082C4FEA272006F164
:1009300060084FEA2227D6E90E1216D1736D0244E1
:1009400003FB0722404625F0A9FA336F0BB1326E44
:100950009B5C726B9A42D7D0326C1AB1716C0B40AF
:1009600032F813302B600120CFE7736A03FB0707CF
:100970007C4302EBE402404625F090FA346F0CB160
:10098000336EE45C4FF00809F36A4B4508DC326DC6
:1009900022EA07077B43F26C24FA03F31340D8E7FB
:1009A000404624F011F92102346F0CB1336EE45C3F
:1009B0000C4309F10809E7E72DE9F04F144695B01B
:1009C0000D4607463C2200212046F5F7ABFC2846A1
:1009D00029F0AFFB002850D0AA49284625F070FD29
:1009E00000284AD0294603A818F0B4FB002842D0BA
:1009F0009DF81060002E3ED1BDF813302360BDF885
:100A0000153063609DF81730A36032469E49284632
:100A10002BF094F805462AF060F86061284629F02A
:100A2000B1FEA661237B13B94FF0FF332361E36965
:100A30005BB9A368012B40F03D813A69A286FA6850
:100A4000E28604F13402E2612362606929F0BBFCB2
:100A5000064648B12168002906DD6368002B03DDE6
:100A6000A368202B40F36C810120884924F0DAFF31
:100A7000606929F087FE00265EE0284629F059FBD0
:100A8000064600286FD00022814928462BF056F8F0
:100A90002BF0DCFA00227F49206028462BF04EF82C
:100AA0002BF0D4FA00227C49606028462BF046F8EF
:100AB0002BF0CCFA0028D4BF0123A0604FF0000235
:100AC0007649D8BFA36028462BF038F8031C18BF1E
:100AD000012323732BF0BAFA0022206170492846C3
:100AE0002BF02CF8064678B329F0FDFA40B3B38812
:100AF000022B25D1002303A9304603932AF0FAF9EB
:100B0000E061304629F03EFE039B102B05D9B3F57A
:100B1000807F06D00023E36108E0624ADA40D10713
:100B2000F8D5013B2362012384F82430E6695EB9DD
:100B30005D49012024F076FF304615B0BDE8F08F06
:100B4000304629F01FFEF1E700224F4928462AF0DF
:100B5000F5FF054629F0C1FF6061284629F012FE25
:100B60000023A3615EE7284629F02DFC58B12846F2
:100B700029F0B9FA70B9B5F80D3003F50073A5F88E
:100B80000D3065610AE0284629F0ADFA0028EED163
:100B90004649CEE7284629F0A0FF60610021606940
:100BA0002AF041F80121206060692AF03CF8022116
:100BB000606060692AF037F80206A0602CD5012336
:100BC00000F07F00A0602373032160692AF02BF8F6
:100BD00004232061A568A3616B067FF523AF05F0B0
:100BE0003F05012303FA05FB0BF1FF38022DA56039
:100BF000C4F8208084F8243026DC04F13409A66986
:100C00004FF000084B46D84508DBE361022303FAA6
:100C100005F5A3692B44A4E70323DBE731466069AC
:100C200001932AF000F8B21C8246711C60690092A0
:100C300029F0F9FF009A019B4AEA002029F8020BEB
:100C400008F101081646DEE7082D16DC002303A98B
:100C500060690393D4F818902AF04CF9A368082B24
:100C60000BDC50B10223AB40039A4B4493423FBF8D
:100C7000A369C4F82080C018E061E369002BC5D1E6
:100C80000B4956E702290600D0420600D12906008A
:100C9000F8300600FE300600053106000B2906007C
:100CA00017290600140101001F2906009C290600CF
:100CB0006A290600022B12D13B69A38655213846CA
:100CC00017F0F2FFAB21E086384617F0EDFF2087E2
:100CD000FB68638704F13403E3610323B4E6FA7A23
:100CE000102A12D1032B03D1204BE3610723ABE67B
:100CF000042B03D11E4BE3610F23A5E6082B7FF4E1
:100D0000A4AE1C4BE361FF239EE6082A04D1042B0A
:100D10007FF49BAE184BEEE7032A7FF496AE042BCC
:100D200007D1134BE3610F232362012384F824309E
:100D30008BE6082B7FF489AE0E4BE361FF23F3E7CC
:100D400001229A40013A072BA262DCBF082292FBE3
:100D5000F3F203FB01F303F10703D4BF02F1FF3207
:100D60000022DB10E2622363E6E600BFA226060053
:100D7000C226060002270600E22606000000000048
:100D80002DE9F04F2DED028BB1B002AF7862F96121
:100D9000014607F174007A6018F0DCF9002800F0D1
:100DA0002182ADF5287DF86929F0BAF90DF1080A1C
:100DB000834620B1FB6983B11D68042D0EDD04223A
:100DC000BF49032024F02EFE00237B62786ABC37E3
:100DD000BD46BDEC028BBDE8F08FFD6942F2107399
:100DE0009FEDB38BC7E90E33C7E90C3300230AF13B
:100DF00024043B623B6AAB4269DBB24A3A65B24AC1
:100E0000B24BFA6507F134027B647A660923B04A73
:100E1000A7F8483007F13C04A7F8543007F138062A
:100E2000A7F86030BA66A7F86C30042207F13003E7
:100E300007F1440178683B67FC64BE6525F06AFBF6
:100E40007A6BFB6B1344013B3A6BFB62BB6B134445
:100E5000013BBB6207F1280300280093324607F1EB
:100E60002C03214607F1740008BF4FF0000B17F068
:100E70007AFFB7F8793013F0700F0CBFD7F8A39052
:100E8000DFF86C92BBF1000F11D054460026AE4241
:100E9000C0F2E980BC6BBB6AA34280F205810024EA
:100EA0000AF16C064FF0A808AC42C0F28C81002415
:100EB0000AF1380AA826AC42C0F28C817B6A7A6AB1
:100EC000B3F80D3003F50073A2F80D307EE7D7E9D3
:100ED00007012AF0BDFB064629F02BF980460028C1
:100EE00000F0AE8000227B4930462AF027FE2246E1
:100EF000B861014607F17400FFF75EFD002800F0BD
:100F0000B0800022714930462AF018FE2BF09EF87E
:100F100000226C4944F8240C30462AF00FFE2BF0D6
:100F200095F8002244F8200C6B4930462AF006FE62
:100F30002BF070FB21F000437B61386180468946CD
:100F40004FF0FF32654BD7E9040130F071FA002809
:100F50007FD14FF0FF32614BD7E9040130F05EFAE8
:100F6000002876D1002200234046494630F042FA5C
:100F700000286ED144E903890022594930462AF0FD
:100F8000DDFD2BF047FB21F00043FB60B86080469D
:100F900089464FF0FF32514BD7E9020130F048FA51
:100FA000002859D14FF0FF324C4BD7E9020130F005
:100FB00035FA002850D144E90589002249493046D4
:100FC0002AF0BCFD2BF037F90022474904F8040C45
:100FD00030462AF0B3FD2BF02EF93B6A04F8030CDF
:100FE000A82000FB03A0FFF7C5F800223F493046C8
:100FF0002AF0A4FD2BF01FF9F0B954F8243CFA6B49
:101000009342B8BFFB63BA6B54F8203CF96B934230
:101010007A6BB8BFBB6354F81C3C0A449342C8BF08
:101020005B1A3A6BB96BC8BF7B6354F8183C0A442F
:10103000934201DD5B1A3B63B86929F0A3FBD846F4
:10104000304629F09FFB3B6A01333B62A834C3461C
:10105000D0E604ED038B8FE79FED177B04ED057B56
:10106000ABE78346E8E7D4E90E1204F1600024F010
:10107000A3F82046D7E90E21FCF775FE0136A83407
:1010800005E701FB02A0FCF765FE0132AA42F8DB8E
:10109000FE6BFB6AB3422DDA00264FF0A808AE4281
:1010A000C0F28B800134F6E60022A821EEE700BFF3
:1010B000000000000000F03F000000000000000001
:1010C0004A3106007C620600F83006002C710600EA
:1010D000FE3006007E310600F0320600FFFFEF7F93
:1010E000F6320600843106008B310600923106008C
:1010F000ED90040000233B6405F1FF384FF0A80B8E
:10110000B8F1000F1EDB0BFB08A3184607F14001E6
:101110003B62FFF7F1FB3B6AD8B193F848305BB113
:101120003A6C530B510A03F0040301F002010B4324
:10113000C2F3001213433B643B6C2246314607F175
:101140007400C84753464FF0000CAC4504DB013631
:101150009FE708F1FF38D3E7D3F89C10D3F88C2031
:10116000D3F8A0000A44D3F89010C3F89C20411A89
:1011700093F82100C3F8A010D8B1D3F88400002A56
:10118000BCBF1218C3F89C20D3F89C208242A4BF95
:10119000101AC3F89C00D3F888000029BCBF0918B6
:1011A000C3F8A010D3F8A0208242A4BF121AC3F83B
:1011B000A0200CF1010CA833C7E708FB06A0FCF740
:1011C0009DFD01366BE708FB04F30134F05829F06C
:1011D000D9FA69E606FB04F301345AF8030029F052
:1011E000D1FA68E67862F1E52DE9F04FE7B00C46F8
:1011F000059001462BA891469A46DDF8C08117F06C
:10120000A9FF28B900230593059867B0BDE8F08FC2
:101210001CAA21462BA8FFF7CFFB0028F2D0002400
:10122000DDE9211213A80E9423F0C6FFB8F1000FD8
:1012300068D11C9B4B445A1E1D9B12925344013B88
:101240003C93BDF8B13013F0700FCDE9109A18D06F
:10125000AF4F554600241D9B5344AB4250DC1698BB
:1012600029F090FA219829F08DFA2BA817F04EFF5B
:10127000059B059AB3F80D3003F50073A2F80D3005
:10128000C2E73CAB009311AA12AB10A92BA817F030
:101290006AFD0028DCD1DDF8DB70DAE713A823F063
:1012A0003AFF40EA08200E9008341E9BDDF8388093
:1012B000A342F3DCE41A2698209A28FA04F30340A8
:1012C0009A4216D0239919B1249A134031F8133059
:1012D0009DF894204AB15A0B590A02F0040201F019
:1012E00002010A43C3F3001313432A4631462BA8D5
:1012F000B84701361C9B4B44B342D6DC0135AAE704
:101300004E46F7E7404628F014FF0028A7D02246B3
:10131000804940462AF012FC2BF07CF921F000476E
:101320000D464FF0FF327C4B3946044630F080F8D2
:1013300070B94FF0FF32784B2046394630F06EF8E6
:1013400030B9002200232046294630F053F808B176
:10135000724D00240022724940462AF0EFFB2BF028
:1013600059F9CDE90201DDE9026323F000474FF0AE
:10137000FF32694B304639464FF0010B30F058F8D8
:1013800040B94FF0FF32644B3046394630F046F8F2
:1013900000B983468BF0010B4FF0FF325E4B3046B5
:1013A00039465FFA8BFB30F043F838B94FF0FF3223
:1013B000594B3046394630F031F898B145EC104B76
:1013C0002DF052FB204653EC102B29462FF0DEFB6C
:1013D000002200232FF0FAFF002854D19FED4A7B12
:1013E0008DED027B1CAF0FCF45AE0FC60FCF0FC6E2
:1013F0000FCF0FC697E8070013AF86E80700CDE9C7
:101400003C9A0FCF54AE0FC60FCF0FC69DED027B97
:101410003B6833603CA800238DED407B8DF8113193
:10142000CDE942458DF810B1FEF7A4FE3C9B0F9329
:101430003D9B10933E9B013B11933F9B12AE013BA2
:10144000336010AA11AB0FA900962BA817F08BFCE4
:10145000DDE90F123CA8FCF786FCBDF8B13013F0B3
:10146000700F40F0C380DDF8DB70109C3368A3423E
:1014700080F2BE8054AD0FCD13AC0FC40FCD0FC49E
:101480002B682360EBE6BDF8B13013F07008A5D1EE
:10149000204629462FF0E2FFCDE9088A07461D9B2A
:1014A000089A934211DC1C9A02FB079207FB03A7E0
:1014B0003CAB1292009311AA12AB10A92BA8CDE954
:1014C000109A3C9717F04FFCC9E61599139ADDF86E
:1014D00024B0CDF808808A180C920E9A0B9213ABA8
:1014E000002206920A93069BBB421BDB099BDDF898
:1014F0000880002FA8BFDB190993089B01330893CC
:10150000CDE700BFAFF30080000000000000000046
:10151000ED900400F0320600FFFFEF7F0000F03F87
:10152000F6320600069B43B10C9A21990A9824F0E2
:10153000B5FC0B9B0E93CDF808804D460023079316
:10154000079A1C9B93420EDC069B01330BF1010BA7
:101550000693C8E70A9823F0DEFD029B40EA0424C4
:1015600008330E9402931E9B029A0E9C9342F1DC68
:10157000D31A26980293DC40209B0440A34233D028
:10158000BDF8C9305B452FDCBDF8CD305B452BDBAA
:10159000239A1AB1249B1C4032F814409DF89430D1
:1015A0004BB1630B620A03F0040302F0020213431F
:1015B000C4F300141C437B190D93BDF8C730AB4234
:1015C0000BDCBDF8CB30AB4207DBDDF8DB305A4635
:1015D0001E46294623462BA8B0470D9B01359D4248
:1015E000EBD1079B0133AAE73D44FAE7184F3CE7EC
:1015F0003CA8FCF7AFFB0F9D119BAB4204DA3CA863
:10160000FCF77CFB013431E70EA93CA8FFF774F925
:1016100098B19DF838315BB10E9A530B510A03F023
:10162000040301F002010B43C2F3001213430E93B3
:101630000E9B224629462BA8B847639B5F9A13440A
:101640006393609A649B9B1A64930135D4E700BF4F
:10165000ED90040070B594B004460E46014603A810
:10166000154617F077FDC0B13346BDF92420BDF90A
:101670002210009503A817F073FC03A8ADF82260B0
:10168000ADF8245017F042FDB4F80D3003F50073A7
:10169000A4F80D30204614B070BD0446FAE7F0B54A
:1016A00095B004460D46014603A816461F4617F09E
:1016B00051FD98B11A9B009332463B46294603A838
:1016C00017F04EFC03A817F021FDB4F80D3003F518
:1016D0000073A4F80D30204615B0F0BD0446FAE7BB
:1016E0002DE9F04F9FB00646894601460DA817F038
:1016F00031FD00283BD0BDF8484004F460480FFAA3
:1017000088FBBBF1000FC4F30C0433DA0022364926
:1017100030462AF013FA00223449054630462AF0B2
:101720000DFA2AF093FC074648462AF0DDFD4FF0FB
:10173000060901468246002204A823F03DFD09FB6C
:1017400004F302930026A3000193B146DDE90421CE
:101750008A4212D3079829F015F8284629F012F882
:10176000504629F00FF8B1454846B8BF30461FB083
:10177000BDE8F08F00273D46D6E7089939B1895C6E
:101780000A2904D14E45B8BF4E464FF00009B8F1C2
:10179000000F07D12046F6F7F5FB814404A823F09B
:1017A00013FAD3E7B8F5005F02D1019B9944F5E73E
:1017B000B8F5804F01D1029BF8E7BBF1000FEDDADD
:1017C0002846039128F0FFFD48B10399B942E5DBB3
:1017D000C91B284629F027FA00FB0499DEE72846B2
:1017E00029F03EFFF8E700BF8D3206009232060076
:1017F0002DE9F04FE3B083460C46984601469DF82C
:10180000B031109326A8924617F0A4FC002800F0EF
:101810005C82BDF8AC3026A803F46042C3F30C0927
:101820000492FCF777FBBDF910300B90002B11935D
:1018300080F29780049BB3F5204F00F09080B3F5C1
:10184000404F14BF012304230022B4490293584699
:101850002AF074F900220D90B14958462AF06EF929
:1018600000220990AF4958462AF068F92AF0EEFBA9
:1018700003909DF8B220BDF89D30ADF8543002F0D1
:101880003002102A9BB274D183F03003BDF89F2040
:10189000ADF89D300AF10103C246A2EB03089DF8A2
:1018A000B23003F00303012B0DD821465846FFF751
:1018B00017FF9DF8B23003F0030303FB000000EBB9
:1018C000D070AAEB600A9DF8B230C3F38103012BFC
:1018D0009FBF0B9A03FB022303EBD373A8EB6308B0
:1018E000BDF8B3300893BDF8B5300693BDF8B730F6
:1018F0000793BDF8B9300593BDF89D30DB0607D5D9
:10190000089B069A08920693079A059B07930592EF
:1019100020462AF0E9FC0022129001461DA823F07F
:101920004BFC029A01239340013B1893062303FBCF
:1019300009F317934FEA89031693C2F1080354463B
:101940001B93DDE91D239A4246D21DA823F0E3FB39
:101950000A2805462CD10B9B54469844F1E70223F4
:1019600072E701230022CDE90232002309930D938F
:101970007FE7202A0ED183F06003BDF89F20ADF8E9
:101980009D300AF10103A2EB030A08F10103BDF83F
:10199000A12082E7302A82D183F05003BDF8A12034
:1019A000ADF89D3008F10103D046A2EB030A76E7BB
:1019B000049B002B40F094800146BDF8AC00F6F784
:1019C000E1FA089B0A901B1AA34220DB0A9B1C44E5
:1019D00022F08EFB0028B4D0209828F0D3FE129875
:1019E00028F0D0FE09990D9829F0A2FDBDF85430D9
:1019F000ADF89D3026A817F089FBBBF80D3003F534
:101A00000073ABF80D30584663B0BDE8F08F079B0C
:101A10009C42DBDABDF8AC70069BDB1B4345D5DA94
:101A2000059B9845D2DA202DD0D93F49049AA5F1DB
:101A300021033E4DDBB20846D6B2B3422ED8C65C77
:101A4000002DC3D02301083B0E934FEA0813083B37
:101A50000F9373190C930C9AAA424FF00D03B5D053
:101A600015F8012BC82A23D83149DFF8C4C0895C96
:101A70001491304900205FFA80FE964513D3149AE2
:101A80000DF1DC0C01EB020E8E450CF1040C11D1B2
:101A900037AA149926A816F079FFDCE711F8016B34
:101AA00001323544C8E71CF801EB01307144E2E72C
:101AB0000021E4E711F8012BB2FBF3F003FB102245
:101AC000D2B212FB07F216460E9A023816440F9A4B
:101AD0002CF8046C10FB07F010442CF8020CD3E730
:101AE000049BB3F5005F27D1089B033BA34212DCA4
:101AF000079B9C420FDA069B053B43450BDC059B8D
:101B0000984508DA109B4246CDE9009321460346EA
:101B100026A817F033FE169B59E700BF9B3106003D
:101B20008D32060092320600E41B0600C31C06003C
:101B30001E1E0600E71E0600049BB3F5804F18D159
:101B4000089B053BA34212DC079B9C420FDA069BD5
:101B5000073B43450BDC059B984508DA109B424642
:101B6000CDE900932146034626A817F031FD179BC7
:101B70002DE7119B002BBFF62BAF099828F023FC13
:101B8000002857D0039BAB4200F39D8037AF002263
:101B90000999384623F010FB039B0026ED1ADDE976
:101BA00037239A4203D2399B1344AB423DDB3B9F20
:101BB00007B1BF5C3A9828F0E5FD089BDB1BA34208
:101BC00042DA079B9C423FDA069B0B9A9B1A4345DD
:101BD0003ADA059B984537DA92FBF9F3029A1393A8
:101BE00053435E43F2100D9937A823F0E5FA3B9D6D
:101BF00006F007060DB1379BED5C029B73439D40D9
:101C000004EB09030C9300230E930E9B9F4256DDB9
:101C10000C9BA3EB09031A930C9B013B199308EB54
:101C200009030A9300230F9335E0384623F073FA33
:101C30000644B4E7099829F013FD039BEE1AAB4262
:101C4000074600FB06F6B8DD07FB0944C0E61B9B10
:101C5000E9B21941109B03B991B1189B090226A85A
:101C6000B1FBF3F117F020F80A9B0A9A0190013BAF
:101C70000093A2EB0902199B1A9926A817F002FA01
:101C8000029B1E44072E11DC9D400F9B01330F93D6
:101C90000A9B4B440A930F9B139A9342D7DB0E9BEC
:101CA00001330E930C9B4B440C93AEE737A822F004
:101CB0008BFF3B9D0DB1379BED5C0026E5E73A9825
:101CC00028F060FDC0E70027BEE783469BE600BF23
:101CD00030B595B00546014603A817F03BFAD8B1D8
:101CE00028F01EF80446A0B10C4829F036FB014646
:101CF000204629F041FE0A4829F02FFB01462046E4
:101D000029F03AFE01220094064B1146284607F0BE
:101D100013FE204615B030BD0446FAE7A031060098
:101D2000AB310600291D030038B5054608460C46B0
:101D300029F098F8072824D901221249204628F0D2
:101D4000C1FEF0B11049204628F0C4FEC8B90F49C1
:101D5000204628F0BFFEA0B90D49204628F0BAFE63
:101D600078B96FF000420721204628F0A0FF044612
:101D70000146284629F0B4FD2046BDE8384028F049
:101D800001BD38BDBA310600C2310600D0310600AF
:101D9000DD3106002DE9F04792B004468A4601463F
:101DA00001A8914698461A9F17F0D4F9002859D0F7
:101DB000504628F008FB40B92B49012023F032FEA1
:101DC0000024204612B0BDE8F087B9F1FF0F01D919
:101DD0002649F2E7404628F0F6FA28B9404628F0AE
:101DE000B7FB08B92249E8E7C7F30726002E4FEAF8
:101DF000274308BF0126012B05DD022B2CD0042B25
:101E00002DD01C49D9E74FF4004552461A492046C7
:101E100029F050FE42461949204629F04BFEF8B2FF
:101E200027F0D6FE16490246204629F05AFE4846BB
:101E300027F0CEFE13490246204629F052FE3544D3
:101E400001A8ADF8185017F061F9B4F80D3003F59A
:101E50000073A4F80D30B4E74FF42045D5E74FF4F4
:101E60004045D2E70446ACE70B32060028320600B4
:101E7000453206006F3206009B3106008D320600A7
:101E8000B5310600923206002DE9F04F97B090462A
:101E90000191014605A81F4617F05CF9002856D0AD
:101EA000019828F090FA002879D00023092202A98D
:101EB00001988DF81030CDE902332AF0C5FA9DF86B
:101EC0000C609DF809009DF80A909DF80B70002E9B
:101ED00040D122F035FB2EF0A7FF0022C44B2FF09B
:101EE00037F9044648460D4622F02AFB2EF09CFFA7
:101EF0000022BF4B2FF02CF9824638468B4622F049
:101F00001FFB2EF091FFBA4B00222FF021F9002287
:101F100006460F460023204629462FF061FA88B96D
:101F200000220023504659462FF05AFA50B9002299
:101F30000023304639462FF053FA18B99DF80F3078
:101F4000002B3BD00120AB4923F06CFD002017B0E3
:101F5000BDE8F08F494622F008FB2EF065FFA2A3F2
:101F6000D3E900232FF0F4F804460D4638463146F5
:101F700022F0FBFA2EF058FF9BA3D3E900232FF0A9
:101F8000E7F882468B469DF80D009DF80E1022F072
:101F9000ECFA2EF049FF94A3D3E90023B5E70198AA
:101FA0002AF0C6FA404655EC104B2AF0C1FA3846E2
:101FB0005BEC10AB2AF0BCFA57EC106B25F0004933
:101FC0004FF0FF328C4B204649462FF031FA002863
:101FD00040F005814FF0FF32874B204649462FF0F5
:101FE0001DFA002840F0FB802BF000494FF0FF3233
:101FF000814B504649462FF01BFA002840F0EF80F5
:102000004FF0FF327C4B504649462FF007FA00282C
:1020100040F0E58027F000494FF0FF32764B304624
:1020200049462FF005FA002840F0D9804FF0FF32E2
:10203000714B304649462FF0F1F9002840F0CF802F
:1020400000226E4B204629462EF058FF2FF006FA4C
:1020500000226A4B0546594650462EF04FFF2FF09E
:10206000FDF900220446654B304639462EF046FF06
:102070002FF0F4F9BDF8191011F4607184F308021F
:1020800085F3080380F3080408D0B1F5C07F19D0A8
:1020900010D880291AD0B1F5807F1CD09DF81F1070
:1020A00010291FD1D8109210C00240EA421040EA15
:1020B000E4004CE7B1F5007F11D0B1F5207FEDD100
:1020C000114601E019461346224606E0194623460A
:1020D00014460A46E2E7194623460C46DEE719464F
:1020E0001346F6E7202906D1180440EA02202043CF
:1020F00040F07F402BE7182904D1180440EA022061
:10210000204324E704292AD10026DFF8F4C06FF029
:10211000004730463CF8021B0D124FEAE10EC900A1
:10212000C9B20EF0FC0E4EEA911E05F0F80545EA24
:102130005515AEEB020EED1A41EA51110EFB0EFEE3
:10214000091B05FB05E501FB0151B942B8BF30464B
:1021500006F10106B8BF0F46102EDBD1F7E60829BD
:102160002AD10026DFF89CC06FF0004730463CF8CB
:10217000021B0D124FEAE10EC900C9B20EF0FC0EAF
:102180004EEA911E05F0F80545EA5515AEEB020E34
:10219000ED1A41EA51110EFB0EFE091B05FB05E588
:1021A00001FB0151B942B8BF304606F10106B8BF84
:1021B0000F46FF2EDBD1CAE6032907D1D811D21171
:1021C000800040EA420040EAE410C0E613441819D7
:1021D000B0F5C07F4FF0FF30B8BF0020B7E60198E0
:1021E00029F03EFAB3E600BF0000000000E06F40B7
:1021F00000002E40AF320600FFFFEF7F000070406E
:10220000C22606000227060070B5044608460D46A1
:1022100027F08FFF002875D000223E49284629F07C
:102220008DFC064650B100231A4601462046FFF7B2
:102230002BFE394B1870304628F0A4FA002237499B
:10224000284629F07BFC064650B100231A46014679
:102250002046FFF719FE304B5870304628F092FAAE
:1022600000222F49284629F069FC064650B1002378
:102270001A4601462046FFF707FE274B9870304666
:1022800028F080FA00222749284629F057FC064604
:1022900050B100231A4601462046FFF7F5FD1E4BBC
:1022A000D870304628F06EFA00221F49284629F0DF
:1022B00045FC064650B100231A4601462046FFF76A
:1022C000E3FD154B1871304628F05CFA00221749DF
:1022D000284629F033FC064650B100231A46014631
:1022E0002046FFF7D1FD0C4B5871304628F04AFAD2
:1022F00000220F49284629F021FC18B129F09BFF44
:10230000054B9871B4F80D3003F50073A4F80D3047
:10231000204670BD97320600300403206635060063
:102320009A3206009E320600A2320600A63206004D
:10233000AA320600F0B593B004460E46014601A845
:1023400015461F4616F006FFF0B1AFB9049B2A46AA
:10235000314601A816F0CAFE01A8ADF81A60ADF822
:102360001C5016F0D3FEB4F80D3003F50073A4F83A
:102370000D30204613B0F0BD00231A4639462046E2
:10238000FFF782FD0346E2E70446F2E72DE9F04F4E
:102390009DB00BAD80460F460146284616461C46AA
:1023A00016F0D8FE0290002800F09B80269B0A932E
:1023B00008AA07A92846CDE90776099416F01BFD5F
:1023C0000AAA09A9284616F016FD0798099B08993C
:1023D0000A9CC21802EBD27252101B1A009203EB35
:1023E000D3730A19641A5B1004EBD4746410059358
:1023F0005B43039302EBD27204FB04F35210049389
:102400000192DDE903326600013E03FB1626002738
:10241000009B03EB070B019B03EB040A52460E9B48
:102420005946284616F0AFFB009BA3EB070952461E
:102430000E9B4946284616F0A6FB019BA3EB040A17
:1024400052460E9B5946284616F09DFB28460E9B89
:102450005246494616F097FB049A7B0003FB022282
:1024600071009142BFBF049A0298033302FB0366D6
:102470004FEA440C039BCCF1010203FB02F2B4BF10
:1024800001370020914208DD039AACF10303013CBF
:1024900002FB1366002CBBDA01E00028FAD1059B91
:1024A000BB4207F101040CDC284616F02FFEB8F8F9
:1024B0000D3003F50073A8F80D3040461DB0BDE89F
:1024C000F08FDDE900120E9B2144284616F05BFBDD
:1024D000DDE900120E9B091B284616F054FB274627
:1024E000DDE7DDF80880E8E713B51C4613440093E8
:1024F000121B0B19091BFFF749FF02B010BD2DE994
:10250000F04F9FB00DF1340A80460E46014650460A
:1025100015461C4616F01EFE0390002800F0898028
:10252000289B0C930AAA09A95046CDE909650B948A
:1025300016F061FC0CAA0BA9504616F05CFC099938
:102540000B9B0C9CCDF818A0CA1802EBD27252104B
:1025500002920A9A1519A41A5B1A04EBD474641037
:1025600003EBD3735B10660005EBD575059304FB95
:1025700004F95B43013E6D10049303FB169600279C
:102580007B0003FB099271009142BCBF033309FB3E
:1025900003660498B8BF039A4FEA44030793C3F154
:1025A000010300FB03F3B4BF0137002299421FDD92
:1025B000029B069803EB070AA3EB070B109B2A1953
:1025C000CDE9002351465B4616F090F9109B069822
:1025D0002A1BCDE9002351465B4616F087F9079B7D
:1025E000049A033B013C02FB1366002CC8DA01E0AD
:1025F000002AFAD1059BBB4207F101040CDC0DA8AF
:1026000016F084FDB8F80D3003F50073A8F80D300E
:1026100040461FB0BDE8F08F109B0299CDE90053F2
:10262000029B2A461B1B21440DA816F05FF9274682
:10263000E0E7DDF80C80EBE713B51C46134400938C
:10264000121B0B19091BFFF75AFF02B010BD00EB5C
:1026500081010023884200D3704751F8042D43EADA
:1026600052030B60D307F5E710B5013A52B21306D7
:1026700001D5002010BD50F8224051F822309C4274
:1026800005D802F1FF32F2D24FF0FF30F2E701201D
:10269000F0E710B500235CB2A24200DC10BD51F897
:1026A000234040F823400133F5E7013910B549B222
:1026B000041D0A06CBB204D4013954F82120002AA3
:1026C000F7D001335BB273B103F18042013A50F8A5
:1026D0002220002022B9013B00EB431318B210BDA9
:1026E00052080130F6E71846F9E710B500231A46FC
:1026F0005CB2A14203DCB2FA82F0400910BD50F88E
:10270000234001332243F3E7002310B51C465AB29D
:10271000914200DC10BD40F823400133F7E7000090
:10272000C3F10803DB0070B50133002403A500BF2B
:102730005B1920C940CAAD1B20C0184720C940CA38
:10274000B54120C020C940CAB54120C020C940CAF7
:10275000B54120C020C940CAB54120C020C940CAE7
:10276000B54120C020C940CAB54120C020C940CAD7
:10277000B54120C06441B4FA84F0400970BD00BF87
:10278000C3F10803DB0070B50133002403A500BFCB
:102790005B1920C940CAAD1920C0184720C940CADA
:1027A000754120C020C940CA754120C020C940CA17
:1027B000754120C020C940CA754120C020C940CA07
:1027C000754120C020C940CA754120C020C940CAF7
:1027D000754120C06441204670BD00BF70B59DF9B1
:1027E00010401E4623460546FFF79AFF38B12346A0
:1027F000324629462846BDE87040FFF7C1BF70BD8C
:1028000070B59DF910401E4623460546FFF7B8FFF8
:1028100030B9224629463046FFF726FF012807D067
:102820002346324629462846BDE87040FFF778BF68
:1028300070BD000007B5154B1A687AB100221A6006
:102840001B680093009B4FF080430122C3F80823CC
:102850000F4B587910B95A711B6898470D4B1A687D
:1028600082B100221A601B680193019B4FF08043E4
:102870000222C3F80823064B1B68012003B05DF851
:1028800004EB184703B05DF804FB00BF00010040F3
:102890009804032004010040074B00221A6082B014
:1028A0001B680193019B054BD3F80805044B1B687B
:1028B000C0B202B0184700BF00D1004000D00040B5
:1028C000DC010320064B00221A6082B01B680193D2
:1028D000019B044B0122C3F804231A6002B0704725
:1028E00000D1004000D000402DE9F74FDFF8EC8028
:1028F00007468946B9F1000F03D1012003B0BDE8B6
:10290000F08F4D46402D28BF40255FFA85FB0024FF
:1029100000230DF106008DF80630F5F7EFFA2D4B88
:1029200093F800A0BAF1000F2ED10DF107008DF839
:1029300007A0F5F7E3FAD8F80030D8F8042093425E
:1029400088BF4132D31A9D4242D8D8F80040D8F807
:102950000460214BB44294BF361BC4F14106B5421A
:1029600004EB030128D82C442A4638462EF0DAFF1F
:10297000412C28BF0024C8F8004000249DF807001F
:10298000F6F74AFBFFF79EFF9DF80600F6F744FBBB
:10299000BAF1000F08D059463846FAF749F942F221
:1029A000070398420446B0D0022CB1D0002CACD121
:1029B000A9EB05092F449DE7324638462EF0B2FFB9
:1029C000054BAC1B22461946B8192EF0ABFFD2E7D7
:1029D0000524D3E789FC022070010320B401032001
:1029E00000F1804000F5E040002382B003600368FE
:1029F0000193019B02B07047F0B5534B534C1B68D9
:102A000085B0002B3DD04FF4827094F82E20FFF754
:102A1000E7FF2AB394F82F3013BB4D4B1B68002BF4
:102A200033D04FF48070FFF7DBFF94F82D20638BD9
:102A300091B28B424ED95B1A21899BB26383CB1A28
:102A4000616801EB4301434BC3F82C16C3F83026F1
:102A50004FF48270FFF7C4FF3F4B01221A6014E06D
:102A6000636802932389ADF80C30E36800218DF888
:102A7000041023BB2374236801A89847002384F81B
:102A80002F3094F82E30002BC7D1344B1B685BB12C
:102A90004FF48870FFF7A4FF0023237402238DF8FE
:102AA000043001A8236898472D4B1B6813B34FF4DB
:102AB0008A70FFF795FF0023237405B0F0BD208BCB
:102AC000608363602081E160002AD4D1214B012220
:102AD0001A60D0E7BCD1E368012184F82F103BB124
:102AE000002161831B49C1F82C36C1F83026AFE7BD
:102AF0006383ADE766694FF000470125002EDCD007
:102B0000B6FA86F227FA02F34632920026EA030664
:102B100002F1804303F5E0431B68002BEED0104622
:102B2000FFF75EFFA2F58C72D30882F00402C2F3B5
:102B300080028DF808308DF804508DF80920236844
:102B400001A89847DAE700BF04710040540403204D
:102B5000007100400070004004700040107100409F
:102B600014710040F0B5394B394C1A6885B07AB110
:102B700000221A601B680093009B637943F00803EE
:102B800003F01202122A637104BF43F02003637141
:102B9000304B1A687AB100221A601B680193019BBE
:102BA000637943F0040303F01102112A637104BF37
:102BB00043F020036371284B1A68B2B100251D60F1
:102BC0001B680293029B254B25480422C3F8082367
:102BD000C3F80055236829469847236821482946A9
:102BE00098470123237105B0F0BD637903F00F020C
:102BF0000F2A08D0D80701D4190704D462799207A4
:102C0000F1D45B07EFD56379266803F0F30313F083
:102C1000200708D023F0300343F010036371012133
:102C20000020B047DFE70E4A92E8030002AD85E8D6
:102C3000030012E9030043F0100382E80300C4E933
:102C40000277637101212846EBE700BF145102406F
:102C50003C0403200451024008510240005002404D
:102C60004C04032044040320B0DF7047F0B5154640
:102C70008BB004460F466A46A988D0F878011E46F4
:102C8000F9F7FCFE10B1636803B19847009A32B3BC
:102C90000021CDE901110121EB898DF80410BDF867
:102CA0004010ADF80C30C91A1E44ADF80E10324475
:102CB000012301A9A88804928DF80A30FFF7D4FFF8
:102CC00010B1636803B19847236843B13868069030
:102CD00007228DF81420099505A9204698470BB0C6
:102CE000F0BDF0B50388502B8BB005460C4656D08E
:102CF000512B00F00281102B6FD100238188D4F872
:102D00007801049304AAF9F7B9FE10B1636803B11E
:102D100098470498002860D0D4F87C1199B3A67C19
:102D200000231322B34229D3D4F8801121B194F89F
:102D300078600023B34228D3D4F8841121B194F8E9
:102D4000DE600023B34225D30021F3F7EBFA638959
:102D5000002B42D0049A012313700022ADF81620F4
:102D6000ADF8143005AA049B6189A8880693FAF788
:102D7000AEFF90B3636883B398472EE031F83370A9
:102D800001333A44CEE71322CEE731F833700133F2
:102D90003A44CFE731F8337001333A44D2E7C1887F
:102DA000B4F86E01022300228842ADF80C30ADF871
:102DB0000E201FD104AAA988D4F87801F9F75EFE85
:102DC00010B1636803B19847049A32B12B8A012B82
:102DD00003D1AB7C1BB1012B01D00BB0F0BD8DF842
:102DE000143053702368002BF7D0099505A92046AD
:102DF0009847F2E7608988421AD104AAA988D4F8D2
:102E00007801F9F73BFE10B1636803B19847049A63
:102E1000002AE2D02B8A012BDFD1AB7C1BB1012B26
:102E2000DBD1062100E005218DF814101370D9E7DD
:102E3000B4F85201884208D142F6222305932A466B
:102E400005A92046FAF72BFFC7E7B4F84E018842E0
:102E500004D142F62222059208220AE0B4F8563143
:102E60008B420FD142F6322305930A23ADF80C3082
:102E70000122ADF80E20009205AA29462046FAF755
:102E8000E7FFAAE7B4F862318B4202D142F633235E
:102E9000D4E7B4F85E318B4217D0A07C134604F11E
:102EA0000E060A27DAB2904216D80DF10E030093EF
:102EB00005AA03AB2046FAF777FE00288DD0BDF8AF
:102EC0000E300093BDF80C30D6E742F6332305935D
:102ED0000B23ADF80C30BFE7013307FB03FC36F8DA
:102EE0000CC08C45DED142F64D23ADF814300123E1
:102EF0008DF816308DF81720A1E70022ADF80E20CE
:102F000082790223012AADF80C307FF466AF018983
:102F10006089884220D104AAA988D4F87801F9F7F9
:102F2000ADFD10B1636803B19847049B002B3FF4DB
:102F300054AFE989ADF81C100022CDE9052205A99E
:102F40000122A8888DF81420ADF81E2008938DF872
:102F50001A20FFF789FE0CE7B4F84E01884204D12D
:102F600042F622220592082209E0B4F856318B423B
:102F70000ED142F6322305930A23ADF80C30ADF89A
:102F80000E2000922A4605A92046FFF76FFE24E78F
:102F9000B4F85E318B4206D142F6332305930B23FE
:102FA000ADF80C30DFE70DF10E03009305AA03AB7B
:102FB0002046FAF7F9FD00283FF40FAFBDF80E30B8
:102FC0000093BDF80C30DDE7ABDF7047A9DF704739
:102FD000BFF34F8F0549064BCA6802F4E062134302
:102FE000CB60BFF34F8F00BFFDE700BF00ED00E0F7
:102FF0000400FA0508B54FF080430022C3F80C2105
:10300000C3F81021C3F838254FF0805203F5404330
:10301000D2F80414C3F82015D2F80814C3F8241504
:10302000D2F80C14C3F82815D2F81014C3F82C15D4
:10303000D2F81414C3F83015D2F81814C3F83415A4
:10304000D2F81C14C3F84015D2F82014C3F8441564
:10305000D2F82414C3F84815D2F82814C3F84C1534
:10306000D2F82C14C3F85015D2F83014C3F8541504
:10307000D2F83414C3F86015D2F83814C3F86415C4
:10308000D2F83C14C3F86815D2F84014C3F86C1594
:10309000D2F84424C3F87025FAF71CFE10B12E4B69
:1030A0002E4A1A60FAF716FE18B12D4BFB22C3F810
:1030B0001825FAF70FFE48B12A492B4B0A681B68FE
:1030C00022F00F0203F00F0313430B60FAF702FE26
:1030D00018B1264B4FF400721A604FF08043D3F8BA
:1030E0000024D20744BF6FF00102C3F80024204A35
:1030F000D2F8883043F47003C2F88830BFF34F8FA2
:10310000BFF36F8F4FF01023D3F80C32DB071ED5BF
:10311000184B0122C3F80425D3F80024002AFBD061
:103120004FF01022D2F80C3223F00103C2F80C3217
:10313000104B1A46D3F800140029FBD00021C3F825
:103140000415D2F80034002BFBD0FFF741FF0A4BE7
:103150000A4A1A6008BD00BF8C560040488103002F
:1031600000F00040E40E004058020010409602407B
:1031700000ED00E000E00140343200200090D00378
:10318000024B03495868002228F0D8BC983400202C
:103190002C2A060070B5174B1C7884420DD0FCF722
:1031A000BDFA05462046FCF7B9FA2A4603461249FD
:1031B0000420BDE8704022F035BC104C002018708F
:1031C000206840B189B1114603F048FC206827F01F
:1031D000D9FA002323600A4C206827F0D3FA002391
:1031E0002360084B01221A7070BD114603F07EFD6A
:1031F000ECE700BF28040320FB290600200403207D
:103200002C0403203704032010B50A460C46002185
:10321000FFF7C0FF2046BDE8104027F0B3BA00001A
:1032200038B5194D2A884FF6FF719142044613D0E4
:1032300001460320FCF78CFA18B1144B186826F0ED
:1032400019FC044613212888F9F7C4F940F66B41AC
:103250000FF0F2FD204638BD0D4B1D78022D0DD12B
:103260000C4828F07AF801462846FFF7CDFFFAF718
:1032700041FD2046BDE8384006F0D2B8064901209D
:1032800022F0D0FBF5E700BF3A32002020040320F3
:1032900028040320782A06008D2A060010B5094B61
:1032A0001C78012C0CD100210846FBF757F8064882
:1032B00028F053F801462046BDE81040FFF7A4BFB0
:1032C00010BD00BF28040320EB2C06000A46002195
:1032D000FFF760BFF7B500223449044628F02EFC02
:1032E00028F0B4FE324B334906460322586828F0D2
:1032F00025FC054630B12246B1B228F06DFB2846C8
:1033000027F040FA00222C49204628F017FC0746F7
:10331000002839D121460820FCF71AFA18B90025EF
:10332000284603B0F0BD254B254E186826F0A2FBB9
:1033300033884FF6FF729A42054607D1214828F09C
:103340000CF801460820FFF75FFFE9E73A46174906
:10335000204628F0F3FB28F079FE013080B2ADF86A
:103360000400ADF8060001A93088F5F7E7F813F07E
:103370003DFF04460028D3D001460820FFF7A6FFF2
:10338000204627F0FFF9CBE727F0FCF900210920C0
:10339000FCF7DEF90028C2D0084B186826F06AFB5B
:1033A0000121054620460FF0DFFBB9E7B22A0600EF
:1033B00098340020BF2A0600A62A06002004032015
:1033C0003A3200208D2A060070B5014606460720D5
:1033D000FCF7BEF968B3184B184D186826F04AFB85
:1033E0002B884FF6FF729A42044608D1144827F002
:1033F000B4FF01460720FFF707FF204670BD0022FB
:103400001049304628F09AFB28F020FE2B8881B224
:1034100000221846F5F7AEFA13F0E8FE054600283C
:10342000EBD001460720FFF751FF284627F0AAF905
:10343000E3E70446E1E700BF200403203A3200201E
:103440008D2A0600B22A06002DE9F04F85B00D4600
:1034500000AF00238046394628463B6027F04AFDEE
:103460000446002D39D0F8B9284625F0EBFC064675
:10347000386020F045FE06F58073834209D937494C
:10348000012022F0CFFA002630461437BD46BDE8B1
:10349000F08FF31D23F00703ADEB030D6C463246AE
:1034A0002146284625F0F6FD00210620FCF750F9BC
:1034B0000028E8D02A4B2B4D186826F0DBFA2B8821
:1034C0004FF6FF729A4206460AD1274827F045FF79
:1034D00001460620FFF798FED6E70028E4D1D2E7A0
:1034E00000222249D7F80090404628F027FB28F018
:1034F000ADFD00221FFA80FA1D49404628F01EFB50
:10350000834640B300221B4928F018FB28F093FEA5
:103510008046584627F036F9002398453B8114BF72
:10352000022301233B71391D012328887B71FC6034
:10353000A7F806A0A7F80A90F5F71AFA13F056FEB6
:1035400004460028A0D001460620FFF7BFFE204613
:1035500027F018F998E78046DEE700BF522F0600F3
:10356000200403203A3200208D2A0600B22A0600E9
:10357000C62A0600D12A060038B50D4601460A20A3
:10358000FCF7E6F820B3134B186826F073FA124BD9
:103590001A884FF6FF719142044608D10F4827F070
:1035A000DCFE01460A20FFF72FFE204638BD2946E3
:1035B0001888F8F791FB13F019FE05460028F4D09F
:1035C00001460A20FFF782FE284627F0DBF8ECE7E9
:1035D0000446EAE7200403203A3200208D2A060040
:1035E000F0B58DB06D460C46294614F0DBFA002884
:1035F00000F0888095E80300ADF80C10090C0290EB
:103600008DF80E100E22002108A8F2F78BFE04237D
:103610008DF82030A023ADF822303D4B09933D4B6F
:103620003D4958680022CDE9062228F087FA28F0A3
:103630000DFDC3074CBF394B394B069320464FF065
:10364000C873079326F075FD002841D00022354944
:10365000204628F073FA28F0DDFF02460B460646A6
:103660000F462DF0E5FE90B900222F4B304639462B
:103670002DF044FC24A3D3E900232DF069FD0022A2
:103680002A4B2DF085FA2DF011FFADF8180000221D
:103690002749204628F052FA28F0BCFF02460B4684
:1036A00004460D462DF0C4FE90B900221E4B204664
:1036B00029462DF023FC14A3D3E900232DF048FD67
:1036C00000221A4B2DF064FA2DF0F0FEADF81A002E
:1036D00002AB93E80300ADF81410090C04908DF8C8
:1036E0001610012306AA08A904A813F0E7FD13F099
:1036F0007DFD044630B101460220FFF7E7FD20467C
:1037000027F040F80DB0F0BD0000000000889340A5
:103710009000040098340020482E060090012003F9
:103720001000A000302E060000408F400000E03F57
:103730003C2E06000A460121FFF72CBD70B50D4B4B
:103740001C78012C054613D100210846FAF706FE25
:103750002146094828F02DF9064607F0E9FE3046D3
:1037600027F010F829462046BDE87040FFF7E2BF79
:1037700070BD00BF280403202C0403207CDF7047A9
:103780002DE9F04F964C85B0236800AF054603F055
:10379000040308460E463B6026F0CBFC002800F0F0
:1037A000AB8000228F49304628F0C8F9B0B128F02C
:1037B0004DFC4FF47A73584340F2712390FBF3F0C1
:1037C00080B2B0F5804F884B28BF4FF4804020284E
:1037D0001A8838BF2020824218BF188000228349EF
:1037E000304628F0ABF938B128F025FD23680028D1
:1037F00062D023F40063236000227D49304628F024
:103800009DF938B128F017FD2368002857D023F41C
:103810008053236000227749304628F08FF9814693
:10382000002873D0002307F10C01FB6027F062FB36
:103830008046002852D1484625F004FB8246F860B5
:1038400020F05EFC0AF5807383423BD96A4901206F
:1038500022F0E8F8484626F095FF284626F069FC55
:10386000814608B9002D54D131462846FBF772FC39
:10387000002D40F0B2800025604C614960682A4606
:1038800028F070FC32465F49606828F06BFC2846DF
:1038900026F078FF3B680BB10FF0BCFA4FF45B7178
:1038A00040460FF0C9FA3B6863B30FF005FF40F2E2
:1038B0006E310FF0C1FA25E043F400639BE743F457
:1038C0008053A6E70AF1070323F00703ADEB030DCE
:1038D000E84652464146484625F0DCFB1123414666
:1038E000BA893B7207F10800FFF748FF40F22D311B
:1038F00080460FF0A1FAADE746B1324642490320B7
:1039000022F090F81437BD46BDE8F08F4FF0000864
:10391000A3E7284626F004FC786000284BD0B5F8D1
:103920000D3003F50073A5F80D30236823F07F7385
:1039300023F40033294607F10C00236021F02DF811
:10394000CB46F86850B9B9F1000F95D0BBF1010F23
:1039500092DD236843F4003323608DE727F06AFE8D
:10396000824626F0E6FB10B9BAF1000F0FD13146BE
:103970005046FBF7EFFB8146F86810B1494627F047
:103980002DFD484626F0FEFED7F8049009E050468B
:1039900026F0C6FB0028F7D1504626F0A4FB0028ED
:1039A000F2D1504626F0EEFE07F10C000BF1010BB0
:1039B00020F0E7FFC5E7284626F095FB00283FF4F6
:1039C0005AAFB5F80D3003F50073A5F80D30236834
:1039D00023F07F7323F40033BEE705464CE700BFB6
:1039E00024040320BF63060038320020012E0600A5
:1039F0000D2E0600502B0600522F06009834002092
:103A0000172E0600212E06006C2C060070B5294CDE
:103A100029492068002228F091F8054618B10021B4
:103A200001200FF0C5F9284626F0ACFE00222349FC
:103A3000206828F083F8054610B101200FF08EF9B8
:103A4000284626F09FFE00221D49606828F076F87F
:103A5000002205461B49606828F070F801460646BA
:103A60002846FFF78DFE2846314627F061FD0022EB
:103A70001549606828F062F8054611F011FB2846E8
:103A800026F080FE60681149002228F057F80446AD
:103A900008B1FBF705FB204626F074FE10F024F871
:103AA0000B4B1B689B0503D5BDE87040FBF79CBC26
:103AB00070BD00BF98340020AB2E06009B2A060084
:103AC000172E0600212E060009300600B62E06002D
:103AD0002404032010B5044615F018FB034B20689E
:103AE00001221A70BDE8104026F04CBEE404032009
:103AF00038B5054600F01EFB044650B10146284685
:103B000015F028FB054610B9204626F03BFE284656
:103B100038BD0546FBE7000030B50F4C227893B066
:103B2000BAB101A8FFF7E4FF98B100220B49019850
:103B300028F004F8054638B1002301991A461DF013
:103B4000D1FE294627F0F4FC019826F01BFE002345
:103B50002370002013B030BDE40403204633060078
:103B600010B5104A137892B0013B01A81370FFF70B
:103B7000BFFFA0B10C4B059C5B7805936FF007026B
:103B8000002101A815F055F901A80594FFF7A2FF3F
:103B9000064B5B68C3F308030BB9FFF7BDFF12B018
:103BA00010BD00BFCC3300203004032000ED00E046
:103BB000034B00221A705A709A70DA70704700BF77
:103BC000E004032070B592B004460D46014601A8FA
:103BD000164615F0BFFA60B33EB140F2FF339D4286
:103BE000A8BF1D46012DB8BF0125BDF91830002B17
:103BF00011DA2B040FD41049204628F0A2FA0F49FD
:103C0000204628F09EFA0E49204628F09AFA0D49DF
:103C1000204628F096FA01A8ADF8185015F076FA6B
:103C2000B4F80D3003F50073A4F80D30204612B03F
:103C300070BD0446FAE700BF9B3106008D320600D6
:103C4000B5310600923206002DE9F84F07460846C6
:103C50000C46154626F0B7FB002800F08F800122A5
:103C60004749204626F02EFF804600283FD02046B8
:103C700027F0F8F8062894BF4FF0FF3606263A21C1
:103C8000204626F0ADFF002834DB461C31466FF09D
:103C90000042204627F00BF828F0D8F9012EB8BFD3
:103CA00001260546721E2046002127F000F8044632
:103CB00041F6FF739D42A8BF1D46012DB8BF0125E7
:103CC000B8F1000F1FD0AEB22E49204626F002FFF9
:103CD000834658B305F58045AEB2204626F052FD26
:103CE000424631463846BDE8F84FFFF76BBF4FF00C
:103CF000FF36C4E7731CC9D1B4F80D3003F5007367
:103D0000A4F80D30D4E71CB905F50056B6B2DBE7D0
:103D1000204627F0A7F80028F6D01B49204626F0B9
:103D2000D9FE0028F0D14FF6FF76CDE74FF6FF73AE
:103D30009E42D2D12146154826F0CAFF5A46014676
:103D40008146384621F06EFF824648B15B465A46AE
:103D500039461DF0C7FD26F015FDA5F50045AEB2AC
:103D60004946504627F0E4FB4FF6FF739E42B4D11C
:103D700022460749012021F055FEAEE7BDE8F88F45
:103D8000A4310600AB310600A0310600F131060077
:103D9000FB31060001381F289DBF034B23FA00F0BA
:103DA00000F00100002070478B80808030B551EC1E
:103DB000100B85B053EC112B8DED000B55EC124B15
:103DC0008DED021B2DF00CFB9DED000B28B19DED40
:103DD000021BB0EE410AF0EE610A53EC102B2046B4
:103DE00029468DED000B2DF0FBFA9DED000B08B17F
:103DF00045EC104B05B030BD38B555EC104B0022EA
:103E0000002310EE100A29462DF0EAFA10B105F150
:103E100000431D4645EC104B38BD10B413460A460E
:103E200053F8044B0021A4465DF8044B60472DE98C
:103E3000F84388469146054618B1077A0024A74200
:103E400001D8BDE8F8832B68686833F8343018442B
:103E500027F083FA014606464846C047304626F01A
:103E600091FC0134EBE728F097B9000000220149EA
:103E700021F05EBFA2380600F0B595B004460D46AD
:103E8000014603A816461F4615F064F998B11A9B1F
:103E9000009332463B46294603A815F0BEF803A816
:103EA00015F034F9B4F80D3003F50073A4F80D30B3
:103EB000204615B0F0BD0446FAE700B593B00146C0
:103EC00001A815F047F908B19DF80F0013B05DF88F
:103ED00004FBF0B595B004460D46014603A816460E
:103EE0001F4615F037F9A8B1079B01931A9B009361
:103EF00032463B46294603A815F0C4F803A815F03E
:103F000005F9B4F80D3003F50073A4F80D30204620
:103F100015B0F0BD0446FAE7F0B595B004460D467D
:103F2000014603A816461F4615F014F9A8B1069BD2
:103F300001931A9B009332463B46294603A815F08D
:103F4000A1F803A815F0E2F8B4F80D3003F50073FA
:103F5000A4F80D30204615B0F0BD0446FAE710B5C0
:103F600092B00446014601A815F0F4F858B101A832
:103F700015F0FAFA01A815F0C9F8002242F2010181
:103F80002046FFF71FFE12B010BD10B5044692B0D8
:103F900019B1FFF7E4FF26F0F5FB214601A815F063
:103FA000D9F870B101A814F0DDFD01A815F0AEF844
:103FB000B4F80D3003F50073A4F80D30204612B0AC
:103FC00010BD0446FAE7000010B5044630B90246B9
:103FD0000649032021F026FD204610BDB0F80D3023
:103FE00003F50073A0F80D30F6E700BF253A060090
:103FF0002DE9F04792B0804626F0E5F9044638B93D
:104000004849032021F00EFD204612B0BDE8F0879C
:1040100000224146684621F0CFF800273D463E4643
:104020003C464FF00009DDE900329A4225D803985A
:1040300026F0A8FB25F077FE04460028E4D03046A1
:1040400025F0C6FD38490246204627F04AFD28469D
:1040500025F0BEFD35490246204627F042FD05FB0E
:1040600006F007300021C01027F028F90546C0B936
:10407000204626F087FB2C46C6E7684621F04BF821
:104080000A2805D159EA040308BF01270134C8E70B
:10409000AC4209F10109A8BF651C4E45B8BF4E46A8
:1040A000C1E73A464146684621F086F84FF00008DD
:1040B00047464FF08009DDE900239A4208D3039870
:1040C00026F060FB2A461A49204627F00AFD9BE7A6
:1040D000684621F020F80A2803D108F101080027DA
:1040E000E9E720281CD0284626F06DF9C0B106FB70
:1040F000087A29464FEADA0209A821F05DF80D99FD
:1041000009B1099BC95C0AF0070A49FA0AFA41EAAF
:104110000A0109A8C9B220F099FC0C9826F032FBDC
:104120000137C8E7FD350600F8300600FE3006000E
:10413000D0420600024B03495868002227F0FEBC1B
:1041400098340020A26C060070B500228AB00E469A
:10415000114927F0F3FC054626F035F9044660B115
:104160000022294601A821F027F80024DDE90123D7
:104170009A4208D3049826F005FB284626F002FB55
:1041800020460AB070BD01A820F0C5FFB04208BFAC
:1041900044F00104E4B2E9E7DB3C060070B50446F4
:1041A00025F0C7FF30B900242546204626F0EAFA5C
:1041B000284670BD00221449204627F0BFFC054662
:1041C00025F0B7FF044618B9284626F0DBFAEBE7DE
:1041D000002DE8D000220D49284627F0AFFC044608
:1041E00025F0C2FF50B1284626F0CCFA002CDBD0D7
:1041F000074D2368EB1A5D425D41D6E7294620460C
:1042000027F096F9CFE700BFA2380600DF45060089
:1042100085930300014900201EF0EEBF52360600D0
:10422000014900201EF0E8BFCA3D060001490020F8
:104230001EF0E2BFE13C06002DE9F04790461D4626
:10424000421E47F6FE739A4292B08246894602D8D1
:104250004A1E9A4208D93F49012021F0E3FB00247D
:10426000204612B0BDE8F0874046FFF793FD0446B4
:1042700020B93949012021F0D5FBF1E7284625F086
:1042800058FFD8B100223549284627F057FC0022B4
:1042900004463349284627F051FC25460646284661
:1042A00025F062FF044688B92A462E49012021F0F4
:1042B000B9FB3146284627F03BF9D1E7B5F80D3078
:1042C00003F50073A5F80D300646E8E736B1304631
:1042D00025F04AFF044608B93246E6E722490020A5
:1042E0001EF08AFF04460028BAD00027012301A847
:1042F0008DF808308DF809708DF80A70ADF80BA0B4
:10430000ADF80D908DF80F8015F02EF96FF07F034A
:104310004FF0FF328DF82C308DF82E308DF827209D
:104320007F238DF8292011498DF828302A46204610
:104330008DF82A308DF82B708DF82D70019427F0B0
:10434000B9FB32460A49019827F0B4FB01A814F0E2
:10435000DDFEAEE78A35060097350600A335060078
:10436000AC350600B535060002290600E935060021
:10437000F335060070B506460D4626F024F80446CF
:1043800030B932461349032021F04CFB204670BD62
:10439000114900201EF030FF32461049044627F034
:1043A00089FB45B1284626F00EF868B9324609491E
:1043B000032021F037FB002025F00AFC08490246C3
:1043C000204627F08EFBE1E72A460649204627F0E3
:1043D00071FBF0E7983C0600C33C0600CA3C0600AF
:1043E000D13C0600DB3C060038B5002208490546F2
:1043F00027F0A4FB044640B906491EF0FDFE04491F
:1044000004460246284627F055FB204638BD00BF2B
:1044100014C006008B3C06002DE9F04317461E46EB
:10442000421E47F6FE739A4293B08146884602D8F0
:104430004A1E9A4205D97549012021F0F3FA002459
:1044400008E03846FFF7A6FC044638B97049012059
:1044500021F0E8FA204613B0BDE8F0836D49002052
:104460001EF0CAFE04460028F4D0002501A88DF8ED
:1044700008508DF809508DF80A50ADF80B90ADF842
:104480000D808DF80F7015F06FF86FF07F034FF00F
:10449000FF328DF82C308DF82E3030467F238DF88A
:1044A0002B508DF82D508DF827208DF828308DF861
:1044B00029208DF82A308DF809508DF80A50019482
:1044C00025F037FE00285CD02A465349304627F0B5
:1044D00035FB27F0B0FE28B1BDF8093043F00103E9
:1044E000ADF8093000224D49304627F027FB27F070
:1044F000A2FE28B1BDF8093043F00403ADF809303D
:1045000000224749304627F019FB27F094FE28B1D6
:10451000BDF8093043F00803ADF8093000224149E5
:10452000304627F00BFB27F086FE88B19DF80F0080
:1045300001280BD1BDF8093043F00203ADF8093072
:10454000BDF80D305B0703D0374976E7374973E78D
:1045500000223749304627F0F1FA054688B135493F
:1045600026F0B8FA50B93449284626F0B3FA08BB09
:10457000BDF8093043F08003ADF80930284626F035
:1045800001F9BDF80D00BDF80B3043439DF80F0055
:1045900058430730C00808F01FFC284A054601466A
:1045A000019827F0E8FA294626F0C2FF01A814F086
:1045B000ADFD4FE72249284626F08CFA20B9BDF818
:1045C000093043F48073D7E71E49284626F082FA63
:1045D00020B9BDF8093043F4C073CDE71A49284625
:1045E00026F078FA20B9BDF8093043F40073C3E728
:1045F0001649284626F06EFA20B9BDF8093043F472
:104600002073B9E7124821F0BBF8B7E78A350600F6
:104610009735060002290600B7340600BE340600AE
:10462000C2340600CE3406000C350600DC34060029
:10463000453506005135060055350600D0420600C6
:10464000593506005D350600613506006535060002
:10465000693506000000000008B500222DED028B30
:10466000B0EE408AF0EE608A002351EC100B2CF083
:10467000CBFE98B1B0EE480AF0EE680A2AF060FB73
:104680000B4B51EC100B00222CF038FCBDEC028BD4
:1046900041EC100BBDE808402AF0CEBABDEC028B0D
:1046A0009FED010B08BD00BF000000000000F87F77
:1046B0000000E03F00000000F8B555EC104B25F07D
:1046C00000474FF0FF32284B204639462CF0B0FE11
:1046D00060B94FF0FF32244B204639462CF09EFE45
:1046E00020B9B5F1004F08BF002C05D145EC104BA7
:1046F000BDE8F84025F05ABA00220023204629469A
:104700002CF06EFEC8B912A1D1E900012B46224659
:104710002CF03EFA06460F462CF050FF04460D469C
:1047200054EA05030DD100220023304639462CF00F
:1047300057FE30B19FED080BDAE709A1D1E900017E
:10474000E4E720462946BDE8F84025F0FCBA00BF62
:104750002083E4FFFFFFDF3F000000000000008037
:104760002083E4FFFFFFDFBFFFFFEF7F2AF060BA87
:1047700029F0E2BE38B555EC104B10EE102A2B464E
:1047800010EE100A29462CF0B9FB02460B46002019
:1047900009492CF0FBF941EC100BFFF75DFF2046B7
:1047A00053EC102B29462CF0D3FCBDE8384041ECEB
:1047B000100B29F0C1BE00BF0000F03F2AF0D8B9AD
:1047C00030B599B0054625F02BFE044638B92A4687
:1047D0001F49032021F026F9204619B030BD0122DF
:1047E000294609A824F0E2F900231A4609A9194824
:1047F00015F072F8044609A820F065F8204600215B
:1048000026F05CFD044618B9134820F0D9FFE3E711
:104810002946012209A824F0C9F921460022684648
:1048200020F0CAFC6B460D4A0A4809A915F054F855
:10483000039825F0A7FF09A820F045F8002120469D
:1048400026F095FB0546204625F09CFF2C46C3E745
:1048500010360600FF700400353606002171040092
:1048600030B599B0054625F0DBFD044638B92A4637
:104870001F49032021F0D6F8204619B030BD01228F
:10488000294609A824F092F900231A4609A91948D3
:1048900015F016F9044609A820F015F82046002165
:1048A00026F00CFD044618B9134820F089FFE3E711
:1048B0002946012209A824F079F9214600226846F8
:1048C00020F07AFC6B460D4A0A4809A915F0F8F861
:1048D000039825F057FF09A81FF0F5FF0021204697
:1048E00026F045FB0546204625F04CFF2C46C3E745
:1048F00010360600FF7004003536060021710400F2
:10490000F8B5051E0C4606DC2949012021F08AF87D
:1049100000242046F8BD084625F00BFC0646A8B149
:1049200000222449204627F009F927F084FC0022C0
:1049300021490646204627F001F927F087FB30F091
:10494000080309D0102809D01C49DEE724B122460B
:104950001B49012021F066F8012400E002242946C9
:10496000204621F099FD07469EB12946204621F0B8
:1049700093FD0546134900201EF03EFC044610B18D
:104980000FB146B13DB92A463946204626F0C3FD4F
:10499000BEE73546EEE73A460B49204627F0A1F838
:1049A000002DB6D02A460949204627F09AF8B0E7EC
:1049B000CC3E0600EB3E06000A3F0600F83E06002D
:1049C0000F3F0600463F0600D04206004F3F06005C
:1049D00038B5044625F0ADFB88B1002209492046D0
:1049E00027F0ACF8054625F0EEFC10B1284626F07D
:1049F00039FA0446284625F0C5FE204638BD04464F
:104A0000FBE700BF511B0600F8B506460D460AB38A
:104A1000104626F025FE002D044603DA304626F027
:104A200021FA0544002C03DA304626F01BFA044430
:104A30001B2025F05DF825EAE57524EAE4740746B5
:104A400030B1A54204DA631B2A46314626F002F94A
:104A50003846F8BD00296FF00044E9DADEE7F8B522
:104A600005460C46C2B1104626F0FAFD20EAE07673
:104A7000002C05DA284626F0F5F9044424EAE4740B
:104A80001B2025F035F8074620B13346224629463B
:104A900026F0E0F83846F8BD6FF00046E8E7F8B5D4
:104AA00007460C46CAB1104626F0DAFD20EAE0754A
:104AB00024EAE474A542B8BF23464FF01B00BCBFF4
:104AC0002C461D4625F014F8064620B12B1B224625
:104AD000394626F0BFF83046F8BD6FF00040E5E7F4
:104AE00070B50D1E064606DA0B49012020F09AFF2C
:104AF0000024204670BD1B2024F0FAFF044615F167
:104B0000FF35F6D31FF0F4FA0028F2D131462046E3
:104B100026F0C8F8F3E700BFB83E0600F8B5064631
:104B20000F46154625F04FFC044698B1284625F05F
:104B30002DFB88B1284626F093FD0446384627F021
:104B4000D3FB054626F08EF9241A09D50024284601
:104B500025F018FE2046F8BD304626F083F9ECE734
:104B6000284626F07FF90719304626F07BF9874260
:104B7000ECDC2246012329463046F2F705FFB0FA65
:104B800080F46409E3E7F8B507460E46154625F0BC
:104B90001AFC044648B1304627F0A6FB002D064615
:104BA00005DA0024304625F0EDFD2046F8BD26F05C
:104BB00059F94419384626F055F98442F1DC0123AD
:104BC0002A4631463846F2F7DFFEB0FA80F464092F
:104BD000E8E72DE9F0418AB027F086FB0546E0B111
:104BE0000146002201A820F0E7FA4FF0FF3400262A
:104BF000DDE90183984514D3049825F0C3FDA6424E
:104C0000DABFA21B013200223146284626F04FF8B7
:104C10000446284625F0B6FD254628460AB0BDE8DC
:104C2000F08101A8039F20F076FA1FF0BBFC00285A
:104C3000DED107EB080336EA240628BF1E461C46D1
:104C4000D6E7000070B505460E4625F072FA58B951
:104C5000284625F025FA044630B92A460E49032095
:104C600020F0E0FE204670BD304625F062FA18B113
:104C70000A49012020F0D6FE25F055F80446002808
:104C8000F0D0284625F055FA0028EBD02A460449F2
:104C9000204626F00FFFE5E7293706005C370600BF
:104CA000A238060008B508B1036823B91B20BDE887
:104CB000084024F01DBF002126F0CAFCBDE80840D2
:104CC00027F0B8BB08B525F0AEFF08BD70B50546A6
:104CD0008AB01B200E4624F00BFF0446E0B12846A4
:104CE00025F071FBC0B1002E16DB3246294601A823
:104CF00020F062FADDE901239A420AD2059B03B152
:104D00009B5C8DF8033001220DF10301204626F053
:104D100021F8049825F036FD20460AB070BD37B55D
:104D200005461B2024F0E4FE044628B1294601A8CC
:104D30001FF033FE019810B9204603B030BD26F0B5
:104D400079FC27F083F901228DF803000DF10301AE
:104D5000204625F0FFFF01A81FF013FEEAE7000040
:104D6000F8B507460E4625F0E4F988B30022194944
:104D7000384626F0E3FE054625F025FB18B3284605
:104D800026F070F8002E01DD86420AD3114938461C
:104D900027F0D7F92C460025284625F0F3FC2046BD
:104DA000F8BD32460021284625F081FF31460446F1
:104DB0006FF00042284625F07AFF06490246384641
:104DC00026F08FFEE8E71B2024F092FE0446E3E77E
:104DD0000446E4E7511B06002DE9F041CB1D23F00A
:104DE000070300AFADEB030D134614466E460D46A8
:104DF00053F8048B0A463146C047A3692B44A3618C
:104E000063692B44636135441C34AE4202D1BD4614
:104E1000BDE8F081204616F8011B1FF01EFE20465B
:104E20001FF0EEFEF1E700002DE9F04792B002AF6F
:104E30000D46144680461BF0A9FC4FF001090646BA
:104E4000F91D284687F80790F3F79CFA002C824654
:104E500005DC002630464037BD46BDE8F0871FF030
:104E60004FF904F58073834204D93B49484620F04A
:104E7000D9FDEEE7E31D23F00703ADEB030D152E7F
:104E800002AD3CD1354B1B78D3B11222002107F182
:104E90000A00F1F747FAE3B2FB6007F108020023CA
:104EA0004FF040212E4887F8089087F809A07D61CF
:104EB000F8F718F8024618B12A49042020F0B2FD8C
:104EC0002146012021F0E8FA06460028C1D001461B
:104ED000002207F1080020F097FF2C4415F8011B71
:104EE00007F108001FF0B9FD07F108001FF088FE68
:104EF000A542F3D107F108001FF0DFFCAAE7002E5E
:104F0000A7D119493246404626F018FE814601468F
:104F100007F108001AF09AFA88B132461349404660
:104F200026F00CFE27F087F9FB79B8730093224630
:104F30002B465FFA8AF107F108001AF0DFF9B87B17
:104F400024F03EFE09490246404626F0B3FD49469C
:104F500026F0EEFAB4E700BF563606001C04032024
:104F600094F902208B3606009E360600A73606000E
:104F70002DE9F04F8BB002AF0C46164681461BF070
:104F800005FC4FF0010BF91D0546204687F807B0D8
:104F9000F3F7F8F90023824607F108013046BB60B9
:104FA00025F0A8FF0446002E47D0F0B9304623F084
:104FB00049FF8046B8601FF0A3F808F5807383426C
:104FC00007D93549584620F02DFD2437BD46BDE8A8
:104FD000F08F08F1070323F00703ADEB030D02ACDC
:104FE00042462146304624F055F8BE68002EECD0EB
:104FF000152D25D1294B1B78002BE6D0FD791422E5
:10500000002107F10C00F1F78DF9002D07F10C02DA
:10501000F6B20CBF202300234FF04021204887F830
:105020000DA03E61BC61F7F75DFF02460028CCD0C1
:105030001C49042020F0F6FCC7E70028C5D0D4E7BF
:10504000002DC2D118492A46484626F077FD06466B
:10505000014607F10C001AF0F9F988B12A46134904
:10506000484626F06BFD27F0E6F8FB79B87400930C
:10507000BA6823465FFA8AF107F10C001AF0A0F92A
:10508000B87C24F09DFD09490246484626F012FDF1
:10509000314626F04DFA98E7522F06001C040320F3
:1050A00094F90220FB3606009E360600A73606005D
:1050B000F0B591B00D4616461C461BF067FB142850
:1050C0009DF8587005D02F49012020F0ABFC11B09D
:1050D000F0BD16B90CB90F2403262B4B1B78F6B282
:1050E000E4B25BB92949ADF810306FF0FF02CDE9A9
:1050F000011201A8264A039216F05CF8FF2F03D094
:10510000002138461BF016FD284625F03FF880B1F7
:10511000284626F0A5FA22463146C0B2F8F77CF9B7
:10512000F2F712FFFF2FD2D0012138461BF002FD0B
:10513000CDE7284625F074F9E8B1802383F3118880
:105140000122294601A823F031FD01A81FF0E7FB49
:10515000054601A825B91FF0B6FB85F31188DFE7E6
:105160001FF003FF22463146C0B2F8F755F901A8F7
:105170001FF060FDE9E72A460649012020F052FCB5
:10518000CEE700BFCE3D060000040320A08601004C
:1051900000010800F63D0600F0B591B00D46164638
:1051A0001C461BF0F3FA14289DF8587005D03049BE
:1051B000012020F037FC11B0F0BD16B90CB9032462
:1051C00001262C4B1B7806F00F0604F00F045BB988
:1051D0002949ADF810306FF0FF02CDE9011201A8A6
:1051E000264A039215F0E6FFFF2F03D00021384630
:1051F0001BF0A0FC284624F0C9FF80B1284626F009
:105200002FFA22463146C0B2F3F71EF8F2F79CFEA1
:10521000FF2FD0D0012138461BF08CFCCBE728466D
:1052200025F0FEF8E8B1802383F311880122294696
:1052300001A823F0BBFC01A81FF071FB054601A8E3
:1052400025B91FF040FB85F31188DFE71FF08DFEC5
:1052500022463146C0B2F2F7F7FF01A81FF0EAFC80
:10526000E9E72A460649012020F0DCFBCEE700BF33
:10527000A63D060000040320A086010000010800EE
:10528000F63D0600F0B58BB004460D461BF07EFAE5
:1052900001AE07463246694620461BF085FA98B3B0
:1052A000009B059396E80F0006AC07C423807DB3EE
:1052B000296800292CDD0139284626F0C9F906465F
:1052C00025F06AF910B330461BF021FB044628464E
:1052D00026F009FF25F056FA304625F053FAFF2C48
:1052E00003D0002120461BF025FC05AA09492846C9
:1052F00023F0AEFC142F01D1F2F726FEFF2C03D0D1
:10530000012120461BF016FC0BB0F0BDFF24E3E7A3
:10531000FF24EAE71B3E03002DE9F041C0B00D4633
:1053200016460BA90CAA1BF03FFA002877D0FF2ED7
:1053300003D0002130461BF0FDFB284624F026FF59
:1053400080462846B8F1000F18D026F089F920A928
:105350008DF880000CAB084601220B9CA0479DF8FD
:10536000800024F035FC0446FF2E03D00121304696
:105370001BF0E0FB204640B0BDE8F08125F023F8AB
:105380000746002831D01B2024F0B2FB42460446D9
:10539000294602A81FF010FFDDE902239A4203D339
:1053A000059825F0EFF9DFE71EF0A2FE0028F7D1FF
:1053B00001AA694602A81FF0CFFB019D002DEBD08A
:1053C000802D28BF80250CAB2A4620A900980B9F72
:1053D000B8472A4620A9204625F0BCFC019B5B1B50
:1053E0000193009B1D440095E7E7284623F02AFD22
:1053F0000146012021F050F804460028B4D03A4676
:10540000014612A8CDE9107720F0FEFC0BAA054951
:10541000284623F01DFC12A81FF04FFAA4E704460B
:10542000A8E700BFD94D03007FB50C4605461BF029
:10543000ADF921460646684619F048FD98B1142E8C
:1054400013D1684615F0B6FE3CB301221549284633
:1054500026F0E0FA034618B1214625F0BFFF0346C7
:10546000184625F08FF904B070BD002EFBD19DF8D1
:105470000500FF2802D0012116F080F89DF80600F3
:10548000FF2802D0042116F079F89DF80700FF28C4
:10549000DAD0012116F072F8D6E70249284626F044
:1054A00050FEE0E79E3606002DE9F04300228DB065
:1054B0002449064626F042FB05AD0146284627F062
:1054C0004BFE1B22541E295D09B1144602E0224600
:1054D000002CF7D10CAB4FF001081C440DF124094E
:1054E00004F81C8C99E807008DE8070095E80F0088
:1054F00027F060FC08F1010807460028F0D10120E0
:1055000024F066FB10490246304626F0EAFA384697
:1055100024F05EFB0D490246304626F0E2FA38469A
:1055200024F056FB0A490246304626F0DAFA38469D
:1055300024F04EFB0749024630460DB0BDE8F0436B
:1055400026F0CFBA502B0600473E06004D3E06001F
:10555000543E0600E34D06002DE9F04F00229DB0B9
:105560000C469A49054626F0E9FA26F06FFDC0B2CE
:10557000772808D0612806D09549012020F052FAFA
:105580001DB0BDE8F08F204626F0AEFE064600288E
:10559000F6D025F067FC82460028F1D000228D4924
:1055A000284626F0CBFA26F051FD00228A49834690
:1055B000284626F0C3FA26F049FD002287490A90C2
:1055C000284626F0BBFA26F041FD00228449814698
:1055D000284626F0B3FA0DAC0146204627F0BCFD64
:1055E0001B22531EE15C09B1134602E01A46002B50
:1055F000F7D11CAA1A44099202F83C9C79490B93F2
:105600000022284626F09AFA26F020FD804600283F
:1056100041D014AFA0F120012022384615F072FBD2
:105620000B9B21465A1C15A82CF06EF9A0B10397CC
:1056300011AB93E807008DE8070094E80F0027F00E
:10564000B8FA804608B9684997E724F0C1FA654975
:105650000246284626F045FA0A9BA3EB0B039A451F
:10566000D84451DB1A46002130460A9325F01FFB2F
:105670004146834606F0BCFD584625F083F8B9F153
:10568000FF0F0A9B4BD15949012020F0CBF930463E
:1056900025F078F874E749F6E073CDE90503402377
:1056A000CDE9036311AF97E807008DE8070094E8A0
:1056B0000F0027F0BFFB0028E9D014AB039397E855
:1056C00007008DE8070094E80F0027F072FA0746FC
:1056D000149820F07F44504624F07AFA3D4902465F
:1056E000284626F0FEF9204624F072FA3A4902468E
:1056F000284626F0F6F9384624F06AFA3949024677
:10570000284626F0EEF9C2E73046414606F070FD25
:105710000AEB0B0024F05CFA2E490246F0E70A93EC
:10572000099B09F1010003F83C0C24F051FA2B49C4
:105730000246284626F0D5F90A9B6FF0004219462A
:10574000304625F0B4FA002349F6E072CDE905327F
:105750004023CDE903030DF14408814698E8070092
:105760008DE8070094E80F0027F064FB00288ED036
:10577000039798E807008DE8070094E80F0027F0EA
:1057800018FA0746149820F07F44504624F020FA77
:1057900010490246284626F0A4F9204624F018FABB
:1057A0000D490246284626F09CF9384624F010FAA6
:1057B0000C490246284626F094F9484625F052FB4B
:1057C0000446484624F0DEFF2046A3E7E34D0600EA
:1057D000713E06004D3E06008A3E0600473E06002A
:1057E000502B0600543E06008E3E0600AA3E0600E0
:1057F0002DE9F04F0022A1B00E466E49054626F075
:105800009DF926F023FCC0B2722808D06A49012015
:1058100020F008F90027384621B0BDE8F08F0022BB
:105820006649284626F08AF926F010FC80460028B2
:1058300000F0BD8000226249284626F07FF926F05C
:1058400005FC00225F498146284626F077F926F0BC
:10585000FDFB00225C498246284626F06FF926F0BF
:10586000F5FB002259498346284626F067F9014690
:1058700009A827F071FC1B22531E09A9C95C09B1B4
:10588000134602E01A46002BF6D120AAD31806933D
:1058900003F85CBCF30F059318BF202600273EBB1E
:1058A0007CE04FF0000846E012F8011BFF291CD0F5
:1058B0000598013300286CD00A296AD100221C46C1
:1058C000059237B91B20079324F012F9079B07466E
:1058D00030B1224610A93846079325F03BFA079BC2
:1058E000059AA1441AB91E1BD9E71C4654E020268C
:1058F000AAEB0904002C3DDCBBF1FF0FD1D0069BC5
:105900000BF1010B03F85CBC18AB03930DAB93E8F0
:1059100007008DE8070009AB0FCB27F04AF9189B69
:1059200023F07F4A8046504624F052F9254902462A
:10593000284626F0D6F8404624F04AF91F49024688
:10594000284626F0CEF8002024F042F91C490246F1
:10595000284626F0C6F8584624F03AF91A49024675
:10596000284626F0BEF8B8F1000F3FF454AF544675
:105970004FF00009202E3346A8BF20239C42A8BF29
:105980001C46224609EB080110A815F0BBF910AA25
:105990000023A34288DB3346002C92D1484624F0F2
:1059A00017F907490246284626F09BF833E70746D1
:1059B00031E700BFE34D0600593E0600543E0600A5
:1059C0004D3E06008A3E0600473E0600502B06006C
:1059D0004FF0FF31FFF70CBF21EAE171FFF708BF7D
:1059E0002DE9F0470022A4B0424926F0A7F805AC03
:1059F00001460546204627F095FB284624F0C2FEC6
:105A00001B22531EE15C09B1134602E01A46002B2B
:105A1000F7D124AA02EB03094FF001080CAD09F8F5
:105A20007C8C0DF1240A03959AE807008DE80700A5
:105A300094E80F0027F0BDF8FF238DF813300646D9
:105A4000002851D00C9921F07F4101390144424690
:105A50000DF1130015F056F900279DF813200C9B4B
:105A6000FF2A23F07F4302D0B8F1FF0F1FD100259A
:105A70000C9C24F07F44641B002C14DD412C28BFB7
:105A800040242246A91914A815F03CF914AA0023B1
:105A900012F8011BFF2925D001339C42F8D10022C6
:105AA0001D44002AE4D0E81924B0BDE8F08708F1CD
:105AB000010809F87C8C03959AE807008DE8070037
:105AC0001F4494E80F0027F074F8064678B10C994B
:105AD00021F07F410139014401220DF1130015F03D
:105AE00011F9BAE70122DBE707460546DBE7054681
:105AF000D9E700BF502B06002DE9F04F0C46A7B0A8
:105B000006466A49204624F0E5FF98B968492046D0
:105B100024F0E0FF50BB6749204624F0DBFF054638
:105B200038BB2246644901201FF07CFF284627B07D
:105B3000BDE8F08F4FF0720A604900201DF05CFB59
:105B400005460028F2D01C220021304625F0AFF88F
:105B50000DF11C0801460646404627F0E3FA1B21DA
:105B60004B1E18F803203AB10B4608E04FF0770AB5
:105B7000E2E74FF0610ADFE71946002BF0D126AAD1
:105B8000D3184F4905933246284601240EAE03F838
:105B90007C4C0DF12C0925F0A4FF039699E8070031
:105BA0008DE8070098E80F0027F003F80E9BBAF184
:105BB000770F074623F07F4B08D128B12846FFF71F
:105BC00073FC4FF0000B5F46002632E0BAF1610F24
:105BD000FAD1FF238DF81B30002FF5D00BF1FF31E8
:105BE000012239440DF11B0015F08CF89DF81B3093
:105BF000FF2B01D0FF2C45D10026ABEB0608B8F1F6
:105C0000000F16DDB8F1400FA8BF4FF04008424624
:105C1000F11916A815F076F816AA002312F8011B40
:105C2000FF2941D001334345F8D100221E44002A08
:105C3000E3D0204623F0CCFF22490246284625F037
:105C400050FF304623F0C4FF1F490246284625F086
:105C500048FF384623F0BCFF1C490246284625F081
:105C600040FF584623F0B4FF19490246284625F064
:105C700038FF504623F0ACFF16490246284625F06F
:105C800030FF53E7059B013403F87C4C039699E8F9
:105C900007008DE8070098E80F0026F08AFF0E9BAA
:105CA000074623F07F4B97E70122BFE78CCA060027
:105CB000A69B060078BB06002B3E06003B3E060076
:105CC000502B0600473E06004D3E0600543E06009F
:105CD0008A3E0600E34D060010B58CB005AC0146C7
:105CE000204627F01FFA0CAB13E907008DE80700E8
:105CF00094E80F0027F05EF80CB010BDF2F744B83E
:105D000026F0D4BE70B5002290B006460846114673
:105D100008F006FF09AC05463146204627F002FA96
:105D20000023CDE90533CDE9035310AB13E9070098
:105D30008DE8070094E80F0027F07CF80446284619
:105D400024F020FD204610B070BD2DE9F0418046C2
:105D500090B008460C4617461E4624F0EAF910B3E8
:105D600000221146204608F0DBFE00260546374695
:105D700009AC4146204627F0D5F90023CDE903536D
:105D8000CDE9057610AB13E907008DE8070094E82C
:105D90000F0027F04FF80446284624F0F3FC204675
:105DA00010B0BDE8F081204623F064FE0546DFE731
:105DB00030B58FB007AC01460025204627F0B2F978
:105DC000CDE903550EAB13E907008DE8070094E811
:105DD0000F0026F035FF044638B1294625F0C7F8F4
:105DE0000546204624F0CEFC2C4620460FB030BDA0
:105DF00070B58EB007AC16460D460146204627F01A
:105E000091F9CDE903560EAB13E907008DE80700C1
:105E100094E80F0026F014FF0EB070BD70B58EB080
:105E200007AC0E460146204627F07CF90023CDE959
:105E300003330EAB13E907008DE8070094E80F0069
:105E400026F0FEFE054668B104F044FC04462846F0
:105E500024F098FC1EB11DF09DFF24F093FC204619
:105E60000EB070BD0446FAE74FF0C04027F002B90B
:105E700013B50C461AF08AFC8DF80700093806287D
:105E800005D80DF107020349204622F0E9FF02B0D0
:105E900010BD00BF995E03000B78C1B2184619F01F
:105EA000B7BE00002DE9F04389B0984605460E467E
:105EB00017461AF06BFCA0F10903DBB2062B04466F
:105EC00032D8A0F10E03DBB2012B10D811F024FA66
:105ED00068B94FF0FF334FF41652CDE904238DF823
:105EE0001C00224B069304A9204611F0A5FC8DF856
:105EF00000401F4C1FB1304626F0F6F906466A46B0
:105F00002146304622F0ACFF17B1304624F03AFC6F
:105F1000B8F1000F05D069460D20A04769460A2058
:105F2000A04709B0BDE8F0830028FAD10246114924
:105F3000284625F003FE224681460F49284625F0D3
:105F4000FDFD04AD024649460446284619F0E2F834
:105F5000204624F017FC484624F014FC95E80F0076
:105F60006C4607C42370054CC4E700BF080001005D
:105F7000350E0500A23306009E360600ED09050029
:105F800000231A46FFF78EBF01231A46FFF78ABF88
:105F900000230122FFF786BF2DE9FF4705461AF0CF
:105FA000F5FB002204464049284625F0C7FD0022A3
:105FB00007463E49284625F0C1FDA4F10906824660
:105FC000002F4CD001463A46684619F0A3F89DF8D8
:105FD0000600FF2802D0002115F0D0FA9DF8070036
:105FE000FF2802D0002115F0C9FA9DF80400FF280F
:105FF00002D0002115F0C2FA9DF80500FF2802D05A
:10600000002115F0BBFAF3B2062B28D9002228494B
:10601000284625F093FD10B326F018F85FFA80F8B3
:106020000021404615F06EFD002019F007F881466A
:10603000A8B1414624F0D8FB804618B10146484635
:1060400026F00EF8484624F0A7FC20B9194B1A494F
:10605000586826F076F84946404625F069FA5146D8
:10606000384625F065FA1149284626F06AF8F6B256
:106070000D49284626F065F8062E12D8A4F10E0325
:10608000DBB2012B08D8204611F062F9FF22002173
:1060900020461AF02BFD04E0A4F10D03DBB2022B25
:1060A000F4D904B0BDE8F0879E360600A23306009E
:1060B000983D0600983400209D3D0600F0B585B05F
:1060C00005460F4614461AF061FB064684B922467F
:1060D0005449284625F032FD044622463946684692
:1060E00019F018F858B9204624F04CFB05B0F0BD63
:1060F000B4F80D3003F50073A4F80D30EDE7009807
:1061000023F066FD48490246284625F0EAFC9CB18A
:1061100022464449284625F0E4FCA6F10903DBB2F7
:10612000062B0ED8A6F10E03DBB2012BDED8694692
:10613000304611F081FBD9E73A49284626F001F8AC
:10614000EBE7002ED2D19DF80500FF2807D00121F2
:1061500015F014FA01219DF805001AF0EBFC9DF8EA
:106160000400FF280BD0052115F008FA602023F069
:10617000FFFD044660B92D4901201FF053FC9DF836
:106180000630FF2BB2D02A4901201FF04BFCADE7AF
:1061900002462849284625F0A4FC204624F064F84D
:1061A000002680F84060044611F046FA009B9DF8F6
:1061B0000A2084F85860C4E914369DF80830134466
:1061C0009DF80920B24218BF0133C4E9120184F8D6
:1061D000593001219DF8040015F094FC0446C8B123
:1061E00023F0F6FC14490246284625F07AFC0120EB
:1061F00018F024FF06460028C1D02A46214625F083
:10620000EBFB304624F0BEFA013C0C4B0C4A43F841
:106210002420B4E79DF804200A4901201FF002FC65
:10622000ADE700BF9E360600A2330600133D060010
:10623000703D0600393D0600983D0600E804032045
:1062400059F00400413D060010B50C461AF09EFAC4
:10625000A0F10903DBB2062B04D82146BDE81040AB
:106260001AF0DABF02490120BDE810401FF0DABB86
:10627000E83C06002DE9F74F9846012313600D69AD
:1062800007468A4616460DB10B68ED5C38782E2815
:1062900000F0FA805B2836D1012388F8093097F89E
:1062A00001B0BBF15E0F02D13368013333604FF0B0
:1062B000000907E02E2C19D12E2D08BF49F0010945
:1062C000013333603368FC5CF818002C00F0DE808A
:1062D0005D2CEFD101333360002388F80930BBF126
:1062E0005E0F14BF484689F0010019E0434601AA39
:1062F0005146FFF7BFFF3368019A49EA00095FFA88
:1063000089F91344DDE75C286CD102233360787887
:10631000642808D1A5F1300009288CBF0020012095
:1063200003B0BDE8F08F442806D1A5F1300009285C
:1063300094BF00200120F3E766286ED062286ED05B
:106340006E286ED072286ED0732805D1284603B00F
:10635000BDE8F04F1EF026B9532806D128461EF09E
:1063600021F980F00100C0B2DAE774285DD0762808
:106370005DD077280ED1A5F13003092B40F284803F
:1063800028461EF003F900287ED15F2D14BF00209F
:106390000120C5E757280CD1A5F13003092B12D9EC
:1063A00028461EF0F3F870B9B5F15F0018BF012060
:1063B000B6E730283DD0A0F13103082B05D8364987
:1063C00001201FF02FFB0020AAE778280AD1BB7814
:1063D00043B1FB7833B104233360F978B8781EF009
:1063E000C4F8C0B298F809302BB33368FA5C2D2A90
:1063F00021D13B445B785D2B1DD0A8F80A003068A2
:1064000001303060434601AA51463844FFF732FF5D
:106410003368019A1344336082E70C20E2E70820D6
:10642000E0E70A20DEE70D20DCE70920DAE70B20B1
:10643000D8E70020D6E798F8082062B1A5F141031B
:10644000192B98BF2035A0F1410398BFEDB2192B4D
:106450009CBF2030C0B2B8F90A30B3F5807F11D0AC
:10646000DBB22AB1A3F14102192A9CBF2033DBB26F
:106470004FF480729D42A8F80A20A4D38542A2D886
:10648000984255E7854281E7012049E70120034909
:106490001FF0C8FA204643E71B40060038400600BC
:1064A00082B02DE9F047ACB00C4634A9054681E82E
:1064B0000C001DF01DFE30B1002630462CB0BDE8AA
:1064C000F04702B070472B780BB17C2B43D1582298
:1064D00034A90DEB02002BF025FADDE93457DDF885
:1064E000DC9023F01DFC2368A2681A440646D21BE8
:1064F0003946284624F0DBFB00210446024630469C
:1065000025F06AFA204624F03DF90DF168080024D0
:106510004C450DDB384623F05BFB704902463046A4
:1065200025F0DFFA2A466E49304625F0C3FAC4E763
:1065300058F8041BD8F820202846521A24F0B7FB3C
:106540000134824602462146304625F045FA50463F
:1065500024F018F9DCE75E2B09D12368A268D34246
:10656000AAD11FF01BFC0028A6D0013507E0242B80
:106570001DD1D4E900329A4205F101050CD8502210
:1065800036A968462BF0CEF934AB0CCB2146284611
:10659000FFF786FF064690E74C2237A968462BF0A6
:1065A000C1F934AB0ECB284600F024FAF2E7282BD1
:1065B0000FD1379B2168A26834A80A44191D082B03
:1065C00040F8212000EB83014A63CADC0133379392
:1065D000C7E7292B0AD1379B002BC2DD34AA02EB77
:1065E00083032168A2680A441A63BAE734AB15AA88
:1065F00021462846FFF73EFE159FEB5DA3F12A02D8
:10660000012A804605EB07064ED801372F4450B9C2
:106610002B2B08D14C2237A968462BF083F934ABD9
:106620000ECB3846C0E7214616A81EF029FA5022A4
:1066300036A968462BF076F934AB0CCB16A9384650
:10664000FFF72EFF0646199824F09CF8D4E90023A2
:106650009A42BFF432AFB8F1000F3FF42EAF20469C
:106660001EF0B2FA34AB15AA21462846FFF702FE07
:106670002146804616A81EF003FA502236A9684625
:106680002BF050F934AB0CCB16A93846FFF708FFB6
:106690008146199824F076F8B9F1000FD6D030462B
:1066A00024F070F84E46D1E7D4E900239A420BD289
:1066B00050B120461EF088FA1FF070FB00283FF40E
:1066C000FBAE159B1D445AE74C2237A968462BF0B8
:1066D00029F934AB0ECB304666E700BF5A400600BE
:1066E000604006002DE9F047BCB00646084614AFEE
:1066F00025F0FAFD002253498046304625F01EFA67
:1067000025F0A4FC002205464F49304625F016FA34
:10671000044623F058FE48B92146404624F008FFBD
:1067200000242046A037BD46BDE8F087404624F04F
:1067300099FBA842F0D3204624F094FB00F1080313
:1067400023F00703ADEB030D0DF1500A421C514637
:10675000204625F079FE204624F014F869213046C1
:10676000FDF7F2FC4FF48072002387F85000A7F881
:10677000522041462A46384687F851307B65C7F893
:1067800048801EF019FD394607F124001EF078F903
:106790005022B9186846FD642BF0C4F807F1480987
:1067A00099E80C0007F124015046FFF779FE0446F2
:1067B000386B23F0E7FF38461EF006FA2CB9D7E90C
:1067C00000239A4205F1010514D3F86823F0DAFF9B
:1067D000404623F0D7FFCCB9022023F089F90025E9
:1067E0000446284623F0F4F916490246304625F0BF
:1067F00078F996E7394607F124001EF041F9502256
:10680000B9186846FD642BF08DF8C9E7672130465A
:10681000FDF79AFCA0B10021204624F019FF0022C8
:1068200080460A49204625F089F925F00FFC0546E7
:10683000404624F017FB0544404623F0A3FFD0E771
:106840000546CEE7D13C0600CA3C06005A40060089
:106850002DE9F84F04460D4623F0B5FD20B94FF061
:1068600000084046BDE8F88F23F05AFA8046002819
:10687000F5D01DB9214625F033F8F2E751492846F5
:106880001FF01EFE00285FD0002023F0A1F94E4922
:106890000246284625F025F921462846FFF722FF23
:1068A0000027064626B1304623F0FAFB8146D0B1D8
:1068B000304623F067FF002023F08AF94249024660
:1068C000284625F00EF9204624F0CCFAB842C8DB61
:1068D00039466FF00042204624F0E9F9014640466F
:1068E00025F04AF8BDE74946304624F0B1FE4A4655
:1068F00036498246304625F021F925F0A7FB81462E
:10690000504624F0AFFA8346504623F03BFFA9EBF4
:1069100007023946204624F0CAF90146404625F0D0
:106920002BF80BEB0907304623F02CFF384623F0F9
:106930004FF925490246284625F0D3F82146284636
:10694000FFF7D0FE0646ADE7284625F0CDFC814690
:1069500088B124F087FA0746204624F083FA0026FF
:1069600000F1010BABEB070A3546554522DC7FB938
:1069700025BB0135F9E70746EEE75D4612E0014623
:10698000404624F0ADFF304623F0FCFEEE19F0E760
:106990005545F2D001232A4649462046F0F7F4FF38
:1069A0000028E6D1AA1B3146204624F080F906468D
:1069B0000028E4D1484623F0E5FE52E75545F1D1E1
:1069C000F8E700BFC33C0600D13C06005A40060071
:1069D00038B5FFF787FE054650B123F061FB80F024
:1069E0000100C4B2284623F0CDFE04F0010038BDFA
:1069F0000446F7E784B0F0B59FB025AE054686E8BB
:106A00000E001FF0CBF968B9044620461FB0BDE860
:106A1000F04004B070475C2C03D16C78002CF4D0AB
:106A20003D4601352C78002CEFD07C2C05F1010778
:106A3000F1D1DDE9251215A81EF0BEFB27A95022D1
:106A400068462AF06FFF96E80C0015A93846FFF754
:106A500027FD0446189823F095FED6E737B505467E
:106A600001910B4848F2080123F050F9044660B147
:106A70002A46084925F01EF82846012301AA214686
:106A800019F0F0FD204623F07DFE03B030BD00BFBD
:106A9000436F0300A62E06002DE9F743054608467E
:106AA0000F46904623F060FB38B93A46254903204B
:106AB0001EF0B8FF03B0BDE8F083B8F1000F0BD0B3
:106AC00000222149284624F0A5FF0446E8B124F01D
:106AD000B5FD04461D4E01E01D4E444600223146E0
:106AE000284625F02BF8814688B93A463146284693
:106AF00024F0E0FFB8F1000FDCD028462146FFF774
:106B0000ADFF204623F03EFED4E78046E2E723F0C7
:106B100007FB38B13946484624F0E2FE484623F0E8
:106B200031FEE7E702216846CDE9009724F041FFF6
:106B3000314607460246284624F0BCFF384623F07B
:106B400021FEEBE755330600793306004B33060090
:106B50005033060010B500220446FFF79DFF204683
:106B6000BDE81040FDF740BC38B51546012204468B
:106B7000FFF792FF25B1002229462046FFF78CFF40
:106B80002046BDE83840FDF72FBC00002DE9F74F47
:106B9000054623F045FC044640B92A463449032003
:106BA0001EF040FF204603B0BDE8F08F31490020C1
:106BB0001CF022FB04460028F4D048F208012E48BD
:106BC00023F0A4F88146D8B122462C4924F072FF64
:106BD00023F0A6F82946824601A81DF0DEFE002615
:106BE0003546019880B9A81B22F0F2FF24490246DD
:106BF000204624F076FF52462249204624F071FFB9
:106C0000484623F0BFFDCDE724F014FD8046FDF794
:106C1000C5FA30B348F260011B4823F077F8074605
:106C2000284622F0D5FF002102468346384625F04B
:106C30007EF9584623F0A6FD22461049384624F036
:106C400039FF39464A464046FFF78EFF394624F061
:106C50006FFC404623F096FD01A801351DF091FE22
:106C6000BFE742462946504624F0B6FE0136F0E71B
:106C7000103606008B3C0600296D0300A62E060088
:106C8000803C0600863C06008D6C03002DE9F04137
:106C90000F46904613490022054624F04FFF25F089
:106CA000D5F9002204461049284624F047FF06463D
:106CB000B0B142463946013C24F08EFE204622F017
:106CC00087FF08490246284624F00BFF1CB93146CD
:106CD0002846FFF7C3FE3046BDE8F04123F052BD21
:106CE000BDE8F081803C0600863C060037B50546CD
:106CF00001910B4848F2080123F008F8044660B1FE
:106D00002A46084924F0D6FE2846012301AA214636
:106D100019F0A8FC204623F035FD03B030BD00BFBC
:106D20003D6F0300A62E060038B500220D46094926
:106D3000044624F003FF58B123F024FD2046054902
:106D400025F0FFF929462046BDE83840FFF7CEBFC1
:106D500038BD00BF863C06002DE9F04385B00646ED
:106D600001914149144625F0ECF94049304625F09F
:106D7000E8F900223E49304624F0E0FE3C49054651
:106D8000304625F0DEF9204623F0CAF9074660B305
:106D9000214603A81DF001FE0024039878B91CF0D9
:106DA000F9FF804658B301462846FFF79FFF2A4661
:106DB0002146404624F0AFFB05B0BDE8F08324F047
:106DC00039FC01AB0122314681461AF08BFD804629
:106DD00017B923F0D7FCA046484623F0D3FC03A8FC
:106DE0001DF0CFFD00274446D7E7002CD7D0204622
:106DF00001AB012231461AF075FD0446CFE74DB3D1
:106E00002046FDF7CBF950B348F20801194822F0AB
:106E10007DFF48F208010646174822F077FF074633
:106E2000A6B198B12A461549304624F043FE2A46B9
:106E30001249384624F03EFE012231462046FFF733
:106E40002BFE424639462046FFF726FE394630469D
:106E500024F06EFB2946204624F06AFBACE721466D
:106E60002846FFF7FBFDF5E74B33060050330600DD
:106E700014C006005D6A0300ED6C0300A62E060038
:106E8000294B2DE9F047B2F10009284E08BF1E46F4
:106E90000D4600223146804624F050FE044670BB69
:106EA00002462349DFF888A0404624F047FE044606
:106EB0004CB9B9F1000F25D12A461E490120BDE881
:106EC000F0471EF0AFBD00223146204624F036FECA
:106ED0000746024648B129462046FFF73DFF2146B6
:106EE0003846BDE8F04724F023BB5146204624F045
:106EF00025FE0746204623F045FC3C46D8E7B9F17D
:106F0000000F05D02A460C49404624F0D3FD4CB171
:106F1000404622462946FFF71FFF2046BDE8F047BE
:106F200023F030BCBDE8F087503306004B33060039
:106F300014C0060082330600793306000022FFF7F2
:106F40009FBF0122FFF79CBF2DE9F74F10F074FBA4
:106F50008946074622F0A0FB834610F06DFB804671
:106F60008A4622F0E0FE0446002800F0A680564B38
:106F700056495868002224F0E1FD0546002800F03B
:106F8000A08023F0E5FC0646284623F0FBFB002307
:106F9000012142F6E0624E484D1EC5EB0515054441
:106FA000B5F80D00800611D00133284601910093F9
:106FB00023F050F9DDE9003142F6E06230B1286893
:106FC0000F250E30B0FBF5F001440344013191422E
:106FD000E1D9B018C01A9D1B22F0FAFD3D490246C6
:106FE000204624F07EFD284622F0F2FD3A49024672
:106FF000204624F076FD42F6E06022F0E9FD3749B4
:107000000246204624F06DFD304622F0E1FD2F4976
:107010000246204624F065FD584622F0D9FD30494D
:107020000246204624F05DFDB8EB07006AEB09013B
:1070300029F036FF00222B4B29F060FF2A4B00225B
:1070400029F05CFF41EC100B22F0B0FD274902460D
:10705000204624F046FD0F2022F0BAFD24490246C6
:10706000204624F03EFD234822F0B2FD224902468C
:10707000204624F036FD002022F0AAFD1F490246DA
:10708000204624F02EFD1E4822F0A2FD1D49024696
:10709000204624F026FD4FF0C04022F099FD1A4909
:1070A0000246204624F01DFD4FF4801022F090FD92
:1070B00016490246204624F014FD204603B0BDE8E0
:1070C000F08F064663E700BF98340020083C0600B6
:1070D00004350020103C0600153C06001B3C060051
:1070E000213C060000408F400000B03E243C0600DA
:1070F0002B3C0600C0440320353C0600453C0600FE
:1071000030780700513C0600623C0600733C0600E4
:1071100010B522F008FE0446314824F01EF931492A
:107120000246204624F0DDFC2F4824F016F92F49B2
:107130000246204624F0D5FC2D4824F00EF92D49B6
:107140000246204624F0CDFC4FF4801022F040FD92
:1071500029490246204624F0C4FC4FF4000022F0E6
:1071600037FD26490246204624F0BBFC022022F0CF
:107170002FFD23490246204624F0B3FC4FF40000C3
:1071800022F026FD1F490246204624F0AAFC4FF4B7
:10719000802022F01DFD1C490246204624F0A1FC5F
:1071A00004F084FA19490246204624F09AFC03F0C0
:1071B00087F917490246204624F093FC154824F02D
:1071C000CCF815490246204624F08BFC134822F0E7
:1071D000FFFC13490246204624F083FC204610BDE4
:1071E000843B0600BB3B06008C3B0600953B06003B
:1071F000A03B0600AA3B0600B33B0600B03B0600DE
:10720000B93B0600C33B060013710600CB3B0600EA
:10721000D23B0600DA3B0600FA3B0600D0330020E2
:10722000023C060038B50849054600201BF0E4FF83
:10723000044638B1284622F079FD0449024620462A
:1072400024F04FFC204638BD413A06009D3F060021
:107250002DE9F74F0D4603210446CDE9002314F034
:107260008DF94FF0000B4FF0010A4FF08008D9461E
:1072700015F1FF3502D203B0BDE8F08F009B0AEA9A
:107280000306019B0BEA030756EA070316D088F3AF
:1072900011880021204613F071FD0A2010F0ACFA8D
:1072A0000121204613F06AFD89F31188372010F080
:1072B000A3FA1AEB0A0A4BEB0B0BD9E788F31188F8
:1072C0000021204613F05AFD412010F095FA0121CB
:1072D000204613F053FD89F311880520E7E710B429
:1072E0000C7802460023204608215DF8044BFFF786
:1072F000AFBF2DE9F8430D460321074614F03EF9D0
:10730000002401264FF08008A14615F1FF3502D276
:107310002046BDE8F88388F311880021384613F031
:107320002DFD032010F068FA0121384613F026FDE8
:107330000A2010F061FA384610F068F900B13443C1
:1073400089F31188352010F057FA7600DDE710B583
:107350000321044614F012F90021204613F00EFD1B
:107360004FF4FA7010F048FA0121204613F006FDA0
:10737000502010F041FA204610F048F904464FF42E
:10738000D27010F039FA84F00100C0B210BD0000D4
:1073900008B50022034924F0D1FBBDE8084019F0EC
:1073A0000BBB00BF9D3F06002DE9F04F8BB00C4694
:1073B000FFF7EEFF064619F009FB28B94FF0000869
:1073C00040460BB0BDE8F08F22F0AAFC80460028B2
:1073D000F4D0631EFF2B28BFF0242246E317CDE92B
:1073E00000234FF000093046FFF7B1FF0028E7D037
:1073F000DDE9002308213046FFF72AFF012400259C
:10740000AA46274601213046FFF773FF01215FFAA4
:1074100080FB3046FFF76DFFBBF1010FC0B22BD1EF
:1074200001283AD1402FCBDD9DF80C30002BC7D07E
:1074300005AC0DF10C090025A34619F8017B3809AC
:107440001CF068FE207007F00F001CF063FE013591
:10745000082D607004F10204EFD1002358468DF826
:10746000243023F07AFF0146404624F085FAD146C5
:10747000BAF1000FA4D0B6E70AAB2B44834513F84A
:107480001C3C2DD14F4524DA1C4214BF4FF0010B98
:107490004FF0000BBBF1000F21D00AAB2B444FF093
:1074A000010B13F81C3C23430AAA2A44012102F8C9
:1074B0001C3C30465A4600236400FFF7C9FE14F016
:1074C000FF0404BF01350124072D07F1010799DDF1
:1074D000A8E70CBF4FF0010B4FF0000BDAE7BA46FC
:1074E00023EA0403E0E770B58EB00C46FFF750FFC7
:1074F000064619F06BFA68B3204622F047FE18B32F
:10750000204624F0ADF80146054601201EF0C4FFD8
:10751000044650B10146002268461EF075FC15F184
:10752000FF3505D268461DF0C8F920460EB070BD83
:1075300008213046FFF7DDFEC1B268461DF08DFA26
:1075400068461DF05DFBEAE708213046FFF7D1FEF3
:1075500022F03EFB0446E8E737B50D461446FFF738
:1075600017FF8DF8070019F031FA80B10DF107020D
:107570000C49284621F074FC9DF807004CB101210C
:1075800013F0FCFB01219DF8070013F0F7FF03B097
:1075900030BD042113F0F2FF01219DF8070013F024
:1075A000EDFBF4E7DF72030010B5FFF7F1FE0446D0
:1075B00019F00CFA38B12046CC2200230821BDE88E
:1075C0001040FFF745BE10BD2DE9F0418AB00C46D2
:1075D000FFF7DEFE054619F0F9F940B1204622F02A
:1075E000F2FE38B92246264903201EF01BFA0AB0E3
:1075F000BDE8F081204623F035FC1028F2D1284662
:10760000FFF7A5FE2146002201A81DF0D5FD0024AC
:1076100027462646A04601A81DF07DFD8DF80000F6
:1076200001A81DF078FD00231A468DF801001021F5
:1076300068468DF802801DF0AFF8A4F12002C4F175
:107640002003A14000FA02F220FA03F31143A04004
:1076500008341943402C47EA000746EA0106DAD10C
:10766000049823F08FF82846552200230821FFF7BD
:10767000EFFD3A46334621462846FFF7E9FDB6E7D7
:10768000493A060010B5FFF783FE044619F09EF94B
:1076900020B12046BDE81040FFF759BE10BD10B123
:1076A000012124F079BA70472DE9F74305460F46CA
:1076B000914622F059FD044640B92A465749032015
:1076C0001EF0B0F9204603B0BDE8F083284622F052
:1076D000F0FC60B3A988286822F018FB0446002853
:1076E000F0D0294668461DF058F9009D7DB3B5F8E5
:1076F0000D3003F50073A5F80D30284623F09AFFEE
:107700008046284622F0B5FED8B1B8F1000F2AD045
:107710000121284624F040FA064630B101462046B1
:1077200024F066F8304623F02DF801260AE02846BA
:1077300022F010FD002814BF0820072022F0D8F9FD
:10774000CCE706464146284623F0F2FE6EB9B9F171
:10775000000F0ED1009D002D45D13A4630492046FC
:1077600024F0A8F9AEE74646ECE768461DF009F9B3
:10777000BBE7494601A81DF010F901980028E9D09F
:1077800023F058FF009D064665B1B5F80D3003F5AE
:107790000073A5F80D30284622F06BFE40B928464C
:1077A00022F0F0FF32460021204624F0C0FB13E017
:1077B00001220021284624F05BFB3146804623F05D
:1077C0000DFE4146204624F013F82846414623F09A
:1077D000AFFE68461DF0D5F8304622F0D3FF01A871
:1077E0001DF0CFF8C9E7B5F80D30012203F500739D
:1077F000A5F80D301146284624F03AFB064630B174
:107800000146204623F0F4FF304622F0BBFF284615
:1078100022F0B8FF68461DF0B4F89BE75D3406001F
:10782000A62E06002DE9F04F93B0814602AF104618
:107830008A46164622F0F4FD0446002856D030460B
:1078400023F02FFBB0F5807F044680460AD902461C
:107850002B4901201EF0E6F8002420464437BD469F
:10786000BDE8F08F8300DA1D22F00702ADEB020DB8
:1078700002AD2A462B440021934219D10122314600
:10788000381D21F093F9381D1DF049F898B9381DBD
:107890001DF019F800231946CDE9008552464846E7
:1078A0001FF0AAFF29460446404623F017FED4E7FE
:1078B00042F8041BE0E7381D1CF0DAFF064622F010
:1078C00075FE60B1304623F0CBFEB0F1000B06DB55
:1078D0005C4504DD381D1DF0B6FB45F82B00304635
:1078E00022F050FF381D1DF0A5F9CCE72EB132462D
:1078F000044901201EF096F8AFE7B0463546C9E7C7
:10790000D9330600223406002DE9F34704460D461C
:1079100022F02AFC30B9444903201EF083F802B05B
:10792000BDE8F087284622F01FFC0028F3D020464F
:1079300022F0BFFB0646284622F0BBFB86420AD057
:10794000284622F0B6FBB4F80D30002842D043F0B0
:107950004003A4F80D30204622F0FCFB06462846E2
:1079600022F0F8FB86420BD0284622F0F3FBB4F855
:107970000D3023F03F0380B343F00803A4F80D302B
:1079800000222A49DFF8A490DFF8A4A0204624F0C2
:1079900041F8002226490746204624F03BF80646D7
:1079A000204624F0E9FB294601A81CF0F6FF019DC2
:1079B000B5B91FB13946204623F01AFF384622F0E8
:1079C000E1FE1EB13146204623F012FF304622F080
:1079D000D9FEA4E723F04003BBE743F00703CDE75C
:1079E000B5F80D3003F5007301A8A5F80D301CF0B3
:1079F000C8FF4946284623F06DF888B95146284605
:107A000023F068F860B90121284624F0C5F88046C3
:107A100030B10146204623F0EBFE404622F0B2FE94
:107A2000284622F0AFFEC2E794340600B2340600C6
:107A300060BC06002DE9F74305460F46144622F0C8
:107A4000D5FD30B9354903201DF0ECFF03B0BDE88A
:107A5000F083384622F0B7FC08B93149F3E72046F5
:107A600022F082FB28B9204622F0ADFC08B92D494E
:107A7000E9E739462C4823F02BF980460028E5D069
:107A800001460122284624F07BF90646404622F0B2
:107A900079FE304623F0CEFD804620BB214630469D
:107AA00023F09CFC3146404623F042FD1F493846F6
:107AB00023F010F80028C9D000221D49284624F0E0
:107AC0003DF8019022F07FFC48B11A492846012375
:107AD00001AA18F0FFFD1649284624F032FB019850
:107AE00022F050FEB2E722F01BFB20B121464046B7
:107AF00023F0F6FED6E722F013F94146814623F043
:107B0000EFFE2146484623F0EBFE4946304623F07F
:107B100065FC484622F036FEC4E700BFAC380600DC
:107B2000E33806001A39060072390600742F060081
:107B3000511B0600151B0600F8B5064608461446FC
:107B40001F4623F00AFC39460546204622F0DEF89F
:107B50002946044602463046FFF76CFF2946204678
:107B6000BDE8F84023F0E4BC73B505460C4622F0AE
:107B70003DFD20B9214903201DF054FF1AE02046A5
:107B800022F021FCC0B121461D4823F0A1F8064691
:107B900080B101460122284624F0F2F8044630461E
:107BA00022F0F0FD34B12846214624F059FA20464F
:107BB00022F0E8FD02B070BDF4B9294601A81CF01E
:107BC000ECFE104E019C002CF4D0B4F80D3003F5FF
:107BD000007301A8A4F80D301CF0D3FE0122314639
:107BE000204622F06FFF18B12146284624F038FACB
:107BF000204622F0C7FDE5E70349BCE7AC380600A4
